:020000040800F2
:100000000832002099890308A51F0308A71F0308C9
:10001000A91F0308AB1F0308AD1F03080000000061
:10002000000000000000000000000000AF1F0308F7
:10003000B11F030800000000B31F0308558B03081D
:10004000598B03085D8B0308618B0308658B0308DC
:10005000698B03086D8B0308718B0308758B03088C
:10006000798B03087D8B0308818B0308858B03083C
:10007000898B03088D8B0308918B0308958B0308EC
:10008000998B03089D8B030809210308A58B03089E
:10009000A98B0308AD8B0308B18B0308B58B03084C
:1000A000EF200308BD8B0308C18B0308C58B030831
:1000B000B51F0308CD8B0308D18B0308D58B03082C
:1000C000D98B0308DD8B0308E18B0308E58B03085C
:1000D000E98B0308ED8B030805210308F58B030862
:1000E000F98B0308FD8B0308018C0308058C0308BA
:1000F000098C03080D8C0308118C0308158C030868
:10010000198C03081D8C0308218C0308258C030817
:10011000298C03082D8C0308318C0308358C0308C7
:10012000398C03083D8C0308418C0308458C030877
:100130000020DFF8F41955222DE9F04FDFF8EC89A3
:10014000DFF8EC79A8F8960AC8F8A80EC8F8A40E4B
:10015000C8F8A00EC8F89C0EC8F8980E0860386061
:100160004FF6FF79DFF8CC19DFF8CCB9DFF8CC49CE
:10017000DFF8CC59086081B0DFF8C81908604FF08B
:10018000160ADFF8C4190860DFF8C0190860DFF844
:10019000C0190860C8F8100BC8F8200FDFF8B419B0
:1001A00008803020C8F8240FC8F8E89E0020C8F85E
:1001B0001C0FC8F8EC0EC8F8F00EC8F8F40EC8F81A
:1001C000000FC8F8040FC8F8080FC8F80C0FC8F8DB
:1001D000100FC8F8140FC8F8180FC8F8980FC8F80F
:1001E000280FC8F8E49EC8F8F89EC8F8FC9E0021C5
:1001F000DFF86409816481630220DFF860190880F8
:100200005521DFF85C090180BF214180892181806F
:100210008E21C180BF210181DFF848190988418101
:10022000DFF844090280BF22428041818922828016
:100230008E22C280BF2202810AF002FC0AF09BFDDE
:1002400000200AF0CFFCABF8000026882888B042D6
:100250000CD3B0B20AF0C6FCB6B22BF81600761C6E
:100260000CF066F82888B1B28842F2D24FF47A7066
:1002700013F035FCAD1CA41CBAF1010AE5D114F051
:100280000DFB14F019FC0AF013FE0AF011FE0AF03F
:1002900072FD10F0C3FBD8F8E40A00EB80014800BF
:1002A000BBF8D0100329B4BFDFF8C018DFF8C018BE
:1002B00001EB8000006AC8F89C0DBBF8D400C8F8B8
:1002C000C00F00F029FB00F059FC00F0FCFB00F02F
:1002D000AFFF01F03DF801F0F0F805F0CDFCD8F8E3
:1002E0009C0EC0F30010A0B900F016FB00F0A0FFB8
:1002F00000F0F8FF01F012F901F0DFF801F0BAF9AF
:1003000001F089F900F0F0FD0020C8F8180BC8F8DA
:10031000140B01F041FCBBF8E815DFF85838481E13
:100320008041C043C00FA8F8500ABBF8D000032892
:100330000CBF40F219204FF49B70A8F8520A00201D
:10034000A8F8540AA8F8560A0320C8F8E00E38683E
:1003500040F400703860BBF8C211A8F89A1ABBF8D4
:10036000C4110A29A8BF00211980A8F89C1A19886D
:1003700001290AD140F002003860DFF8AC17DFF83D
:10038000A807006840F0040008606420DFF81CAB98
:10039000DFF8E427AAF800000020A8F8940ABBF8C8
:1003A000E2004844C8F8C40EC8F8C80EBBF89E1155
:1003B000BBF8360102291BBFBBF83811002948449D
:1003C000A9EB0000C8F8CC0E0023BBF8E400DFF86E
:1003D000E01A0880BBF8E600DFF8D81A0880002091
:1003E000DFF8D41A0880BBF8D007DFF8D01A0880ED
:1003F000DFF8CC0ADFF8CC1A20F8023B21F8023BE8
:1004000022F8023B0123C8F8AC3E002320F8023B4F
:1004100021F8023B22F8023B20F8023B21F8023B84
:1004200022F8023BD8F8AC3E9B1C0B2BC8F8AC3E24
:10043000EBDBBBF8E804B0F57A7F38BF4FF47A7095
:1004400004D3BBF8DE10814238BF0846C8F89C0FC1
:10045000DFF8747AD8F8100FDFF8706ADFF8704AA6
:10046000DFF8705A40F01000C8F8100F40F2334027
:100470000AF0B8FBBBF8D0170229DFF85C1A18BFE6
:10048000002008804FF485600AF0ACFBDFF84C1ABE
:1004900008800020DFF8481A0880BBF8B601D8F8B9
:1004A000101F60F34921C8F8101FBBF8CA11D8F813
:1004B000100F02290CBF40F4806020F48060C8F85F
:1004C000100F0020C8F8D80A13F04CFDD8F8180F08
:1004D00040F04000C8F8180F24E000BFB0F5637F7B
:1004E00002D1BBF818073880B8F8AA0A012813D13E
:1004F000B8F8620AB0F57A7F0EDD0020A8F8AA0AE3
:100500004FF4A360D8F8481540448847D8F89C0EAB
:1005100040F01000C8F89C0E01F064FA16F004FDDB
:1005200016F076FDD8F8EC0EC0F3800020B12888D4
:1005300001001CBF484428802088C00602D5A08C3A
:10054000002105E0D8F81805A18CC1EB4000C117C7
:10055000C8E90001B8F88E0A1428BCBF401CA8F8EE
:100560008E0AB8F8900A1428BCBF401CA8F8900A5C
:1005700005F0BCF907F0C2FE0BF0DAFE98F8580A55
:10058000012818BF00200CF0FFFC0CF0E7FA17F070
:10059000B9F917F02FFC1AF041FB13F089FA09F0B2
:1005A00079FB1CF07AF8B8F88E0A142819DBD8F811
:1005B000100FC0F3001090B9BBF8460800281CBF0C
:1005C000B8F8940A02280AD0032818BF0C2806D0CD
:1005D000092818BF062802D021F0DEF801E01CF03F
:1005E000EDF9B8F8600A012804BF98F8580A012804
:1005F00004D113F08CF90020A8F8600A1BF0F8FE73
:100600001FF0A6FA15F0CEFD07F0DEFE08F0F3FAB3
:10061000D8F8581DD8F8D40F012904BFD8F8641DA4
:1006200000290AD1D8F8D81F884207DAD8F8EC1E7A
:10063000C1F3402111B1401C00E00020C8F8D40FE4
:1006400009F098F822F056FB3088002801BFDFF847
:1006500094080088012814F04DFAD8F8E00E48B943
:10066000D8F8B80E42F210714843BBF8DE1090FB88
:10067000F1F00BE001280BD1D8F8B80E42F210715E
:100680004843BBF8DE1090FBF1F04042ABF8A00FFE
:1006900008F03AFCD8F8A00EC0F3400008B91FF0EB
:1006A000B1FB05F0E9FA00F069FAD8F89C0EC0F346
:1006B0000010A0B900F030F900F0BAFD00F012FE11
:1006C00000F02CFF00F0F9FE00F0D4FF00F0A3FFD3
:1006D00000F00AFC0020C8F8180BC8F8140B01F051
:1006E0005BFA24F03DF9D8F8140FD8F8141FC0F3C2
:1006F000802080F0010060F38A21C8F8141F00F008
:100700002CF8DFF82414BAF800000968C1F380015E
:10071000012808BF002912D1BBF8020041F288313C
:100720004843D8F8181590FBF1F0B8F8A41A82B233
:100730009142BFF4D9AEA8F8A40A3A80D4E60022C8
:100740000029A8F8A42A7FF4CFAEB0F5A77F7FF4E4
:10075000C5AEDFF8F00B0068C5E62DE9F041DFF823
:100760007057DFF8C843B5F800C0D4F81805B4F8DE
:10077000A68AC117A0FB0867D4E9002301FB08770C
:100780007F005FEACC6147EAD6770CD512EB4602D0
:100790007B414000121843EBE073A88C0021101A33
:1007A00063EB010106E0A88C002110EB46007941C3
:1007B00010185941C4E90001DFF8F006008802284A
:1007C00001BFDFF864030068C0F3800000280FD188
:1007D000D4E900014822002324F050F9DFF8681B17
:1007E0000A88824208D208800888DFF8DC1602E016
:1007F0000020DFF8541B08800020C4E90000A4F8A2
:10080000A60ABDE8F08130B5CB4CC84DB4F8BE03A4
:1008100081B024F0D3F9B4F8C00324F0D2F9B4F8CD
:10082000B60324F0C8F9B4F8CC0024F0CDF9B4F83C
:10083000400624F0CCF9B4F8420624F0CBF9B4F821
:10084000440624F0CAF9B4F8460624F0C9F9B4F80D
:10085000480624F0C8F9B4F84A0624F0C7F9B4F8F9
:10086000540624F0C6F9B4F86C0624F0C5F9B4F8BF
:100870006E0624F0C4F9B4F8720624F0C3F9B4F893
:10088000CC0624F0C2F9B4F8CE0624F0C1F9B4F8CD
:10089000D00624F0C0F9B4F8D20624F0BFF9B4F8B9
:1008A000D80624F0BEF9B4F8DA0624F0BDF9B4F89D
:1008B000DC0624F0BCF9B4F8DE0624F0BBF9B4F889
:1008C000E00624F0BAF9B4F8EE0624F0B9F9B4F869
:1008D000F00624F0B8F9B4F8F20624F0B7F9B4F849
:1008E000F40624F0B6F9D5F8CC1CD5F8C80C24F0E1
:1008F00049FBD5F8C01FB4F8D400062918BF062854
:1009000008D1814206D0C5F8C00F01B0BDE8304023
:1009100010F002BD01B030BD70B5874EDFF8444D18
:10092000B6F8EE00B6F85416804D01280CBFB6F8A4
:10093000DE0041F2883025F06BF9014611224FF4B8
:10094000A01025F0ADF9E062C822B6F85406C0EB5D
:100950000011C800B6F84A16B0FBF1F0C821B0FB90
:10096000F1F1A6F84816206302FB110060636528C8
:10097000B6F8481626BF4800801C4800A6F848066E
:10098000DFF8E41CB6F848060228BCBF0220A6F82F
:100990004806B6F844060C22000525F081F9C5F892
:1009A000280D0D22B6F84606DFF8C01CC00325F05E
:1009B00077F9C5F8380D6421B6F8540625F088F9A2
:1009C000C5F8300D0B22DFF8A81C25F069F9A060EE
:1009D00001464FF4002025F07BF9C5F8340D01469F
:1009E000D5F8280D0C2225F05BF9D5F8381D0C221E
:1009F00025F056F920611022D5F8341DD5F8280DC0
:100A000025F04EF96061D5F8381DD5F8280D25F090
:100A1000A7F9C5F83C0D0C22D5F8341D25F040F996
:100A2000C5F8400D0C22D5F8341D206925F038F9A1
:100A3000D5F8341D142225F033F9A0614FF42001BC
:100A4000B6F86C06000525F043F90146D5F8380DD7
:100A50000C2225F025F9E0614FF0C071606925F0A6
:100A6000C7F920620C22D5F8280D6062D5F8341D34
:100A700025F016F901460C22DFF8640E25F010F976
:100A8000A0624FF48010D5F8381D25F021F9E06000
:100A90004FF48010D5F8281D25F01AF920604FF08A
:100AA0008070D5F8501125F05BF9C5F82C0D4FF08A
:100AB0008070A96E25F054F96060FFF7A4FEBDE8D0
:100AC000704004F0F9B970B51B4D234CB5F87406AD
:100AD0004FF44811C00325F0FBF8144EE065D6F83A
:100AE000381D25F0F5F8E065E88A0105B5F8D00075
:100AF0000328B9BF0C2299200C22E62025F0D0F85B
:100B0000D6F8281D25F02CF9206600202063E0622D
:100B100043F203002065DFF8400E60650020E063CB
:100B20002064606470BD00004821002000000020A7
:100B3000442100208C5E002038430020D49102081C
:100B40007C910208905E00205C5C0020985C002094
:100B5000E86300207A5C0020145D00201E21002044
:100B6000D020002000210020E0200020D0C7020873
:100B7000C4CB020824210020A020002070B5DFF89B
:100B8000AC46DFF8C857B4F8860A002804BFB5F8A9
:100B90004006002840F06681D4F8941ED4F8500D29
:100BA000002940F0C080B5F8D4100A46062A26D1A4
:100BB000B5F83211C4F8541DB1F57A6F05DBB5F8FC
:100BC0005626D4F8B83E9A4202D34FF47A6104E034
:100BD000B1F5FA5F03DD4FF4FA51C4F8541DD4F8AF
:100BE0009C1EC1F3001111B94FF47A609BE0D4F858
:100BF000541D01F10A028242C0F28D808DE000296D
:100C000018BF012A38D1B5F85616D4F8B82E91423B
:100C10000AD340F6C33240F6B8319042C4F8541DAE
:100C200079DA40F6AE327AE0B5F83211C4F8541DE4
:100C300040F6C4129142B8BFC4F8542D15DB41F6FA
:100C400059329142A4BF41F65831C4F8541DB5F849
:100C5000BE140329A2BFD4F8541D41F2514291425F
:100C6000A4BF41F25041C4F8541DD4F8541D01F101
:100C70000A0282424FDB50E0B5F83E11012952D002
:100C8000B5F83211C4F8541DB1F5487FBCBF4FF41C
:100C90004871C4F8541D032A1CBFB5F8121103296A
:100CA00016D1D4F8541D42F229329142A4BF42F227
:100CB0002831C4F8541DB5F8BE140329A2BFD4F8D6
:100CC000541D41F2717291421FDB41F270711AE0C2
:100CD000B5F8BE24B5F80215032A0ADB01290AD1AA
:100CE000D4F8541D41F6912291420EDB41F6902139
:100CF00009E0012909D1D4F8541D42F2351291427C
:100D000003DB42F23411C4F8541DD4F8541D01F130
:100D10000A02824201DA0A3805E0A1F10A02904291
:100D2000B4BF0A300846DFF8B81CC4F8500D91FB78
:100D3000F0F3B5F83E1101290AD1B5F8D410022913
:100D400018BF032904D1D4F89C1EC1F3001109B9BE
:100D5000C4F81835B5F87016D4F8B82E49420B2AE5
:100D600038BF0021A4F83C15D4F89C1EC1F3001133
:100D700021B9D4F81815DFF8102E118025F040F8AD
:100D800001464FF07E5025F055F8C4F8D40CB5F864
:100D90003E0101280AD1B5F8D400022818BF032863
:100DA00004D1D4F89C0EC0F30010A0B9B5F85406D5
:100DB000642124F02DFF0646D4F8D41C4FF0974050
:100DC00025F0B6F825F020F901461122304624F02E
:100DD00067FFC4F86C0700F02BFA00F0B9FAD4F8FA
:100DE000180100EB80014800C4F86803C4F8A003B0
:100DF0003222D4F87001C4F8D80300EB8001490016
:100E0000C4F82C13C4F81004C4F84804C4F8080942
:100E1000C4F82009D4F88C115143C4F80C19C4F853
:100E200024196421B5F8B40424F09AFFC4F8C40F5F
:100E30006421B5F8B60424F093FFC4F8C80F4FF04E
:100E40009740D4F8D41C25F073F825F0DDF802465D
:100E500094F8EC0E00F00101D4F89C0EC0F30010E1
:100E600023F06AFFB5F85416B5F8160524F078FF9C
:100E7000C4F8500BB5F81625B5F81A3593420AD2C6
:100E8000B5F85416B5F818051D189542A8BFD01A24
:100E900024F066FF00E00020C4F8540BD4F8F80EEC
:100EA000C0F30030C4F85C0B70BD000004210020CA
:100EB000F0210020F2210020645C00206C5C002006
:100EC000445C00202C5C0020F22000206C200020DC
:100ED000002C014028210020665C0020685C002076
:100EE000825C0020685E0020F0B5D04CD4F89C0EE7
:100EF000C0F30010002881B040F09681DFF84C5418
:100F0000B5F83E01012808D10520C4F8FC0D4FF4C6
:100F1000FA61012024F024FF17E0D4F8501DB1F548
:100F2000FA5F07DC012024F01BFFD4F8501D4FF4BA
:100F30007A7206E0032024F013FFD4F8501D40F627
:100F4000B83291FBF2F1C4F8FC1DC4F81C0E4FF44A
:100F5000B471B5F8880624F003FFC4F82C0E6421A0
:100F6000B5F88A0624F0FCFEC4F8600E6421B5F8DA
:100F70008C0624F0F5FEC4F8840E6421B5F88E06C4
:100F800024F0EEFEC4F8880E4FF09746D4F8842E75
:100F9000DFF8F81B801A24F0E3FEC4F88C0E6421FD
:100FA000B5F8900625F052F8C4F86C0E3046D4F827
:100FB000D41C24F0BDFF25F027F8C4F8AC054FF48D
:100FC0007A71B5F8800624F0CBFE0146C4F8B0155E
:100FD000D4F8AC05091824F0C3FE0746D4F8D41C95
:100FE000C4F8B475304624F0A3FF25F00DF8D4F80A
:100FF000B015C4F8C805C4F8E405C4F8CC15C4F8A5
:10100000D0754FF47A71B5F8820624F0A9FE014636
:10101000C4F8E815D4F8E405091824F0A1FE074641
:10102000D4F8D41CC4F8EC75304624F081FF24F0C9
:10103000EBFFD4F8E815C4F80006C4F83407C4F888
:101040005007C4F80416C4F80876D4F81C0ED4F877
:10105000B015D4F8B425C4F85406C4F83817C4F849
:101060003C27C4F85417C4F858274FF47A71B5F8E0
:10107000840624F075FE0146C4F85816D4F85406C8
:10108000091824F06DFED4F81C1ED4F85826C4F8B4
:101090005C06C4F87806C4F82406C4F84006C4F810
:1010A0000407C4F82007C4F87016C4F87426C4F8FE
:1010B0001C16C4F82026C4F83816C4F83C26C4F818
:1010C000FC16C4F80027C4F81817C4F81C27C4F885
:1010D0008C164FF47A71B5F8860624F041FE01466D
:1010E000C4F89016D4F88C06091824F039FEC4F818
:1010F0009406C4F8B006C4F8CC06C4F8E806D4F8E0
:101100001C1ED4F89026C4F8A81644F28910C4F81E
:10111000AC26C4F8C416C4F8C826C4F8E016C4F84F
:10112000E426C4F87405DFF8681AC4F87815DFF807
:10113000641A24F015FEC4F87C053046D4F8D41C9B
:1011400024F0F6FE24F060FFDFF8D41DC4F89415F7
:10115000C4F89005091824F003FEC4F8980532205D
:10116000B5F8541624F0FCFDC4F8880F4FF47A71DA
:10117000B5F8800924F0F4FDC4F88C0F1420B5F8FC
:10118000541624F0EDFDD4F86C1724F031FEC4F8A9
:10119000940F4FF47A71B5F84C0624F0E1FDD4F8C1
:1011A0003C1D24F0DDFDC4F8A40DD0F1807048BFD3
:1011B0000020C4F8C80DB5F85406B5F84826C0EBB1
:1011C0000011C800642190FBF1F1B5F84A065043C4
:1011D00024F0C6FDD0F1807048BF0020C4F8DC0DBB
:1011E00040F2BB32B5F84206B5F84A16504324F037
:1011F0002DFFC4F8CC0D4FF4206124F06FFFC4F82C
:10120000900E4FF48071D4F8CC0D24F067FFC4F831
:10121000D40DCC21D4F8CC0D24F060FFC4F8D80D47
:1012200041F62110C4F8100E01B0F0BD00000020FE
:1012300030B5DFF8184CDFF82C54D4F8400DD4F852
:10124000D41CC4F8E40081B0D4F83C0DC4F8E0002C
:10125000D4F8340DC4F8E800D4F8380DC4F8EC0024
:10126000D4F8280DC4F8F400A868C4F8F800A869F8
:10127000C4F8F0006869C4F800014FF0974024F00A
:1012800057FE24F0C1FEC4F8180101B0DFF8940C39
:10129000D4F8A811C4F81C01DFF88C0CC4F82001A4
:1012A000DFF8880CC4F82401DFF8840CC4F82801A6
:1012B000DFF8800CC4F82C01DFF8200DC4F83001F1
:1012C000286AC4F83401E869C4F83C01686AC4F8C3
:1012D0003801A86AC4F8440104F1E000BDE83040D8
:1012E0000847000010B5DFF8644BD4F8BC0BD4F805
:1012F000AC11C4F80401D4F8B40BC4F80801D4F854
:10130000C80BC4F80C01D4F8C40BC4F81001D4F80D
:10131000C00BC4F8140104F1E0008847D4F85C0164
:10132000A062D4F86001E062D4F84C012063D4F8E4
:1013300050012066D4F868016066D4F88C01C4F8C6
:10134000980010BD941200201C6500203843002036
:1013500030B5DFF8F84AD4F8D01CD4F86801DFF8CB
:10136000805C81B024F044FDC4F81C08D4F8D01C83
:10137000D4F8680124F03CFDC4F83408D4F87001B6
:10138000C4F81808C4F83008D4F8D01CD4F86801A0
:1013900024F02EFDC4F84C08D4F8D01CD4F8680111
:1013A00024F026FDD4F88811C4F87C18C4F89418E9
:1013B000C4F8AC18C4F8C418C4F8DC18C4F8F4189D
:1013C0003222D4F88C11C4F864085143C4F80C19C3
:1013D000C4F82419D4F87001D4F87C11C4F8480872
:1013E000C4F86008C4F87808C4F89008C4F8A808DD
:1013F000C4F8C008C4F8D808C4F8F008C4F808094C
:10140000C4F82009A066C4F89410C4F88009C4F890
:101410009809D4F8D01CD4F8680124F0E9FCC4F889
:101420008409D4F8D01CD4F8680124F0E1FCC4F895
:101430009C092022B5F8B809DFF8E41A0006C4F8C0
:101440001C0BB5F8BA0924F02BFC0146C4F8201B8C
:10145000B5F8BC090006C4F8240BD4F87001C4F830
:10146000000AD4F8680124F0C3FCC4F8040AD4F8D4
:101470007001D4F8201BC4F8B009D4F8680124F036
:10148000B7FCC4F8B409D4F87001D4F8201BC4F830
:10149000180AD4F8680124F0ABFCC4F81C0AD4F88C
:1014A0007001D4F8201BC4F8CC09D4F8680124F0EA
:1014B0009FFCC4F8D00901B030BD10B5DFF88C49ED
:1014C000D4F878194FF0A060C4F86C09D4F89001F2
:1014D000C4F86809D4F87C01C4F8640904F66410FF
:1014E0008847D4F8CC1CD4F870090E2224F0D8FB1D
:1014F000C4F830030E22D4F8C81CD4F8740924F0C0
:10150000CFFBC4F83403D4F8700100EB800148002D
:10151000C4F82C030020C4F8580310BD2DE9F04195
:10152000DFF8BC5ADFF82449B5F81C05112244F253
:101530008911C00324F0B4FBC4F888041122B5F863
:101540001E05DFF8486B3146C00324F0A9FBC4F840
:1015500084041122D4F8180100EB80014800C4F87B
:1015600080043146DFF8280B0068C4F89004C4F802
:101570008C0440F28D67B5F8F804C00324F090FBAA
:10158000C4F870031122B5F8FA043946C00324F0F8
:1015900087FBC4F86C034FF080780020C4F88C03FC
:1015A000C4F87883C4F874831122D4F8180100EBCE
:1015B00080014800C4F86803B5F8F8047043C4F823
:1015C0007003DFF85C69B5F8FA047843C4F86C037B
:1015D0003146B5F8DE04C00324F062FBC4F8A8036A
:1015E0001122B5F8E4043146C00324F059FBC4F8D5
:1015F000A403C4F8B0830020C4F8C403C4F8BC0337
:10160000C4F8AC83D4F8180100EB80014800C4F89A
:10161000A003BDE8F08110B5DFF83048DFF8740AA8
:10162000D4F884110160D4F850114160D4F86411E9
:101630008160416988474FF40000C4F8DC03C4F8B6
:10164000F403C4F8FC034FF020714FF08070C4F82D
:10165000E803C4F8E403C4F8E013D4F87001C4F854
:10166000D80310BDFC11002062100D00CA32240006
:10167000FC87640070B5DFF8D447DFF81C5AD4F853
:101680008001296ADFF858692860D4F85001E860C1
:10169000D4F854012861D4F858016861D4F848019D
:1016A0006860D4F84C01A86028468847A96AA869F0
:1016B00024F09EFBC4F81404696AE86924F098FBDE
:1016C000C4F81804296BA86924F092FBC4F84C04F0
:1016D000E96AE86924F08CFBC4F850044FF4A021B7
:1016E000B6F86E06C00324F03BFBD4F8501424F087
:1016F0007FFBC4F850044FF4A021B6F87206C00373
:1017000024F02EFBD4F84C1424F072FBC4F84C04E3
:1017100094F8280F00F00500012822D1B6F84206FF
:1017200051280CDBD4F818144FF4000024F060FBAF
:10173000C4F818044FF40000D4F814140DE029285C
:101740000FDBD4F818144FF0C07024F051FBC4F82C
:1017500018044FF0C070D4F8141424F049FBC4F8F6
:10176000140440F28652D4F87001D4F89811C4F8E9
:101770001004C4F82014C4F81C14B6F844065043EE
:101780004FF47A7290FBF2F06863DFF8385C284619
:1017900024F02EFBC4F858042846D4F8981124F0FD
:1017A00027FBC4F85404D4F87001C4F8480470BD91
:1017B0002DE9F04DDFF82808B0F8B014022918BF61
:1017C000032940F08A80DFF88446D4F8981EC1F3DC
:1017D0000012002A00F08180B0F8B224D4F8B83E9C
:1017E0009A427AD3D4F8EC2A002A02BFDFF8D85BF9
:1017F0002A68002A71D1C9076DD494F8141F11F01A
:10180000300F68D1B0F8D410002941D0D4F8581561
:10181000D4F8ACB7D4F8A8A7D4F8506DC4F8FCBA83
:10182000002948BF4942C4F8041BC4F800ABB0F813
:101830003E11D4F8048BB0F85406012908BF4FF4C8
:10184000FA66D3498845B8BF88464FEAE871A0FBDD
:10185000082300FB0133A6FB0201F71706FB031167
:1018600007FB021142F21072002323F007F9000E69
:1018700040EA012071000A2291FBF2F18842B8BFD0
:1018800008469AFBF0F19BFBF0F0A960686009E064
:10189000DFF8385D284624F02CFE002280212846FF
:1018A00024F032FED4F85805002848BF4042C4F85E
:1018B000040B0120C4F8EC0A0020C4F89C04C4F80E
:1018C0009804C4F89404C4F8A004C4F8A404C4F8A8
:1018D0007804BDE8F08D01202860BDE8F08D00009F
:1018E0006666E60010B5DFF86445D4F8EC0A012816
:1018F00030D1DFF8EC06B0F8D4100A0018BF062982
:1019000028D1D4F8EC1EC1F3402119B3DFF8C01C74
:101910000A68521C0A60B0F8200590421ADAD4F81E
:101920000C0F40F02000C4F80C0F0020C4F8A807EA
:10193000C4F8AC0708604FF4A360D4F848152044FD
:1019400088470220C4F8EC0AD4F80C0F40F01000CD
:10195000C4F80C0F10BD0000E9B50900DFF8EC0475
:10196000B0F8502AB0F8541A012A02BFDFF8642CEC
:101970001288022A2FD14FF6FF72914222D0DFF84F
:101980006036B3F8E8C5491C89B2B1EB4C0F19DBDE
:10199000DFF828CDB3F8D030DCF800C0032B1146B7
:1019A00006D140F219239C450AD2A0F8523A09E028
:1019B000BCF59B7F04D24FF49B73A0F8523A01E030
:1019C000A0F852CAD0F89C3EC3F3001323B11146CD
:1019D000A0F8541A70470021A0F8541A704700006C
:1019E0000051250230B4DFF8F815DFF86004B1F8D3
:1019F000E82552B9B1F8D030032B0CBF40F21923BF
:101A00004FF49B73A0F8523A00E00122A0F8502A4C
:101A1000B0F8504AB0F8563AB0F8522A012C02BF3A
:101A2000DFF8B04B2488022C23D1D0F89C4EC4F3AD
:101A30000014F4B9D0F8EC4EC4F3400404B15B1CBC
:101A4000B1F8EA459DB2A54214D32346DFF86C2CC9
:101A5000B1F8D0401268032C05D140F21924A242FB
:101A600008D2224606E0B2F59B7F03D24FF49B7268
:101A700000E00023A0F8522AA0F8563AB0F8520A23
:101A8000C88130BC70472DE9F047DFF8346CDFF8CF
:101A90009074DFF8B88304460D469146B4604FF069
:101AA000407024F0A5F930612946384624F0A0F9A9
:101AB000F0604FF080754FF4000070614FF07F4A86
:101AC000DFF8000CB06100214FF04070C8F8B84456
:101AD000C8F8C004C8F8BC744FF02060C8F8C454FB
:101AE000C8F8C8A47064F46300203064B5647167FA
:101AF000C6F84CA03467F767C6F8A440C6F8B4A08F
:101B0000DFF8C40BB067C6F8AC00DFF8C01BDFF825
:101B10007C05C6F8A800C6F880100020C6F8B00002
:101B2000C8F8EC4449464FF0407024F061F9C8F819
:101B3000F4044946384624F05BF9C8F8F854C8F86C
:101B4000FCA4C8F8F004BDE8F087DFF8741B00209F
:101B500008630022BD48C0F8E0244A66C1F8982016
:101B6000C1F8CC20C0F814258A62C0F8D824CA6510
:101B7000C1F89020C1F8C420C0F80C25C0F8D02FBF
:101B8000C0F8CC2F704700002C2C0140AE476100FC
:101B900033333300BC7433002DE9F043AB4CDFF832
:101BA000305BD4F89C0EDFF8386481B0C0F30010CD
:101BB00068BBB6F82605642124F0D2F80746B6F8CB
:101BC0002405642124F0CCF80146D4F870013A468B
:101BD000FFF759FFD4F83C0D0111D4F8340D24F06F
:101BE000BFF82860B6F8D020D4F8E40ADFF8E41A89
:101BF000032AB4BF0FF258220FF2D82252F8200065
:101C000024F0AEF8296824F0ABF86860C0E0B6F8BC
:101C1000D010B6F8280503290FDA642124F0A0F8C3
:101C20000746D4F8281D4FF0346024F099F869680D
:101C300024F0DEF8DFF8F01C0EE0642124F090F8C8
:101C40000746D4F8281D4FF0346024F089F86968FD
:101C500024F0CEF8DFF8D41C24F0CAF8394624F07A
:101C6000C7F8A8608046D4F8E00E012812D1B6F873
:101C7000CE0040F2DC51884208BF4FF0007105D021
:101C800040F24C41884205D1DFF8A41C404624F0C4
:101C9000AFF88046B6F8D400022812BF0328B6F881
:101CA0003E01012807D1B6F822050A2124F058F890
:101CB0004FF4400111E0D4F8500DB0F57A6F14DA0A
:101CC0004FF44861C0F57A6024F04AF80746B6F848
:101CD00022050A2124F044F8394624F089F800F15D
:101CE0008071404624F084F88046D4F8E00EC4F8B1
:101CF000B48A00280CBFB4F96605B4F964056528F8
:101D0000A8BF64200A2124F02BF8074639464FF07B
:101D1000407024F06DF8C4F8C0043946DFF8008242
:101D2000404624F065F8B7F1807FC4F8BC04B8BF22
:101D30004FF0807704DBB7F1206FC8BF4FF020670A
:101D4000D4F8E00EC4F8C47400280CBFB4F964756C
:101D5000B4F96675332FA8BF3227B6F8260564217B
:101D600023F0FEFF81460A21384623F0F9FF494659
:101D700024F03EF8074639464FF0407024F038F81A
:101D8000C4F8F4043946404624F032F8C4F8F004AC
:101D9000B6F8DE00B6F8541600F5FA7023F0E0FF4E
:101DA000E8606421B6F8C20423F0DAFFDFF8941C7F
:101DB00024F01EF8C4F8AC0AB4F85C0A012826D155
:101DC000B6F8D400022818BF032820D1B6F886152B
:101DD000B6F8C02428698A4238BF104609D3884221
:101DE000B8BF084605DBD4F8EC1EC1F3400101B1D1
:101DF000401E2861B6F84616B6F8CC0023F0B0FFB6
:101E000006462869642123F0ABFF31460FE0B6F89F
:101E1000C0042861B6F84616B6F8CC0023F0A0FF3F
:101E20000546B6F8C004642123F09AFF294623F042
:101E3000DFFF014623F0DCFFDFF8A81D081824F0BF
:101E4000C5FBC4F8B00A01B0BDE8F0830000002073
:101E50008400000084000000840000008400000072
:101E6000840000009C000000E0000000BE000000B4
:101E700010010000D601000030020000A80200009E
:101E80003403000034030000E80300006009000090
:101E9000600900006009000060090000600900009E
:101EA000600900006009000060090000600900008E
:101EB000600900006009000060090000600900007E
:101EC000600900006009000060090000600900006E
:101ED00060090000FC030000FC030000FC0300009C
:101EE000FC030000FC030000FC030000FC030000F6
:101EF000FC030000FE01000052030000A8020000E5
:101F0000A80200003403000034030000EE020000C9
:101F10000A0500000A0500006009000060090000D1
:101F200099991900E00B0300143DB50F9D755C22D3
:101F30008A9EDA07999999002948B0F8CA14DFF8FF
:101F4000A80C012914D0022902BFD0F8981F43F62B
:101F50002102114212D0D0F84C15D0F85825D0F8F3
:101F6000E03E53BB8A4221D10021C0F8C81A704715
:101F7000D0F8981F42F621021142ECD1D0F8A01FF0
:101F80000129E8D1D0F82C1AD0F8382AD0F8E03E50
:101F900043B98A42E8D091421FDA4FF07F41C0F83E
:101FA000C81A15E08A420AD017DA0DE0914214DA15
:101FB0004FF07F41C0F8C81A0AE08A4203D10021DD
:101FC000C0F8CC1A704708DA4FF08071C0F8CC1A0C
:101FD0000021C0F8D41AC0F8D01A7047297A6A1FB5
:101FE00038430020DFF8040CB0F8CA14DFF8400DC5
:101FF000012914D0022902BFD0F8981F43F621020C
:10200000114212D0D0F84C15D0F85825D0F8E03E47
:102010004BBB8A4221D10021C0F8CC1A7047D0F8BE
:10202000981F42F621021142ECD1D0F8A01F0129DD
:10203000E8D1D0F82C1AD0F8382AD0F8E03E3BB9D5
:102040008A42E8D020DA4FF08071C0F8CC1A16E04E
:102050008A420AD0914217DA0DE015DA4FF080710A
:10206000C0F8CC1A0BE08A4203D10021C0F8C81A8C
:102070007047914208DA4FF07F41C0F8C81A00213A
:10208000C0F8D41AC0F8D01A704700005C8F020064
:10209000F861002060120020C0110020DFF8940CCD
:1020A0004FF4B5612DE9F043DFF8409B866BB9F83A
:1020B0004406DFF8348B4843820AF717A2FB060177
:1020C00002FB0711B8F8522A002322F0F9FC01465E
:1020D000B9F8BE0403288BB0C0F2DF8003BFDFF87D
:1020E000582CD8F8AC3AD21A0022B9F8CA34DFF822
:1020F000D065012B3BD0022B02BFD8F8983F43F6A6
:1021000021073B4239D0099008924FF49660404431
:102110000790069606F19C000590D8F8B40A049042
:10212000D8F84C050390D8F85805D8F8F039D8F805
:10213000B02A0290D8F8E00E0190D8F8F409009087
:10214000D8F8AC0A24F0B6FAC8F8B80AD8F8B00A39
:10215000014623F04DFE0746D8F8F409014623F066
:1021600047FE381A01281FDB24F030FA1DE0D8F8AA
:10217000983F42F621073B42C5D1D8F8A03F012B3A
:10218000C1D1099008924FF496604044079006969A
:1021900006F19C000590D8F8B40A0490D8F82C0AEF
:1021A0000390D8F8380AC0E70020B9F8CA1401290A
:1021B0003BD0022902BFD8F8981F43F621021142F2
:1021C00039D008F2E4410191D8F84C15D8F85835C7
:1021D0000091D8F8E02ED8F8F01924F0D7FAC8F812
:1021E000BC0AB8F96475B8F966C5D8F8F009D8F82A
:1021F0005825D8F84C35D8F870E1D8F8B84AD8F84E
:10220000E01ED8F8BC5A06950029059420D14FF459
:102210007D6141440491CDF808E006F13401039159
:10222000CDF804C0009700211EE0D8F8981F42F6B0
:1022300021021142C5D1D8F8A01F0129C1D108F24D
:10224000E4410191D8F82C1AD8F8383A0091C0E747
:102250004FF47D644444049406F134040394CDF8AF
:1022600008E00197CDF800C024F0A8FAC8F8C00A29
:1022700008F6CC70029006F168000190D8F8700161
:10228000D8F84C35D8F85825D8F8E01E0090D8F882
:10229000F40924F0D3FAC8F8C40AB9F8BE04032834
:1022A00031D1B8F85A0A012812D1D8F8E03ED8F84E
:1022B000C40AD8F8C01AD8F8B82A002B0CBFC8F83E
:1022C000C82AC8F8CC2AC8F8D01AC8F8D40A01E03D
:1022D000FFF732FEB9F8D40001002FD004282DDA20
:1022E000D8F8E03ED8F8BC2AD8F8C40AD8F8C01A02
:1022F000002B19BFC8F8C82AC8F8D01AC8F8CC2AC9
:10230000C8F8D01A59E004281CD1B8F85A0A012894
:1023100012D1D8F8E03ED8F8C40AD8F8C01AD8F8D4
:10232000B82A002B0CBFC8F8C82AC8F8CC2AC8F8AD
:10233000D01AC8F8D40A01E0FFF7FEFD0BB0BDE8E3
:10234000F0434FE605282DD1B9F8D400010001D0A3
:10235000042802DBFFF746FE20E0D8F8E03ED8F87C
:10236000BC2AD8F8C40AD8F8C01A002B0CBFC8F889
:10237000CC2AC8F8C82AC8F8D40AC8F8D01AB8F8BD
:102380005A0A01280AD1D8F8B82A002B14BFC8F875
:10239000CC2AC8F8C82A0BB0BDE8F0830BB0BDE862
:1023A000F043C9E54FF07F40C8F8C80A4FF080708D
:1023B000C8F8CC0A0020C8F8D00AC8F8D40A0BB074
:1023C000BDE8F08399991901486100202DE9F04397
:1023D000DFF81848B4F85A021D2881B005D14FF42F
:1023E0000041DFF8580924F0D5FADFF8FC57DFF890
:1023F0005069B5F8A60A401CA5F8A60A00F06CF9C9
:10240000B4F87C06DFF83C19DFF82829C00381FB0B
:10241000000110F5801041F10001400D40EAC1209B
:102420007060D36B776883FB070110F5000041F102
:102430000001000E40EA0120C5F8F40C106CDFF832
:10244000082903EB400087FB0001000E40EA012051
:102450000916A2FB008902FB019918F5000049F159
:102460000001000E40EA0120C5F8F80CD5F89C0EDA
:10247000C0F3001030B90120A5F85A0A0020A5F8D1
:102480005C0A0AE0D5F80C0FC0F30010002802BF68
:10249000B4F864020028FFF701FE00F09DF8B5F8DB
:1024A000860A01280AD1B4F8D40006282FD0D5F81E
:1024B000800BC5F8A00D04F0C9FD6BE0D5F89C0EAB
:1024C000C0F30010002865D0D5F8A00EC0F340007E
:1024D00000285FD1FFF76CF9D5F80C0FC0F300109E
:1024E0000028B4F8D4004ED1010018BF01280CD147
:1024F00000F020FA00F0A8FA00F044FC01F08AF99C
:1025000001F0B0FA01F040FC1EE0062802D102F012
:10251000A9F83FE00020C5F8580D00F00BFAD5F8F7
:102520007807C5F8240D01F075F9B4F8CA0401283C
:102530000FD0022802BFD5F8980F43F621010842B8
:102540000DD00020C5F8180B02F056F902F08EFAF3
:1025500020E0D5F8980F42F621010842F1D107F0AA
:1025600035FAB4F8EA04D5F8501D4FF47A725043A6
:1025700024F050FA306021F027FF22F0B3F8012058
:10258000C5F8180B06E0062802D101F073FE01E041
:1025900002F0FAFF0D480188C90643BFD5F81815A7
:1025A000808CC0EB4100808C6080B4F85A021D28FA
:1025B00008D101B0BDE8F0434FF40041DFF87C07DB
:1025C00024F0E6B901B0BDE8F0830000002C014022
:1025D000D8630020645E0020F0B4DFF81006DFF856
:1025E0000856B0F8B615DFF86427D5F89C6E51434D
:1025F000DFF85C279368D468C6F30016002E59D024
:10260000B5F8866A002E04BFB5F8886A012E51D14C
:10261000D5F8B86EB6F5FA7F4CD9B0F8AE65012E94
:1026200043D11668DFF80C77761C1660D7F83CC0EB
:10263000BCF1000F48BFCCF1000C8C4505DAD2F894
:1026400004C00CF1010CC2F804C0D7F840C07F6C84
:10265000BCF1000F48BFCCF1000C8C45B8BF5B1C2F
:10266000002F48BF7F428F42B0F83E11B0F8BE0540
:10267000B8BF641C00290CBFD5F8501D40F6980166
:102680004843864216D3CD21A1FB0001000A40EA4F
:102690000160516881423CBF8342844205D3DFF828
:1026A000B406016841F400510160002010605060E0
:1026B00000230024D4609360F0BC70479412002083
:1026C000445B0020EC51F8FFCCCC4C006766E6FF81
:1026D000A411002040420F002DE9F04BDFF878668E
:1026E000DFF87846B068DFF84C76DFF8FCB4DFF846
:1026F000FC54A4FB002312F5000043F10001000E7E
:1027000040EA012078613068A4FB002312F5000044
:1027100043F10001000E40EA01207863F068A4FB59
:10272000002312F5000043F10001800E40EA811001
:10273000DFF82C1608807068A4FB002312F5000057
:1027400043F10001000E40EA01203861DBF89C0EE5
:10275000C0F3001030BBB5F87406DFF8E815C0030D
:1027600081FB0001B0F17F4061F1FF31400E40EA92
:10277000C110F865DBF8381D23F0AAFAF865B5F842
:10278000D000032803DA10B1E88A992101E0E88A31
:10279000E6214843DBF8281D23F0E2FADFF8C415F0
:1027A0003866486138693968D7F850C0401A80FBEC
:1027B0000C23F86DA0FB0289C11700FB039901FBF4
:1027C000029918F5002049F10001000D40EA01309E
:1027D0007968C0F1000E7869C7F83CE0401A80FBC8
:1027E0000C23F86DA0FB0289C11700FB039901FBC4
:1027F000029918F5002049F10001000D40EA01306E
:1028000040423864704440427864796B386E41438A
:10281000B86BB9640A1ADBF87031DFF84C158B42DB
:10282000B8BF83FB022304DBD3171B0643EA122342
:10283000120612F5000243F10003120E42EA0322CF
:102840008018DFF808158842B8BF0846B86301460B
:10285000DFF8180523F084FAF864B5F86A23D6F88F
:102860000004A4FB008918F5000049F10001000EE6
:1028700040EA0120DFF8F8140B689F188742B8BFC0
:102880000F6004DB17189F42B8BF981A08600868E9
:10289000B0F5805FA4BF40F6FF700860D6F804046E
:1028A000A4FB008918F5000049F10001000E40EA80
:1028B0000120DFF8C0140B689F188742B8BF0F6073
:1028C00004DB17189F42B8BF981A08600868B0F573
:1028D000805FA4BF40F6FF700860B5F84C03012884
:1028E0000CBFD6F80C04D6F80804A4FB006716F554
:1028F000000047F10001000E40EA0120DFF87814E3
:102900000B689C188442B8BF0C6004DB14189C420E
:10291000B8BF981A08600868B0F5805FA4BF40F699
:10292000FF700860BDE8F08BB1BF0C00E53F04000C
:102930001D555501F0B5AC4CD4F89C0EC0F30011F8
:10294000002981B074D0B4F8861A002904BFB4F805
:10295000881A012902BFA54EB6F8EE14012967D1E5
:10296000B6F8BE14032963DADFF810542968012988
:1029700006D010F0030F03D1D4F8680B012850D112
:10298000DFF8FC03B6F9F0140068401A00B2002822
:1029900005D56FF08B0188420ADA084608E0012865
:1029A000A1BF0121C4F8681B29608D28A8BF8C2015
:1029B0004FF00C61000523F0D3F9C4F86403D4F898
:1029C000680B18B9C4F88403C4F864030020C4F881
:1029D00060034FF45870D4F8941320448847D4F817
:1029E0008C23B6F8F204D317A0FB026700FB037731
:1029F00016F5000047F10001000E40EA0120D4F86E
:102A0000681B012905D1012804DA0020C4F8680BED
:102A100000E0002094F89C1EC90706D5002129601B
:102A200003E00020C4F8680B2860D4F8A01D21B989
:102A30000020D24AC4F8680B1060C4F8640B01B0DF
:102A4000F0BD000028EDBD0170B5674CD4F8A00DB5
:102A5000002848BF40420128C0F2C280D4F89C0E32
:102A6000C0F30010002800F08F80B4F8860A002818
:102A700040F08A80D4F8580D012840F08880D4F8BE
:102A8000D40FD4F8D81F884243DAAA4DE96B052247
:102A9000084623F005F90646286C0522014623F076
:102AA000FFF88619686C0522014623F0F9F8DFF873
:102AB000E05CDFF8E01C8019286023F0F3FF286059
:102AC00023F0F8FF2860C000C4F80C0BDFF8C81C26
:102AD00023F08EF9D4F8F41AC4F8080BC4F8F00AFD
:102AE000C4F87C14C4F878044FF48F60D4F8AC14A4
:102AF00020448847D4F8A404002848BF44F2891031
:102B000004D4B0F1807F42DD4FF08070C4F8A4049B
:102B10003DE00120C4F8640D0020C4F85C0D334989
:102B2000D4F8D02EB1F8DA0090420ED232280CDB65
:102B30000022C4F8B02F94F8282FD20705D4D4F877
:102B4000142F42F00202C4F8142FD4F80C2F42F0D4
:102B50004002C4F80C2FD4F8142FC2F3400232B153
:102B6000B1F85416C903C00323F0FAF800E00020BE
:102B7000C4F85805D4F8E00E012808D1D4F8580557
:102B80004042C4F8580502E00020C4F8640DD4F8AF
:102B9000C00C6E4A00284CBF41420146914211DAF6
:102BA000D4F8A01D002948BF494201290ADBD4F806
:102BB000641D39B90120C4F8580DD4F8680DC4F863
:102BC000600D70BD0021C4F8581D0128E16EC4F8E5
:102BD000601DAEBF5018DFF8180C4018C4F8680D1F
:102BE00070BD00003E0AD7FF0000002038430020DF
:102BF00030B44F48DFF8FC2BD0F8081D002948BF3F
:102C00004942914214DBD0F8C04CD0F85433002C28
:102C100008D4DFF8E44BA3420ADADFF8E03BC0F85F
:102C2000543305E0DFF8D84BA342A8BFC0F85443A3
:102C3000DFF8D03B994214DB914212DADFF8C82B5F
:102C4000DFF8C84B52186260D0F8C05CD0F854432B
:102C5000012D01DBA24201E052429442A8BFC0F81C
:102C60005423994215DADFF8A43B4FF07F425A60B3
:102C7000D0F8C04CD0F85433012C03DBB3F17F4FB4
:102C800007DC04E0B3F1807F03DB4FF08072C0F813
:102C90005423DFF87C2BB2F8BE24022A46D1254A01
:102CA000DFF8684B926B23689A42A4BFDFF86C5D33
:102CB000A94227DBD0F89C1EC1F3800129B1D0F8CE
:102CC000681B11B90121C0F8781BDFF8241B616073
:102CD000D0F8C03CD0F85423012B0FDBDFF8403D87
:102CE0009A4201DAC0F85413D0F8781B01291DD19B
:102CF000D0F8C01C00290FD549420DE013498A4283
:102D0000F2DBEFE7DFF8144DA1420CDBDFF8141D16
:102D1000C9189142E8DB06E0D0F8A02D002A48BF90
:102D20005242914202DA0021C0F8781B30BC704751
:102D300000000020145D00205A64BB01000C01401B
:102D4000501200200AD7A30035CD93005C8F0200FB
:102D500038610020905E00203C24014099991901BF
:102D60008A12002034120020343333001056BB0185
:102D700074100020FC1000208011002080620020D0
:102D8000981200202DE9F047DFF89C4CDFF8806AAC
:102D9000D4F8C00C00284CBF414201460B464FF00E
:102DA0008078C4F8C41CC4F8B080B6F8D010B6F867
:102DB0004226032980F2C5800128DFF8701C45DB1C
:102DC0008B4206DA4FF00070C4F8D00CDFF8603C9C
:102DD00022E0B3F1807F10DADFF8140AC018122164
:102DE00081FB0001A0F17E40C4F8D00CDFF8400C5C
:102DF000834211DADFF8383C0EE0B3F1007F07DAE6
:102E000003F17F400A2181FB0001A0F16C4001E049
:102E10004FF0F050C4F8D00CC4F8EC3FD4F8D07C9C
:102E2000D4F8683107F17F4080FB0301000E40EACF
:102E30000120C4F81C08C4F8340887FB0301000E05
:102E400040EA01200146034607463CE1052A3ADAFA
:102E50008B4206DADFF8DC0BDFF8D43BC4F8D00C89
:102E600027E0B3F1807F15DADFF88409C0184FF04E
:102E7000945181FB00592D0E45EA0925DFF8B40B6A
:102E80002818C4F8D00CDFF8A80B834211DADFF859
:102E9000A03B0EE0B3F1007F07DA03F17F400A2187
:102EA00081FB0001A0F16C4001E04FF0F050C4F84C
:102EB000D00CC4F8EC3FD4F8D07CD4F86831DFF8FB
:102EC000780BC019EEE08B4206DADFF8700BDFF802
:102ED000603BC4F8D00C2AE0B3F1807F15DADFF84C
:102EE0001009DFF85C1BC01881FB00592D0E45EA64
:102EF0000925DFF8480B2818C4F8D00CDFF8300B90
:102F0000834214DADFF8283B11E0B3F1007F0ADADC
:102F100003F17F400A2181FB0001000E40EA0120FD
:102F2000A0F16C4001E04FF0F050C4F8D00CC4F8B0
:102F3000EC3FD4F8D07CD4F86831DFF8080BC01926
:102F4000B0E0512A1EDBDFF8000B8342B8BF4FF020
:102F5000206030DBDFF8F40ADFF8F41AC01888428A
:102F600038BF4FF0706026D36FF08070C018B0F19A
:102F7000807F2FBF4FF02050192080FB0301A0F16C
:102F8000206018E0252A2DDBDFF8C80A8342B8BF8D
:102F90004FF0A0600FDBDFF8C00ADFF8C01AC018DE
:102FA000884206D20C27DFF8B80A0021C7FB0301CC
:102FB00001E04FF02050C4F8D00CDFF8740AD4F8C8
:102FC000D01CC4F8EC0FD4F8680181FB0001000E9E
:102FD00040EA0120C4F81C08034607460146C4F82D
:102FE000340870E0042ADFF8441A31DB8B4208DA37
:102FF0004FF00070C4F8D00CDFF8343AC4F8EC3F5E
:103000004AE0B3F1807F10DADFF8E407C01812213C
:1030100081FB0001A0F17E40C4F8D00CDFF8100A5B
:103020008342E9DBC4F8EC3F36E0B3F1007FA8BF90
:103030004FF0F05006DA03F17F400A2181FB0001D6
:10304000A0F16C404346C4F8D00CC4F8EC3F23E038
:103050008B42B8BF4FF0007018DBB3F1807F08DA05
:10306000DFF88C07C0180A2181FB0001A0F17E4027
:103070000CE0B3F1007F07DA03F17F400A2181FB06
:103080000001A0F1744001E04FF0B050C4F8D00C42
:10309000DFF89C09C4F8EC0FD4F8D07CD4F8683180
:1030A00007F17F4080FB0301000E40EA0120C4F8D5
:1030B0003408C4F81C0887FB0301000E40EA012015
:1030C000034607460146C4F84C08C4F86418C4F81F
:1030D0009C39C4F88479512AA8BFD4F8D80C28DACE
:1030E000B6F8140510B1D4F8D80C22E0D4F894073F
:1030F000A16E626E206482FB0123216ED4F8DC0C89
:10310000E063120E80FB0101000EE76D42EA03222C
:1031100040EA01201B160916C01BA0FB025961EBF7
:10312000E77100FB039901FB02992D0E45EA092581
:103130007819E065D4F8F40CA060D4F8F80CE060DD
:10314000B6F8B609012857D1D4F8241BD4F8680181
:1031500022F04EFED4F8B01C22F04AFE0746D4F806
:10316000241BD4F8680122F043FE216E22F040FEB9
:103170000146D4F8CC0722F03BFE3F1AD4F8B41C29
:10318000D4F89C0022F034FEC119A06E22F030FE6B
:10319000D4F8B01C081AC4F8B80CD4F8241BD4F81E
:1031A000680122F025FED4F8B41C22F021FE074667
:1031B000D4F8241BD4F8680122F01AFE216E22F004
:1031C00017FE0146D4F8D00722F012FE3F1AD4F8B9
:1031D000B01CD4F89C0022F00BFE391AA06E22F02D
:1031E00007FED4F8B41C081AD4F8B81CC4F8BC0CF8
:1031F000C4F8B01CC4F8B40CD4F89C072169A061D1
:10320000D4F8A007E061A068401A20626169E06814
:10321000401A6062B6F8D010B6F84206032904DA04
:103220000F2804DADFF8587B05E00F2801DB47465A
:1032300001E0DFF8507B216B384622F0D9FD0146D2
:10324000A06822F0D5FD0546216AE06A22F0D0FD93
:103250000146D4F8EC0F22F0CBFDA16E22F080FDE8
:10326000A169491B091AA06A22F0C2FD60633846B1
:10327000216B22F0BDFD0146E06822F0B9FD074652
:10328000616AE06A22F0B4FD0146D4F8EC0F22F046
:10329000AFFDA16E22F064FDE169C91B091AA06AA5
:1032A00022F0A6FDA1682161A063C4F88C0804F691
:1032B0007400E1686161616BC4F87418D4F888180F
:1032C0008847D4F8A01804F68C008847D4F88408FE
:1032D000D4F8B818C4F8A408D4F89C08C4F8BC08FA
:1032E00004F6A4008847D4F8D01804F6BC00884738
:1032F000D4F8B408D4F8E818C4F8D408D4F8CC0842
:10330000C4F8EC0804F6D4008847D4F8001904F691
:10331000EC008847D4F8FC28606BD4F8E418401A15
:10332000A16B6063891AA163C4F82C18C4F814084F
:1033300004F61400D4F828188847D4F8401804F686
:103340002C008847D4F82408E064D4F83C082065B1
:10335000B6F8B609A0B9E06E23F0E2FBE16D80FBA0
:103360000101000E40EA0120C4F84408E06E23F099
:1033700017FCE16D80FB0101000E40EA012021E015
:10338000D4F8B81CD4F8BC0C23F048FC074623F052
:10339000C7FBE16D80FB0101000E40EA0120C4F88B
:1033A000FC09384623F0FCFBE16D80FB0101000EB7
:1033B00040EA0120C4F8140AD4F8FC09C4F844080F
:1033C000D4F8140AD4F85818C4F85C0804F6440079
:1033D0008847D4F8701804F65C008847D4F854087D
:1033E0006065D4F86C08A065B6F8B60900287AD1F3
:1033F000B6F8B026206EA168012A2CD122F0F8FC84
:103400000746D4F8B810D4F8D40022F0F1FC0546F1
:10341000D4F8D01CD4F8640122F0A2FC294622F092
:10342000E7FC381AC4F8C000E168206E22F0E0FC26
:103430000746D4F8B810D4F8D00022F0D9FC0546DD
:10344000D4F8D01CD4F8640122F08AFC294622F07A
:10345000CFFCC0192BE022F0CBFC0746D4F8B81003
:10346000D4F8D40022F0C4FC0546D4F8D01CD4F81B
:10347000640122F075FC294622F0BAFC381AC4F81F
:10348000C000E168206E22F0B3FC0746D4F8B81003
:10349000D4F8D00022F0ACFC0546D4F8D01CD4F807
:1034A000640122F05DFC294622F0A2FC381AC4F81F
:1034B000C400D4F8C000D4F89019C4F87C09D4F83A
:1034C000C400C4F8940904F67C108847D4F8A819FD
:1034D00004F694108847D4F88C09C4F8D000D4F8C6
:1034E000A409C4F8D400B6F8D000032815DAD4F83B
:1034F000C00CDFF8681C002848BF404288420CDA44
:10350000D4F8C42CDFF8580C4FF0207383FB02234F
:10351000120E42EA0322801A00E04046636DC4F8AE
:10352000700D024683FB0267E06CA36D360E46EA1F
:1035300007268019C4F8C80083FB0223206DDFF83A
:10354000246C120E42EA03228018C4F8CC00D4F88E
:10355000CC10D4F8C800E067C4F8801080FB0023CA
:1035600081FB0101120E000E42EA032240EA012013
:10357000101823F02BF8B042A8BF404604DADFF859
:10358000E81B8842B8BF084620670228B8BF002061
:1035900036DBD4F8580D88BBE16FD4F8800023F0F7
:1035A0003DFB94F8281F01F00501012923D1D4F82F
:1035B0009010D4F8943FD4F8E05E421AC4F8902FEB
:1035C0003DB99A420EDAD4F8B82E642A0AD25818B5
:1035D00008E0C3F10008904504DAD4F8B82E642A54
:1035E00038BFC81AB042A8BF00F17F4003DA0028F4
:1035F00048BF00F18070C4F8900001E0D4F8600D7D
:10360000E066206FE16FC4F8440D81FB0123D4F81C
:10361000800080FB0001120E000E42EA032240EA05
:10362000012010180228A0672CDBD4F8581D49BBD4
:10363000A16E22F0DDFB0546D4F88410D4F880009A
:1036400022F0D6FB0646D4F88810E06F22F0D0FBBB
:103650002946301A22F084FBC4F89C00216FD4F86C
:10366000940722F07DFB0546616E206E22F0C0FBC0
:10367000294622F0BDFBC4F8A400D4F8B01022F013
:10368000B7FB02E00020C4F89C00C4F8A400E06F7F
:10369000D4F8C41CDFF8842DC4F884009142D4F817
:1036A0008000C4F88800D4F8A40005DAD4F8C01C5F
:1036B00000293BD400283BD4D4F89C10081AC4F845
:1036C000B400D4F858ABD4F8B820D4F8580D90BB57
:1036D000D4F8B460D4F89480A06EB61A86FB08675C
:1036E000360EC11746EA0726A6FB00593F1606FB11
:1036F0000199D4F89C60A6EB0A0607FB009986FBAB
:103700000867360E46EA07262D0E3F1645EA0925BC
:103710005219A6FB005906FB019907FB00992D0ED3
:1037200045EA092513460AEB050007E00128C3DB3B
:10373000D4F89C00C3E7002200230020C4F8580BF3
:10374000C4F8083DC4F8B8201A46D4F80C0DD4F8D3
:103750007031C4F8102DA2EB000888FB0367360E09
:1037600046EA07268019C4F80C0D104600F016F83A
:10377000E06EC4F8240D23F013FAC4F8E00AD4F87C
:10378000240D23F0CDF9C4F8DC0ABDE8F087000071
:10379000DC630020A9AA0A00E7FB690110B5A24C6E
:1037A000D4F8E01E11B9002804D404E0012902D1A4
:1037B000012800DB0020C4F8100DC4F88C0504F2C9
:1037C0008C50D4F8A4158847D4F83C0FD4F8A01531
:1037D0000818D4F8381F491C202904D34011C4F814
:1037E000600F00210020C4F8381FC4F83C0F10BD42
:1037F000A470FDFF666666013533B3FF3433B3FF53
:10380000CCCC4C003333B300CDCC4CFE64610020F3
:1038100038430020F0B5844CD4F8F40CD4F8981751
:10382000C4F8840781B0D4F8F80CC4F88807D4F839
:10383000240DC4F88C0704F284708847D4F8F40C83
:10384000D4F89C17C4F8E409D4F8F80CC4F8E809D3
:10385000D4F8A00723F0E2F9C4F8EC0923F0A0F9AA
:103860000546D4F8EC0923F05BF90646D4F8E409E0
:10387000314622F0BDFA0746D4F8E809294622F07D
:10388000B7FAC019C4F8F0093146D4F8E80922F0B3
:10389000AFFA0646D4F8E409294622F0A9FA301A0C
:1038A000C4F8F409DFF8785BB5F8D400062823D112
:1038B000D4F8C00CDFF86C1B002848BF4042884297
:1038C0000FDAB4F8860A60B9DFF87C0DC16B026CC0
:1038D000406CC4F82C05C4F82825C4F8241501B0A0
:1038E000F0BD002100220020C4F82C05C4F82825D2
:1038F000C4F8241501B0F0BDD4F88C01322148433E
:10390000C4F80C09C4F82409D4F87001C4F80809F3
:10391000C4F82009D4F89007D4F81819C4F8040999
:10392000D4F89407C4F81C0904F604108847D4F8A6
:10393000301904F61C108847B5F8D40002283FD18E
:10394000B5F8120103283DD0D4F81409D4F82C1985
:10395000C4F8C007C4F8C417D4F8240DD4F8C817A5
:10396000C4F8BC0704F2B4708847D4F81409D4F83A
:10397000E017C4F8D8070020C4F8DC07D4F8240DF9
:10398000C4F8D40704F2CC708847D4F8B407D4F84C
:10399000F817C4F8F007D4F8B807C4F8F40704F22D
:1039A000E4708847D4F8E407C4F8240501B0D4F8DB
:1039B000E807C4F82805D4F8EC07C4F82C05F0BDD6
:1039C0000328C1D1D4F81409D4F8C015C4F8A80547
:1039D0004FF4B56020448847D4F8BC05D4F8DC1512
:1039E000C4F8C40504F2C4508847D4F82C09D4F8AC
:1039F000F815C4F8E0054FF4BC6020448847D4F8BB
:103A0000F405D4F81416C4F8FC0504F2FC508847F9
:103A1000D4F8D805D4F810169AE70000B91E0500AE
:103A2000A570FDFF3433F3FF000000205C8F02001F
:103A3000CCCCCC006666A6019A9959FFCCCC4C033D
:103A4000F528DC103433B3FE295C0F00D7A3F0FF58
:103A5000D8A3F0009A9919006666E6FF6766E60249
:103A6000CCCCCC032DE9F04FDFF8BCA9DFF8B0399E
:103A7000DAF8284F04F00500012881B007D0B3F828
:103A80009C09B0F5FA7FA8BFDAF8C00C01DADAF8C1
:103A9000080D002848BF4042CAF8C40C4FF080709F
:103AA000DAF8C42CCAF8E80FB2F1007F04DC4FF456
:103AB00000054FF0207019E0B3F8A256DFF8A80611
:103AC000EE03A0FB068918F5804649F10007F60BC6
:103AD00046EA4745B3F8A066F603A0FB068918F549
:103AE000004049F10001C00B40EA4140CAF8DC53F4
:103AF000CAF8E003DAF8585D012D08BFDAF8A4042B
:103B000000F03981DAF84C0D002D4CD1B3F8D0001B
:103B100003283EDAB3F84216DAF8A00D08291BDABA
:103B200008B997483FE0DFF8240B8242B8BFDFF8BE
:103B3000200B38DBDFF81C0BDFF81C1B80188842D9
:103B400007D2DFF8181BDFF8080B8918A0EB61001B
:103B500029E0DFF80C0B26E0C0B1DFF8F00A824262
:103B6000B8BFDFF8740C1EDBDFF8E80ADFF86C1C66
:103B7000801888420AD24FF0207080FB0201000EAC
:103B8000DFF85C6C40EA0120301A0CE0DFF8540CDE
:103B900009E0B3F89606DFF8501C000681FB00012F
:103BA000000E40EA0120CAF84C0DB3F8B609DAF865
:103BB000346B012808BF002D62D104F005000128F4
:103BC00040D1DAF84C0DDFF8241C88423ADBDAF8F1
:103BD000800FDFF81C1C81FB0001000E40EA012071
:103BE00009160024A142B8BF4042CAF8280B4FF082
:103BF0004861DAF8080D81FB0001000E40EA01205F
:103C00000916A142DAF8281BB8BF40424518B5F1A1
:103C1000807FCAF82C0B13DAB3F8BE39DFF8C88BF3
:103C2000C1F18071081AC117A0FB034B01FB03BB54
:103C3000A8FB040108FB0B11000E40EA012002E082
:103C4000002000E00020CAF8300BDFF89C1BDAF8F7
:103C50007001DAF8303B81FB0001000E40EA0120E0
:103C60000916A3EB0608A8FB004B4FEAE87308FB14
:103C700001BB03FB00BB240E44EA0B24301900E017
:103C80000020CAF8340BDAF8341BDAF84C0D411A6C
:103C9000DFF8600BCAF84C1D824208DB114622F0A7
:103CA0005FF80146DAF84C0D22F0A2F80146CAF896
:103CB000D81C0A46DAF82C0DCAF8D42380FB02017E
:103CC000000E40EA0120CAF8E00CDAF8440DDAF8F8
:103CD0000414CAF8D0034FF4747050448847DAF8DB
:103CE000C40CDAF8FC23DFF8C01CCAF8F42F8842B1
:103CF000B8BF002013DBDFF8B41CDFF8B43C0918B0
:103D000099420AD2DFF8AC1C0818DFF84C1D81FB81
:103D10000001000E40EA012001E04FF08070CAF877
:103D2000F00F82FB0023DAF8E01CC0F1807080FB0A
:103D30000101120E000E42EA032240EA012010188F
:103D4000CAF8DC0CDAF89007DAF83C14CAF8080470
:103D5000DAF8DC0CCAF80C044FF481605044884750
:103D6000DAF82014DAF83404CAF8481D8142A6BFF4
:103D7000494288420846CAF8EC0C01B0BDE8F08F11
:103D80006666E600C2F5A8002DE9F04FDFF89896C8
:103D9000DFF88CB6D9F8C00CD9F8CC1C002848BF85
:103DA0004042C9F8C40C81B0D9F870090E2221F044
:103DB00077FFC9F830030E22D9F8C81CD9F8740966
:103DC00021F06EFFC9F834034FF48027D9F8C40CF2
:103DD000DFF8941388423C463D463E461FDABBF866
:103DE000A6064FF0C871800422F080FF0446BBF89D
:103DF000A8064FF0C871800422F078FF0746BBF890
:103E0000AA064FF0C871800422F070FF0546BBF887
:103E1000AC064FF0C871800422F068FF0646D9F85E
:103E2000C40CDFF8C48940F61C518842B8BF2E4646
:103E30001FDB40451CDA40F6092A5146E01B22F000
:103E400055FF0146D9F8C00CA0F61B50801122F096
:103E500095FF241A5146A81B22F048FF0146D9F8C5
:103E6000C00CA0F61B50801122F088FF2E1A00E033
:103E70003C46BBF84206D9F8D81C5128D9F86C0149
:103E8000ACBF05250A2521F0B3FF0146BBF8480663
:103E9000000621F0ADFF01464FF4400021F0A8FFDD
:103EA000C9F8DC0F8111D9F8C42CD9F83403424584
:103EB00005DA22F01BFF214622F060FF01E022F02C
:103EC00015FFC9F83403BBF84226D9F8DC1FD9F82E
:103ED000C40C512A0CDB4045B8BF4FF0C0600BDB6F
:103EE000B0F1807FACBF4FF040704FF0C06016E083
:103EF00040450DDA4FF0207021F032FF0146D9F82D
:103F00003003082221F0CCFE314622F037FF0EE0CC
:103F1000B0F1807FB4BF4FF020704FF0C07021F03F
:103F20001FFF0146D9F83003082221F0B9FEC9F875
:103F30003003D9F89C01C9F8E00F014621F058FF81
:103F40000646D9F8DC0C014621F052FF301A22F067
:103F50003DFBC9F8E40FD9F8E00C014621F048FF19
:103F6000DFF8F81A081AB0F5000FB8BF4FF40000D8
:103F700022F02CFBD9F8E41FC9F83813C9F83C1318
:103F8000C9F8640FD9F8581D002940F0AB80D9F862
:103F9000001DA942C0F2A080D9F8281FC1F3400239
:103FA000A2B121F00201C9F8281FCA0744BF41F09D
:103FB0000401C9F8281FD9F8E41C8911C9F848136D
:103FC000D9F8101DC9F85815C9F8C01CD9F8281F10
:103FD00001F00C02082A1ED121F00801C9F8281F9F
:103FE0000146D9F8E40C21F0BBFE0028D9F8641F83
:103FF000D9F8E40C03D521F0B3FE404201E021F0F2
:10400000AFFED9F8541F401A48BF0020C9F84C0F22
:104010000020C9F84803D9F8080DD9F85C13C9F88D
:104020002403D9F8C00CC9F828034FF44970484458
:104030008847D9F8581FD9F8640F21F0D9FEC9F87C
:10404000700FD9F85C1FD9F8640F21F0D1FEC9F8C0
:10405000740F99F8280F00F00500012829D1D9F82C
:104060007C1FD9F8640F21F0C3FED9F8E41FD9F8FA
:10407000E02ED9F848338142B8BF08460146012AEC
:10408000D9F8542308BF404212180028C9F8800FFD
:1040900008D446F26760834211DB46F26660C9F8D5
:1040A00048030CE0DFF8B809834208DAC9F848038E
:1040B00005E0FEF79DFDD9F85423D9F8701FC9F823
:1040C000781FC9F8E42CD9F8741FD9F8780F00F0DC
:1040D0004DF80020C9F8000DD9F8000D401CC9F8B2
:1040E000000D06E00020C9F8E40CC9F85403C9F833
:1040F0004803D9F89407D9F87414DFF8DC56C9F8E6
:104100004004D9F8E40CC9F844044FF488604844EA
:104110008847D9F86C04DFF84C19C9F8F00CD9F8C5
:10412000C40C8842B4BF28464FF08070C9F8E80F2D
:10413000D9F8EC0C014621F05BFE281A22F046FA71
:10414000D9F8F01CC9F8480D8842A6BF4042814208
:10415000C9F8F00C01B0BDE8F08F0000E17A14005E
:10416000333333010100000199991900F0B5AE4CC9
:10417000D4F8E03ED4F8E42C012B81B015D14042B4
:104180008242B8BFC4F8E40CD4F8E40C0128A2BF02
:10419000A34DB5F8EE24022A03DBB5F8D420062A95
:1041A00013D1814262DD014660E09042C8BF1046F3
:1041B0000028C4F8E40C56D5994DB5F8EE24022A2F
:1041C00051DBB5F8D420062A4DD0D4F84C05D4F8EC
:1041D0005815002848BF4042002948BF494288423C
:1041E00034DBB5F8F064B5F8C604DFF87C78D4F8B1
:1041F000281DB04238BF0646786B864238BF064657
:10420000DFF84404806C082221F04AFDB6B20015A4
:10421000B042B86303D2B5F8EE04032828D194F86D
:10422000280F00F00500012804D10020C4F8E40C98
:1042300001B0F0BD0020C4F8E40CC4F84803C4F891
:10424000500301B00120C4F8980DF0BDD4F8980DCA
:1042500001280DD1D4F8100DC4F8580501B0002084
:10426000C4F8980DF0BD4942884201DAC4F8E41C54
:1042700001B0F0BD10B56C4C22F005FEC4F8240D61
:10428000FFF7C8FAD4F80C0FC0F3401000280CBF99
:10429000D4F8C40FD4F8C80F21F0B9F8D4F8100F2F
:1042A000D4F8941740F48070C4F8100FD4F8900735
:1042B00021F054FABDE8104030B55B4CE24DD4F823
:1042C000240DC4F8A40781B022F0E9FDC4F8A807C2
:1042D00022F0E8FDC4F8AC0704F29C70D4F8B017E3
:1042E0008847D4F89C17E86C21F082FDC4F8FC07DD
:1042F000D4F8A017E86C21F07BFDC4F8000804F2A4
:10430000FC70D4F810188847D4F80408D4F8441581
:104310008012A4F81E0501B0D4F808088012A4F891
:104320002005D4F80C088012A4F822054FF4A360ED
:104330002044BDE83040084710B5394C0020A4F8AF
:1043400040064FF4487006F04DFCB4F84016814228
:1043500007D04FF4487006F095FCBDE8104006F019
:104360000ABD10BD30B581B022F03BFD2C4C88B1A8
:1043700022F07DFDA4F8D20640F26935284606F009
:1043800031FCB4F8D216814204D0284606F07AFCFB
:1043900006F0F1FC22F030FD88B122F06BFDA4F8AC
:1043A000CE0640F26735284606F01CFCB4F8CE165F
:1043B000814204D0284606F065FC06F0DCFC22F0C1
:1043C00026FD88B122F059FDA4F8D0064FF45A70AA
:1043D00006F008FCB4F8D016814205D04FF45A70AC
:1043E00006F050FC06F0C7FC22F036FDA0B122F02A
:1043F00047FDA4F8CC0640F26635284606F0F2FBED
:10440000B4F8CC16814207D0284606F03BFC01B038
:10441000BDE8304006F0AFBC01B030BDB81E0500AD
:1044200038430020CCCC0C0000000020F0B5DFF8B1
:10443000F44CB4F88C0A002881B06BD0B4F8860A2A
:10444000002867D1D4F8A00EC0F34000002840F047
:10445000E8800120A4F8860A0020A4F88C0A4FF412
:104460007A60C4F8500DC4F850050020C4F858050F
:10447000C4F84C05C4F8240D6421DFF8AC0CDFF857
:10448000AC5CC4F8D40C4FF0974742F22830C4F823
:104490001805B5F8540621F0BBFB0646D4F8D41C29
:1044A000384621F045FD21F0AFFD0146112230468E
:1044B00021F0F6FBC4F86C073846D4F8D41C21F080
:1044C00037FD21F0A1FD024694F8EC0E00F0010149
:1044D000D4F89C0EC0F3001020F02EFCFCF793F9EA
:1044E00022F090FD4FF4A360D4F84815204488478B
:1044F000B5F89411481E8041C043C00FC4F8E00EC7
:104500000E20DFF82C1C0880D4F89C0E40F0100020
:10451000C4F89C0EB4F8860A002800F08280D4F813
:10452000D40C4FF0974121F003FD21F06DFD0246C0
:1045300094F8EC0E00F00101D4F89C0EC0F30010CA
:1045400020F0FAFBFFF70EFF22F06CFC30B1FFF712
:1045500009FFFCF758F9012020F09CFB22F06BFCCE
:10456000F8B1DFF8C85BB5F85406B5F84A56B5F5AA
:104570007A7F0FDD21F04EFCDFF8B81B21F0D8FC6C
:104580000646284621F046FC0146304621F052FC02
:1045900023F048FDC4F8C00ED4F84C0520F067FBAA
:1045A00001E0C4F8C00ED4F8D40EC4F8B00ED4F8AC
:1045B000D80EC4F8B40ED4F89C0EC0F3001080B32B
:1045C000D4F8980EC0F3400008B122F013FE22F098
:1045D000EDFB28B922F0F3FB10B922F0F9FB00B390
:1045E000DFF8485B0020A5F840064FF4487006F05D
:1045F000F9FAB5F84016814205D04FF4487006F03C
:1046000041FB06F0B8FB22F0D1FB30B922F0D7FB1A
:1046100038B1D4F8B80E0B2803D2FFF7A3FE03F08D
:1046200033F922F0B6FB28B9B4F8860A50B122F06B
:10463000CFFB38B12020A4F8940A01B0BDE8F040C7
:1046400017F048BE01B0F0BD145D0020B91E050092
:1046500047E1FA0047E1FAFF3333330048E1FAFF5C
:10466000AE47E10070B5DFF8BC4AB4F8860A84B002
:1046700018B122F0E9FB002853D0D4F8A037D4F8C1
:104680009C27D4F8F81CD4F8F40CDFF8A06A20F0CA
:10469000EFFE22F001FCFFF781F8B6F8BA0610B180
:1046A000012808D03AE022F0EEFBC4F8240D0120E6
:1046B000A4F8A80A2FE0B4F8A80A30BB22F0E3FB64
:1046C000D4F87817DFF8385C401A48BF40422860B9
:1046D000DFF8300C58B1D4F85805D4F88017C4F876
:1046E00068074FF4ED6020448847D4F87807B6F89F
:1046F000BC1689036960D4F8C02C9142A8BFCA4295
:1047000005DA0121A4F8A81A01E022F0BCFBC4F8E4
:10471000240DB4F8A80A20F04BFA0BE022F0B3FB0A
:1047200006E00120A4F8A80A20F042FA22F0BDFB1E
:10473000C4F8240DFFF76EF8B4F8860A10B122F021
:1047400083FBA8B3DFF84C0DDFF8B45B816BDFF8B7
:10475000280E21F005FBE860D4F8FC17084621F08C
:1047600047FB0646D4F80008014621F041FB8019BA
:1047700021F02CFFE96821F03BFB0013A8600290B8
:10478000D4F85C0FD4F8CC3CD4F8C82CD4F89417E7
:104790000190D4F8580F0090D4F8900721F00AF84F
:1047A00000F02AF8D4F8C01CD4F8E00E20F054FA37
:1047B000B4F8860A60B1D4F89417D4F8900723F0BF
:1047C0008FFB22F0E9FA18B1D4F8100DC4F858059F
:1047D00004B0BDE870406FE5CCCC0C01703D0A0020
:1047E000999919013333F3005C8F0200CDCCCC00D2
:1047F0007C3F55038FC2F5002DE9F047DFF82449CF
:10480000D4F8C00ED4F8641BDFF82089B8F8F2247D
:104810000818B8F8DE105118884228BF08464FF62D
:10482000E9518842B8F8541628BF4FF6E850C9033A
:10483000C00321F095FAD4F8EC1A0129D4F8E01E4F
:1048400008BFD4F8040B012908BF4042C4F8A00DEA
:10485000C4F84C050129D4F8680B11D1012804D102
:10486000B8F9F464B8F9F6C41AE0B8F87A06D4F8DE
:10487000B06ED4F8B4CE010012D00FFA80FC0FE075
:10488000012804D1B8F9F4C4B8F9F66408E0B8F81E
:104890007A06D4F8B46ED4F8B0CE010018BF06B2D0
:1048A00094F8280F00F00500012820D1B8F86AA973
:1048B0000FFA8CFC44F289124FEAEC73AAFB0C014C
:1048C0000AFB0311A2FB005902FB01992D0E45EAD8
:1048D000092C30B25646C117A6FB005906FB0199B8
:1048E000A2FB056702FB0977360E46EA0726A4F805
:1048F00064C5A4F8666505F069F8B8F8D400062820
:1049000002D122F043FAA0B1D4F80C0FC0F380100A
:1049100000281EBF94F8280F00F0050001280AD1D6
:10492000D4F8580D38B9D4F86C1504F24C508847B7
:1049300001E0A4F8A80AD4F8780B00281CBFB8F846
:10494000D40006280EBFD4F85805D4F8080DC4F8D2
:104950005805D4F8E01EC4F8C00C012908BF404235
:10496000461C94F8280F00F00500012805D1D4F862
:10497000600F002848BF4042461CC4F8EC6DF71792
:10498000B8F85406A0FB062300FB0733D4F8EC0A62
:10499000120E42EA0322012808BFB8F8B224C4F874
:1049A000B82EBDE8F08700009A9919006666E6FF08
:1049B0006766E6006766E6FFDFF86807D0F8EC3A5E
:1049C000D0F8002BD0F8FC1A012B3FD1DFF85C3770
:1049D000B3F8D4C0BCF1020F16D1B3F812C1BCF1C8
:1049E000030F14DA40F28D639A4226DBDFF88C1B4A
:1049F0008968521A0021C0F8A827C0F8AC17C0F87F
:104A0000FC1AC0F8002B7047BCF1030F03D0B3F8B9
:104A10001231032B11D140F28D6399420DDBDFF887
:104A20005C2B5268891A0022C0F8AC17C0F8A8277E
:104A3000C0F8FC1AC0F8002B7047D0F80C3F43F0C8
:104A40003003C0F80C3F0223C0F8EC3AC0F8FC1A5F
:104A5000C0F8002B70470000B4711C01FAEDEB00A8
:104A60009A99FFFFCDCCCC01C011002070B5DFF8C2
:104A7000105BDFF8B046B5F8D400010018BF01287C
:104A800040F00581B5F8140548B9D4F8EC0CC4F829
:104A9000A807D4F8F00CC4F8AC07E06E5AE1D4F8DB
:104AA0005805D4F88017C4F868074FF4ED60204427
:104AB0008847D4F87807E16E401AC4F83C0BD4F864
:104AC000380B012834D1D4F87011DFF8B80A21F07E
:104AD0008FF9D4F8441B494221F08AF9D4F8441BD9
:104AE0004018C4F8440B03F08BFDD4F8441B08189D
:104AF00048BF002004D4B0F1807FC8BF4FF0807061
:104B0000C4F8400BD4F83C0B22F00AF80146D4F864
:104B1000400B21F06DF9C4F8A807D4F83C0B22F043
:104B20003FF80146D4F8400B21F062F9C4F8AC0715
:104B3000D4F85C0B012804BFB5F8140501280CD08B
:104B4000D4F8C00CD4F8541B002848BF4042884217
:104B500034DAB5F81405022830D1D4F8380B01281E
:104B60002CD1D4F8080DC4F85805C4F8C00CD4F8FA
:104B700094078011C4F84803C4F8E40CD4F8AC07D7
:104B8000C4F86404C4F8F00CD4F89007C4F8F40333
:104B9000C4F8DC0CD4F8A807C4F82C04C4F8EC0C56
:104BA000DFF8F008C06C00F17F40C4F8480B4FF00C
:104BB0008070C4F84C0B0020C4F8380BD4F8701186
:104BC000DFF8C00921F014F9D4F84C1B494221F058
:104BD0000FF9D4F84C1B4018C4F84C0BD4F8380B20
:104BE00038B9D4F8EC1CC4F8A817D4F8F01CC4F8F1
:104BF000AC17D4F85C1B002904BFB5F814150129C3
:104C000012D0D4F8C01CD4F8502B002948BF494218
:104C10008A4203DAB5F81435022B05D08A4234DA19
:104C2000B5F81415032930D178BBD4F8EC1CD4F8AE
:104C3000F00C21F0F3FFE16E4018C4F87007C4F8DF
:104C40007807D4F8580BC4F85805C4F8C00CD4F849
:104C5000EC0C014621F0CCF80646D4F8F00C0146E5
:104C600021F0C6F8801921F0B1FC064603F0C8FC1B
:104C7000301AC4F8440BDFF81C08C06C00F17F4008
:104C8000C4F8480B0120C4F8380BE06E62E0B5F8B8
:104C9000121103293ADA022838D1B5F81001DFF8E9
:104CA000401CA1FB0001B0F17F4048BF002005D4AB
:104CB000DFF8301C8842A8BFDFF82C0CD4F8581558
:104CC000B5F8022580FB0101000E40EA012012B177
:104CD000D4F8F02D8018C4F86807C4F8EC0D4FF430
:104CE000ED60D4F880172044884703F089FCC4F8AD
:104CF000A807B5F8020528B1B5F8CA0410B900F044
:104D000003F923E00020C4F8AC071FE0B5F83E012A
:104D1000012804D0D4F8500DB0F5FA5F30DA6420E1
:104D2000C4F8180E00F045F900F006FA00F0ECFAAD
:104D300000F0B2FBD4F87C0EC4F8EC0DC4F86807A0
:104D40004FF4ED60D4F8801720448847FFF734FE15
:104D5000D4F87807D4F8B017C4F8A40704F29C700C
:104D60008847B5F8D400010018BF012864D1B5F810
:104D7000140530BBDFF81C57D4F89C17E86C74E0BE
:104D8000D4F8180E032803D30020C4F8180E04E04A
:104D900018B102280FD006D3C4E700F00AF90120A9
:104DA000C4F8180EC6E700F0C7F900F075FB022042
:104DB000C4F8180EBEE700F0A7FA0020C4F8180ED9
:104DC000B8E7B5F8340188BBD4F87011DFF8B40740
:104DD00021F00EF8D4F8481B494221F009F8D4F824
:104DE000481BD4F8382B4018D4F89C17C4F8480B4B
:104DF000012A0CD100F1807020F0FAFFC4F8FC0702
:104E0000D4F8480BD4F8A01700F1807034E0DFF834
:104E10008456EA6C101A20F0EBFFC4F8FC07D4F8B3
:104E2000482BE86CD4F8A017801A25E0DFF8645608
:104E3000D4F89C17E86C18E0D4F8C00CDFF8B81C64
:104E4000002848BF4042884206DBD4F8D40A002834
:104E50005CBF0020C4F8D40AD4F8D40ADFF8345672
:104E600000F18070E864D4F89C1720F0C1FFC4F80A
:104E7000FC07D4F8A017E86C20F0BAFFC4F80008CB
:104E800004F2FC70D4F810188847D4F80408D4F859
:104E900044158012A4F81E05D4F808088012A4F85E
:104EA0002005D4F80C088012A4F822054FF4A36062
:104EB0002044BDE87040084710B59C4CB4F8300160
:104EC00023F0C2F8B4F8460623F0C1F8B4F854064B
:104ED00023F0C0F8B4F86E0623F0BFF8B4F87206F9
:104EE00023F0BEF8B4F8980623F0BDF8DFF8280DDB
:104EF000D0F8D41C4FF0974021F01AF821F084F834
:104F0000BDE8104023F0E2B870B58848B0F83E1113
:104F1000012905D0B0F8320140F2DD5188422DDB85
:104F2000804CD4F85815D4F8E00E23F09FF8DFF841
:104F30006405806C23F0ADF8D4F8A80723F0ACF832
:104F4000D4F89467D4F89057D4F8D40C4FF0974124
:104F500020F0EEFF21F058F83246294623F096F96A
:104F600023F022FBC4F8A80723F021FBC4F8AC0708
:104F700023F020FB6B49C1F8F00D70BD694A694907
:104F80000020C2F8AC07C1F8F00D70BD40F223312B
:104F900088420DD1DFF8840CB0F84606232148433F
:104FA0006421B0FBF1F189B24FF4537005F06ABE91
:104FB000704730B55B4CD4F81016D4F8D8050029EA
:104FC00048BF4942002881B048BF404221F026FE38
:104FD000C4F818064FF4C360D4F83016204488474C
:104FE000D4F82C06D4F84C16C4F8340604F2346015
:104FF0008847D4F8380ED4F8341ED4F84826401C1C
:105000005118D4F8302E212802D34A110021002053
:10501000C4F8380EC4F8341ED4F82C0E8242B8BF3F
:10502000024604DBB2F5800FC8BF4FF48002C4F81B
:10503000302E104621F074FDC4F83C0ED4F8300E2A
:1050400021F0AEFDC4F8400ED4F8D805014620F09A
:10505000CFFE0546D4F81006014620F0C9FE4019DF
:1050600021F0B4FAC4F8F8064FF4DF60D4F8101752
:1050700020448847D4F80C07D4F82C17C4F8140738
:1050800004F214708847D4F8C00DD4F82817081813
:10509000D4F8C41D491C202904D34011C4F8200EA3
:1050A00000210020C4F8C41DC4F8C00DD4F8401E6F
:1050B000D4F8200E20F09CFEC4F8240ED4F83C1E38
:1050C000D4F8200E20F094FEC4F8280E0A21DFF850
:1050D000B004B0F8460620F0B9FF0146D4F8200E1F
:1050E000082220F0DDFDC4F8B80D0822D4F83C1EDB
:1050F00020F0D6FDC4F8BC0D0921012020F030FEBF
:10510000D4F8301E8842B8BF4FF0807005DB4FF0F6
:10511000106020F06DFEC0F10070C4F85C0E01B0AC
:1051200030BD0000000000206F128339384300209A
:105130002421002000007A4470B5DFF8DC4ADFF853
:10514000E05AD4F8E02ED4F8800ED4F85815012A8D
:105150000CBF081A4018C4F87C0E0028D4F8781D3B
:1051600048BF404220F0FCFDC4F8500ED4F8901D1A
:1051700020F03EFEA842A8BF4FF08070C4F8440E55
:10518000D4F8241ED4F8A40D20F032FEC4F8480E42
:10519000D4F8281ED4F8A40D20F02AFEC4F84C0E32
:1051A000D4F8441E084620F023FE0646D4F8480EE4
:1051B000014620F01DFE301A0128C4F8500E06DB0F
:1051C00021F004FAD4F84C1E4018C4F84C0EEC48F8
:1051D000B0F834110A0029D001290BD0D4F8C01E30
:1051E000D4F8B82E91421AD3D4F8E01ED4F8DC2EAD
:1051F000914214D1DFF82C1AB0F84406096820F067
:10520000AFFDDFF8241A20F0F3FDC4F8680ED4F8DF
:10521000441E20F0EDFDD4F8441E401A0BE0D4F8F3
:10522000641ED4F8440E20F0E3FD04E04FF08070DB
:10523000C4F8680E0020C4F8640ED4F8441ED4F8F4
:105240004C0E411AD4F85C0E20F0D2FD0646D4F87C
:10525000601ED4F8F00620F0CBFDDFF8D01920F066
:10526000C7FDD4F8641E89194018C4F8540E4FF0D5
:105270002070D4F8F01620F0BBFDD4F8441E20F0C6
:10528000B7FDD4F8541EC4F8500E8842B8BFC4F815
:10529000540ED4F8540EDFF898198842A4BFDFF8F2
:1052A0009409C4F8540ED4F8540ED4F86816C4F80F
:1052B00050064FF4CA6020448847D4F86406D4F8F6
:1052C0008416C4F86C0604F26C608847D4F8440E67
:1052D000D4F880160818D4F8681E8142B8BF084672
:1052E000A842A8BF4FF0807002DA002848BF002013
:1052F000C4F8580EC4F8AC070020C4F8A80770BD65
:10530000781200208D6D020870B59D4DDFF80849B8
:10531000B5F84C064FF4FA7120F098FED4F8B81D99
:105320000646084620F0DAFE314620F0D7FEC4F8E3
:10533000700ED4F8BC1DD4F8B40D20F0CFFED4F814
:10534000701E401AC4F8740ED4F8BC1DD4F8B40D05
:1053500020F0C4FED4F86C1E20F0C0FED4F8741EF9
:10536000C4F8780E8142B8BFC4F8740EB5F8480688
:10537000042120F06BFE0546D4F8741E4FF4406003
:1053800020F0ACFE294620F0A9FEC4F8700E6FF0A4
:105390000102D4F87C0ED4F8301D002848BF4042EA
:1053A00020F07EFCD4F8101E20F098FEC4F8740E95
:1053B0000146D4F8700E20F049FED4F8901E8142C8
:1053C000B8BF0846C4F8D00DD4F8CC1D20F0C8FCF6
:1053D000C4F8C0064FF4D860D4F8D81620448847E3
:1053E000D4F8D406D4F8F416C4F8DC0604F2DC6071
:1053F0008847D4F87C0EDFF84018002848BF4042A8
:105400008842A8BFD4F8880E0FDA5E498842B8BF38
:10541000D4F8840E09DBDFF824180918D4F88C0EB0
:1054200020F0E6FCD4F8881E4018C4F8700ED4F8BA
:10543000DC1DD4F8F00620F0DBFC0146D4F8700E39
:1054400020F0D6FCC4F8740EC4F888064FF4D1607E
:10545000D4F8A01620448847D4F89C06D4F8BC168B
:10546000C4F8A40604F2A4608847D4F8E40DD4F884
:10547000B8160818D4F8E81D491C202904D3401197
:10548000C4F8800E00210020C4F8E81DC4F8E40D23
:1054900070BD0000145D0020F0B5394EDFF878478C
:1054A000B6F8D400022881B01FD1B6F81201032843
:1054B0001DD0D4F8D855D4F8F80DD4F8FC1D401CF4
:1054C0008842C4F8F80D4DD30020C4F8F80D2946E1
:1054D000D4F8580520F044FC0028D4F85805294693
:1054E00008D520F03DFC404206E00328E1D1D4F885
:1054F0001056E0E720F034FCC4F8700E4FF07F4106
:1055000020F076FC0146D4F8F40DDFF83477C4F8C7
:10551000741E281A786020F06BFCC4F8700E94F8A2
:105520009C0EB6F85416C00754BF0F20B6F8C0053D
:1055300020F016FC38604142D4F8702E8A42B8BF81
:10554000C4F8701E03DB9042B8BFC4F8700ED4F8E4
:10555000E01ED4F8700EC4F8F45D012908BF404283
:10556000C4F8F00DD4F87C0ED4F8F01D0818C4F877
:105570007C0E01B0F0BD00005A64BB014861002000
:1055800038430020B81E0500F0B5DFF88C46DFF880
:10559000B456D4F87807DFF8B076C4F8240D81B09B
:1055A000FEF738F92A6CE86B80FB000182FB0223CE
:1055B000C00ED20ED5F844C040EA411042EA431270
:1055C00012188CFB0C01C00E40EA41108018DFF865
:1055D0007C1681FB0001400D40EAC120386021F0BB
:1055E00069FA3860C000DFF86816DFF8307681FBB2
:1055F0000001000E40EA0120C4F8080BC4F8F00ACC
:10560000B7F8D0000328B8BF4FF05C5602DB08BFE4
:105610004FF0BE46B7F83E01012806D1B7F8D400D6
:10562000022814BF03280A2005D0D4F8500D4FF4E7
:10563000C87190FBF1F0A4F8A00AD4F8281DDFF897
:10564000140620F08DFBC4F8FC0FB7F85406C10314
:10565000D4F8C00EC00320F083FBD4F8E01ED4F8C9
:10566000B42E012908BF4042C4F8A00DC4F84C056F
:105670000129D4F8B00E0EBF11460146104694F829
:10568000282F02F00502012A0BD1B7F86A2909B2C6
:1056900000B251434FF47A73504391FBF3F190FB06
:1056A000F3F0A4F86605A4F86415B7F8BC0401008B
:1056B00036D1D4F80C0FC0F340100028B7F8D4004E
:1056C0000DD1022807D1B7F81201032803DAB7F881
:1056D000B40431460CE0B7F8B404314611E00228B6
:1056E0000CD1B7F81201032808DAB7F8B60431462E
:1056F000800520F035FB0146002006E0B7F8B6042F
:105700003146800520F02CFB0021C4F8AC07C4F81A
:10571000A817D4F8100F40F48070C4F8100F96E06A
:10572000012851D1D4F80C0FD4F8AC14C0F34010B8
:1057300000280CBFD4F8F40AD4F8F80AC4F87C04A2
:10574000D4F8F00AC4F878044FF48F6020448847F6
:10575000D4F8A404002848BF44F2891004D4B0F15E
:10576000807F03DD4FF08070C4F8A404B7F8D40044
:1057700002280BD1B7F8121103291CDAD4F8A404BB
:10578000C4F8A8070020C4F8AC0770E0032813D0C1
:1057900000286ED1D4F8A404C4F8A8070020C4F8E7
:1057A000AC07D4F8600DC4F8A407E06EC4F8680D27
:1057B000C4F8600D5DE0EBD1D4F8A404C4F8AC07E4
:1057C0000020C4F8A80752E0022852D1D4F80C0FE8
:1057D000C0F340100028B7F8D4001DD102280FD123
:1057E000B7F8120103280BDAB7F8B4043146800584
:1057F00020F0B6FAC4F8A8070020C4F8AC0726E0E9
:10580000B7F8B4043146800520F0AAFAC4F8AC0712
:105810000020C4F8A8071AE0022807D1B7F812211F
:10582000032A06DA0020C4F8AC070AE0032801D1F5
:1058300004E003D0002818BF012802D10020C4F8DA
:10584000A807D4F8100F40F48070C4F8100FB7F810
:10585000D400010018BF012807D1E06EC4F8A407E6
:10586000C4F8680DC4F8600D03E0D4F87807C4F8F4
:10587000A407D4F8B01704F29C708847B7F8D40096
:1058800010B14FF08070E864D4F89C17E86C20F0F9
:10589000AFFAC4F8FC07D4F8A017E86C20F0A8FA17
:1058A000C4F8000804F2FC70D4F810188847D4F843
:1058B0000408D4F844158012A4F81E0501B0D4F8E9
:1058C00008088012A4F82005D4F80C088012A4F867
:1058D00022054FF4A3602044BDE8F04008470000D3
:1058E0005C8F02009A99190199991901F0B5CB4C76
:1058F000B4F8D40001001CBF0128062881B040F094
:10590000A180C54DB4F86206D5F8B83E02469A4269
:105910000DD3B4F85A064FF0C871800421F0E6F9AF
:10592000C5F8C80C4FF0C871B4F85C0685E0B4F84F
:1059300064160E469E4237D3081AC103981AC00354
:1059400021F0D4F90646B4F85E0681040E223046F2
:1059500020F0A6F90746B4F85A0681040E22304614
:1059600020F09EF9B4F85A2607EB82424FF0C87136
:10597000101A21F0BBF9C5F8C80C0E22B4F8600665
:105980008104304620F08CF90746B4F85C068104A7
:105990000E22304620F084F9B4F85C2607EB8242F0
:1059A0004FF0C871101A49E0B4F86A06984237D32C
:1059B000401AC103981BC00321F098F90646B4F8B9
:1059C000660681040E22304620F06AF90746B4F8D4
:1059D0005E0681040E22304620F062F9B4F85E269D
:1059E00007EB82424FF0C871101A21F07FF9C5F819
:1059F000C80C0E22B4F868068104304620F050F935
:105A00000746B4F8600681040E22304620F048F9BB
:105A1000B4F8602607EB82424FF0C871101A0DE00F
:105A2000B4F866064FF0C871800421F05FF9C5F83C
:105A3000C80C4FF0C871B4F86806800421F056F91C
:105A4000C5F8CC0C01B0F0BD744830B5B0F84A03CD
:105A5000002881B03FD08048008800283BD17F4C8F
:105A60004021204622F086FE40B36B497C4D91F8E0
:105A7000581A288801290FD1062807BF79480188BC
:105A8000794931F81010204622F06CFE2888401C1D
:105A9000288080B207280EE0052807BF71480188DA
:105AA000714931F81010204622F05CFE2888401C15
:105AB000288080B20628A4BF00202880202120460C
:105AC00022F058FE38B1204622F050FE674900F01F
:105AD000FF00088003E066480088012806D1644979
:105AE00000200880634961480088088001B0BDE853
:105AF000304015F0ACBB00006766E60070B4464865
:105B0000D0F84C124FF4137500230A4600240544C4
:105B10002E68B142B8BF31469642B8BF3246F3183C
:105B20006E68641CB142B8BF31469642D8BF324657
:105B3000F318AE68641CB142B8BF31469642D8BF74
:105B40003246F318641C0C35122CE1DB591A891A01
:105B50000911C0F8581C70BC704770B42E48D0F8BA
:105B600094124FF4257500230A46002405442E683C
:105B7000B142B8BF31469642B8BF3246F3186E689C
:105B8000641CB142B8BF31469642D8BF3246F318C2
:105B9000AE68641CB142B8BF31469642D8BF3246A7
:105BA000F318641C0C35122CE1DB591A891A0911FF
:105BB000C0F85C1C70BC704770B41748D0F8DC1299
:105BC0004FF4377500230A46002405442E68B1427D
:105BD000B8BF31469642B8BF3246F3186E68641CAF
:105BE000B142B8BF31469642D8BF3246F318AE68CC
:105BF000641CB142B8BF31469642D8BF3246F31852
:105C0000641C0C35122CE1DB591A891A0911C0F8F1
:105C1000601C70BC7047000000000020384300206A
:105C20000100000194120020900F6A019999190057
:105C30006766260066662600676666009A9999FF81
:105C40006C610020145D0020DC630020A9AA0A001A
:105C5000E7FB6901333303001E21002000380140B7
:105C6000F020002002210020E02000201021002050
:105C70000E210020222100202DE9F04FDFF8208E98
:105C8000B8F8D400042881B007DB062841F0D181A0
:105C900001B0BDE8F04FFEF7C9BBDFF8089EB9F8C8
:105CA000860A002840F01781B9F8880AB8F840162B
:105CB000014352D1B8F84C064FF0FA71C00320F0FE
:105CC0004FF8C9F8B40BD9F83C1D20F049F8C9F8D1
:105CD000D40B4FF0FA71B8F84E06C00320F040F82C
:105CE000C9F8BC0BD9F83C1D20F03AF8C9F8DC0B18
:105CF000DFF8B41DB8F85006000320F031F8C9F8F9
:105D0000CC0BD9F8401D20F02BF8C9F8F80BDFF8C0
:105D10009C1DB8F85206000320F022F8C9F8C80B01
:105D2000D9F8401D20F01CF8C9F8E80BD9F8C81BB9
:105D3000D9F8CC0B0818C9F8C00BD9F8401D20F0D1
:105D40000FF8C9F8E00BC9F8E40B0120D9F8C01B23
:105D5000C9F8C41BA9F8880ABDE0B9F88C1A012952
:105D600001BF0028D9F8A00EC0F34000002841F080
:105D700060810120A9F8860A42F22830C9F8180586
:105D8000B8F8D000032809D1B8F8CE0040F23A7133
:105D9000884203DBB8F97006404200E00020A9F811
:105DA0003C050020DFF8087DB8863887B8874FF0BB
:105DB0009744B8F85406C103B8F87606C0031FF03C
:105DC000CFFFC9F8800B6421B8F9E400A9F8640595
:105DD000B8F9E600A9F866054FF47A60C9F85005ED
:105DE0000020C9F85805C9F87807DFF8C80CC9F8C9
:105DF000D40CB8F854061FF00BFF0646D9F8D40CA3
:105E0000214620F095F820F0FFF801461722304691
:105E10001FF046FFC9F8880B6421B8F854061FF03C
:105E2000F7FE0646D9F8D40C214620F081F820F080
:105E3000EBF80146112230461FF032FFC9F86C071B
:105E40002146D9F8D40C20F073F820F0DDF8C9F819
:105E5000180109F1E000D9F8A8118847FBF7E8F923
:105E6000FBF776FAD9F88C0132214843D9F8701142
:105E7000C9F80C09C9F82409C9F83C09C9F854093A
:105E8000C9F80819C9F82019C9F83819C9F85019FA
:105E9000B8F84006032805D04FF4A360D9F8481598
:105EA00048448847D9F89C0EDFF8181E40F01000CF
:105EB000C9F89C0E0120A9F88A0A0020A9F88C0ACA
:105EC0000E2008800020A9F8820AC9F8980BC9F8AA
:105ED000940B0DF067FEB9F8860A012802BFD9F8C5
:105EE000A00EC0F34000002841F0A380DFF8D80DD9
:105EF00001884FF67F721140DFF8D02D13884FF6DE
:105F0000F7763340B8F8946136B94FF6BF74214044
:105F10004FF6EF74234004E0012641F0400143F0C6
:105F20001003C9F8DC6E13800180C9F8E06E99F89F
:105F3000583A0088DFF8981DDFF8982D012B18D10A
:105F400055231380702353801F2393805B23D380BA
:105F500070231381FF23538155220A804B817022C5
:105F60004A8088811F228A805B22CA8070220A812F
:105F700013E0552313805081F823538086239380A8
:105F80009223D380F823138155220A804B808622E6
:105F90008A800B819222CA80488142F2283BDFF836
:105FA000381DB8F89206096800FB0BF0B0FBF1F061
:105FB000ABEB0000A9F89E0AB8F8D0100329B8BFCF
:105FC0006C200CDB0DD1B8F8CE00DD28B8BF562010
:105FD00005DB40F2EF229042B4BF5D20B420A9F867
:105FE0006C0AB9F88A0A020007D1DFF8F06C306851
:105FF00040F48060306000F059BFB8F84026032AB2
:1060000008BF012840F0E480D9F8E80ADFF8D0ACF6
:1060100000EB800252000329B4BFDFF8E04DDFF847
:10602000E04D04EB820140F22630096989B204F0A8
:1060300029FED9F8E80A00EB8001480004EB800053
:1060400040F22735416989B2284604F01BFED9F891
:10605000E80ADFF8B05D00EB8001480004EB800047
:1060600040F22936816989B24FF44A7004F00AFE81
:10607000D9F8E80A00EB8001480004EB80004FF0FB
:10608000000BC16989B2304604F0FCFDDFF8784DA1
:10609000DFF8486CB9F8820A002845D1D9F89C0E7F
:1060A0000BF1010BC0F3001010B102200DF058FDF0
:1060B000FFF7CAFCBAF80000442810D0D9F8F00E57
:1060C00000F44170B0F5417F09D1D9F8FC0EC0F35E
:1060D000002000281CBFB9F8840A002804D101F070
:1060E000D3FB0120A9F8820AD9F8281DA86B082241
:1060F0001FF0D6FD001520602168B8F8BA05884267
:1061000003DBBBF5FA6FC5DB0EE00020A9F88A0AB5
:106110000320A9F8940A306840F00200306016F0BD
:10612000D9F80120A9F8820A5FF00007B9F8820ABD
:10613000002848D1D9F89C0E7F1CC0F3001010B184
:1061400002200DF00DFDFFF77FFCBAF80000442897
:1061500010D0D9F8F00E00F44170B0F5417F09D1AC
:10616000D9F8FC0EC0F3002000281CBFB9F8840A3F
:10617000002804D101F088FB0120A9F8820AD9F88F
:10618000281DA86B08221FF08BFD001520602168D8
:10619000B8F8BA05884207DBB7F5FA6FC6DB04200A
:1061A000A9F88A0A00F082BE0020A9F88A0A032012
:1061B000A9F8940A306840F00200306016F08AF8BE
:1061C0000120A9F8820A0420A9F88A0A00F06EBE0C
:1061D000012840F06682112244F289114FF4C81060
:1061E0001FF05EFDC9F888041122DFF84C1EDFF8AD
:1061F000C078DFF8144CDFF80C5CDFF8E4AADFF8B5
:10620000DC6A4FF420301FF04BFDC9F88404A9F874
:1062100068BAD9F8180100EB80014800C9F8800479
:106220004FF08070C9F89004C9F88C040020C9F8B8
:106230009C04A9F87C0AA9F8640A4FF40000C9F884
:106240007C040020A9F87E0A3068C0F38020002872
:1062500004BFB9F8820A00284FD1B9F89E0AB9F8EC
:10626000681A81420CD2A9F8680A0021384620F049
:1062700040F90020A9F88A0A306840F48060306054
:10628000FFF7E2FBBAF80000442810D0D9F8F00E6E
:1062900000F44170B0F5417F09D1D9F8FC0EC0F38C
:1062A000002000281CBFB9F8840A002804D101F09E
:1062B000EBFA0120A9F8820AD9F8281DA86B082258
:1062C0001FF0EEFC001520602168B8F8BA0588427E
:1062D0000EDA0020A9F88A0A0320A9F8940A306887
:1062E00040F00200306015F0F5FF0120A9F8820AA5
:1062F000B9F87E0AB0F5FA6FA6DBB9F88A0A002869
:1063000063D03068C0F3802000285ED10120A9F856
:10631000640A0027B9F8820A002847D1B9F88A0A26
:10632000002852D0D9F89C0E7F1CC0F3001010B189
:1063300002200DF015FCFFF787FBBAF80000442897
:1063400010D0D9F8F00E00F44170B0F5417F09D1BA
:10635000D9F8FC0EC0F3002000281CBFB9F8840A4D
:10636000002804D101F090FA0120A9F8820AD9F896
:10637000281DA86B08221FF093FC001520602168DF
:10638000B8F8BA05884202DB962FC3DB0EE0002086
:10639000A9F88A0A0320A9F8940A306840F002009C
:1063A000306015F097FF0120A9F8820AB9F88A0A2F
:1063B00058B1FFF7D2FBFFF7FFFBD9F85C0CC9F827
:1063C000980CD9F8600CC9F8640C0020A9F87C0A74
:1063D000A9F8640ADFF8640CC9F87C040020A9F865
:1063E0007E0AB9F88A0A002800F05B813068C0F3A1
:1063F0008020002840F06580B9F8820A00285BD12F
:10640000B9F89E0AB9F8681A814213D2A9F8680A45
:106410000021DFF89C76384620F06BF800228021BE
:10642000384620F071F80020A9F88A0A306840F454
:1064300080603060FFF708FBBAF80000442810D0F5
:10644000D9F8F00E00F44170B0F5417F09D1D9F8C8
:10645000FC0EC0F3002000281CBFB9F8840A0028F5
:1064600004D101F011FA0120A9F8820AD9F8281DF7
:10647000A86B08221FF014FC001520602168B8F8F2
:10648000BA0588420EDA0020A9F88A0A0320A9F882
:10649000940A306840F00200306015F01BFF0120C4
:1064A000A9F8820AB9F87E0AB0F5FA6F04DA306802
:1064B000C0F3802000289FD0B9F88A0A002800F095
:1064C000F0803068C0F38020002840F0EA8001208E
:1064D000A9F8640A5FF00007B9F8820A002848D1D9
:1064E000B9F88A0A002800F0DC80D9F89C0E7F1CDD
:1064F000C0F3001010B102200DF032FBFFF7A4FA38
:10650000BAF80000442810D0D9F8F00E00F4417019
:10651000B0F5417F09D1D9F8FC0EC0F30020002866
:106520001CBFB9F8840A002804D101F0ADF901209C
:10653000A9F8820AD9F8281DA86B08221FF0B0FB21
:10654000001520602168B8F8BA05884202DB962F52
:10655000C2DB0EE00020A9F88A0A0320A9F8940AF9
:10656000306840F00200306015F0B4FE0120A9F858
:10657000820AB9F88A0A002800F09380FFF7BEFA71
:10658000FFF7EBFAFFF718FBD9F8643CD9F8580C81
:10659000D9F85C1CD9F8602CC9F8900C9A42C9F85B
:1065A000941CC9F8682C06DA0020C9F8D40BA9F8A5
:1065B0008A0A00F07BBCD9F8982C891A1FF018FCC5
:1065C000D9F8681CD9F8642CC9F8500C891AC9F894
:1065D000541C00271FF0C4FB0146DFF8640A1FF0BB
:1065E00007FCC9F8D40BD9F83C1D1FF001FCC9F811
:1065F000B40B0021DFF8B8041FF07BFFB9F8820A62
:10660000002847D1B9F88A0A00284AD0D9F89C0E48
:106610007F1CC0F3001010B102200DF0A1FAFFF7AB
:1066200013FABAF80000442810D0D9F8F00E00F49C
:106630004170B0F5417F09D1D9F8FC0EC0F30020BC
:1066400000281CBFB9F8840A002804D101F01CF905
:106650000120A9F8820AD9F8281DA86B08221FF08A
:106660001FFB001520602168B8F8BA05884202DBDC
:10667000642FC3DB0EE00020A9F88A0A0320A9F8E2
:10668000940A306840F00200306015F023FE0120CB
:10669000A9F8820AB9F88A0A18B10220A9F88A0A68
:1066A00004E0B9F88A0A022840F01C82B9F8860A88
:1066B000012840F01782DFF824663078C00700F127
:1066C00011820020A9F87C0AA9F8640AC9F8A00B75
:1066D000C9F8A40BC9F8AC0BA9F86E0AC9F86C0C80
:1066E000C9F8700CC9F8740CC9F8780CC9F87C0C9E
:1066F000C9F8800CC9F89C0CA9F868BAD9F8881BAD
:10670000D9F8800BDFF83C4908221FF0C9FAC9F814
:10671000840BB8F87616DFF83009C9F89C4BB0FB4B
:10672000F1F0A9F8800A0020A9F8640A03F0D0FC6F
:10673000D9F89C0EC0F3001010B102200DF010FA31
:10674000112244F289114FF4C8101FF0A9FAC9F8B8
:1067500088041122DFF8E018DFF8A856DFF880A5DA
:106760004FF420301FF09CFAC9F88404C9F87C4427
:10677000D9F81801DFF8904600EB80014800C9F80D
:1067800080044FF08070C9F89004C9F88C04002090
:10679000C9F89C04A9F87E0A3068C0F3802000285C
:1067A00004BFB9F8820A00283CD1FFF74DF9BAF8C6
:1067B0000000442810D0D9F8F00E00F44170B0F574
:1067C000417F09D1D9F8FC0EC0F3002000281CBF7E
:1067D000B9F8840A002804D101F056F80120A9F87C
:1067E000820AD9F8281DA86B08221FF059FA001553
:1067F00020602168B8F8BA0588420EDA0020A9F8AE
:106800008A0A0320A9F8940A306840F00200306038
:1068100015F060FD0120A9F8820AB9F87E0AB0F5EA
:10682000FA6FB9DB0020A9F8780A00275FF00100B1
:10683000A9F8640AB9F8820A002849D1B9F88A0A85
:10684000002800F04F81D9F89C0E7F1CC0F3001087
:1068500010B102200DF084F9FFF7F6F8BAF8000045
:10686000442810D0D9F8F00E00F44170B0F5417F03
:1068700009D1D9F8FC0EC0F3002000281CBFB9F8DC
:10688000840A002804D100F0FFFF0120A9F8820A41
:10689000D9F8281DA86B08221FF002FA0015206005
:1068A0002168B8F8BA05884203DBB7F5487FC1DB39
:1068B0000EE00020A9F88A0A0320A9F8940A30689B
:1068C00040F00200306015F005FD0120A9F8820AB1
:1068D000B9F88A0A002800F00581FFF70FF9FFF7E1
:1068E0003CF9FFF769F9D9F85C1CC9F8841C002051
:1068F000A9F8640AA9F87C0AD9F8601CD9F8580CE0
:10690000C9F88C0CC9F8881C20F00AF9C9F8900B5A
:10691000D9F88C0C20F044F9C9F88C0B4FF00070BA
:10692000D9F8841C1FF064FA0746D9F8901BD9F8EF
:10693000880C1FF05DFA39461FF012FAC9F8D80B1F
:106940004FF0C071D9F8D40B1FF052FAD9F8D81B08
:106950008842B8BF0846C9F8D80BD9F8D41B401AEA
:10696000C9F8DC0B4FF00070D9F8841C1FF040FA16
:106970000746D9F88C1BD9F8880C1FF039FA39462C
:106980001FF0EEF9C9F8EC0B4FF00070D9F8801B3E
:106990001FF02EFA0146D9F8EC0B1FF0E1F9C9F807
:1069A000F80BC9F8FC0BB8F87806642810DA4FF039
:1069B000C84100061FF0D4F90146D9F8D40B1FF0E6
:1069C00017FAD9F8DC1B8142B8BF0146C9F8DC1BB5
:1069D000D9F83C1DD9F8D80B1FF00AFAC9F8B80B42
:1069E0000027D9F83C1DD9F8DC0B1FF001FAC9F8D3
:1069F000BC0BD9F8401DD9F8F80B1FF0F9F9C9F80C
:106A0000CC0BD9F83C1DD9F8EC0B1FF0F1F94FF481
:106A100000011FF0EDF9C9F8D00B002124481FF048
:106A200068FD00BFB9F8820A002854D1B9F88A0A73
:106A3000002857D0D9F89C0E7F1CC0F3001010B16D
:106A400002200DF08DF8FEF7FFFFBAF80000442891
:106A500010D0D9F8F00E00F44170B0F5417F09D1A3
:106A6000D9F8FC0EC0F3002000281CBFB9F8840A36
:106A7000002804D100F008FF0120A9F8820AD9F803
:106A8000281DA86B08221FF00BF900152060216853
:106A9000B8F8BA0588420FDB642FC3DB1BE000BFE8
:106AA000384300200000002000006A180000710236
:106AB000002C01406F1283390020A9F88A0A0320B4
:106AC000A9F8940A306840F00200306015F002FC2A
:106AD0000120A9F8820AB9F88A0A18B10320A9F896
:106AE0008A0A04E0B9F88A0A032840F0DF81B9F87D
:106AF000860A012840F0DA81784E3078C00700F12C
:106B0000D581B8F84006012840F06A810020A9F834
:106B1000640AA9F87C0AB8F89411D9F8800B21B955
:106B2000B8F9E410B8F9E62006E04042C9F8800B55
:106B3000B8F9E610B8F9E420B34CB24DDFF8A0A1E3
:106B4000C9F84C05A9F864150020A9F86E0AC9F81F
:106B5000AC0BC9F86C0CC9F8740CC9F8780CC9F8FE
:106B60007C0CC9F8800CA9F8780AA9F86625D9F830
:106B7000800BD9F8881B002848BF404208221FF02C
:106B80008FF8C9F8840BB8F87616DFF8BC04B0FBB0
:106B9000F1F0A9F8800A4FF4A360D9F848154844E9
:106BA000884700BFD9F8C00CD9F8801B884242D072
:106BB000B9F8820A00283ED1B9F88A0A00283AD0EA
:106BC0000020A9F8780AFEF73FFFBAF80000442831
:106BD00010D0D9F8F00E00F44170B0F5417F09D122
:106BE000D9F8FC0EC0F3002000281CBFB9F8840AB5
:106BF000002804D100F048FE0120A9F8820AD9F843
:106C0000281DA86B08221FF04BF800152060216892
:106C1000B8F8BA058842C5DA0020A9F88A0A032024
:106C2000A9F8940A306840F00200306015F052FB79
:106C30000120A9F8820A0020A9F8780A002701207B
:106C4000A9F8640AB9F8820A00285AD1B9F88A0A60
:106C5000002800F00481D9F89C0E7F1CC0F30010BE
:106C600010B102200CF07CFFFEF7EEFEBAF8000037
:106C7000442810D0D9F8F00E00F44170B0F5417FEF
:106C800009D1D9F8FC0EC0F3002000281CBFB9F8C8
:106C9000840A002804D100F0F7FD0120A9F8820A37
:106CA000D9F8281DA86B08221EF0FAFF00152060F5
:106CB0002168B8F8BA05884214DBB7F57A7FC1DBE2
:106CC0001FE000BF2421002000210020022100201D
:106CD000E0200020D020002094120020905E0020B0
:106CE000222100200020A9F88A0A0320A9F8940A8A
:106CF000306840F00200306015F0ECFA0120A9F88D
:106D0000820AB9F88A0A002800F0A9800020A9F8B0
:106D1000640AA9F87C0AFEF7F1FEFEF71EFFD9F817
:106D2000580CD9F85C1CC9F88C0CC9F8841C1FF0ED
:106D3000F7FEC9F8900BD9F88C0C1FF031FFC9F899
:106D40008C0BD9F8901BD9F89C0C1FF051F8D9F88E
:106D5000841C1FF005F8C9F8F00BD9F88C1BD9F882
:106D60009C0C1FF045F8D9F8841C1EF0F9FF06466C
:106D7000D9F8EC1B4FF400001FF03AF8D9F8801B4B
:106D8000301AC9F8F40B002948BF49421EF0E8FF49
:106D9000C9F8E80BD9F8F81B0818C9F8E00BC9F8CE
:106DA000E40BD9F8401D1FF023F8C9F8C00BD9F83F
:106DB000401DD9F8E40B1FF01BF8C9F8C40BD9F833
:106DC000401DD9F8E80B1FF013F8C9F8C80BD9F823
:106DD000401DD9F8F80B1FF00BF8C9F8CC0B3EE0BA
:106DE00002283CD1D9F8E80A00EB80014800B8F845
:106DF000D0100329B4BF0149014907E0D0C70208F8
:106E0000C4CB0208145D00209812002001EB800022
:106E100040F22936C16989B2304603F033FF03F0EE
:106E2000AAFFB8F85206DFF8301A00021EF098FFE9
:106E3000C9F8C80BD9F8401D1EF092FFC9F8E80B3D
:106E4000D9F8C81BD9F8CC0B0818C9F8C00BD9F869
:106E5000401D1EF085FFD9F8C00BC9F8C40BD9F846
:106E6000E80BD9F8F81B0818C9F8E00BC9F8E40BCF
:106E7000D9F8401D1EF0BCFFC9F8C00BD9F8401D61
:106E8000D9F8E40B1EF0B4FFC9F8C40BD9F8401DC3
:106E9000D9F8E80B1EF0ACFFC9F8C80BD9F8401DB3
:106EA000D9F8F80B1EF0A4FFC9F8CC0BB8F84006CF
:106EB000032803D10020C9F8800BA8E0B9F88A0A9A
:106EC000002800F0A980B9F8860A012840F0A280C5
:106ED000D9F8B40B01224FF47A311EF0E1FE4010D4
:106EE000A8F84C0681B240F2263003F0CBFED9F868
:106EF000BC0B01224FF47A311EF0D2FE4010A8F8EC
:106F00004E0681B240F2273003F0BCFED9F8CC0B1C
:106F1000DFF8481901221EF0C3FE40100128B8BF57
:106F20000120A8F8500681B24FF44A7003F0AAFE7F
:106F3000B8F8400601280ED1D9F8C80BDFF81819A7
:106F400001221EF0ADFE4010A8F8520681B240F2B8
:106F5000293003F097FE0020C9F8800BB8F84006EE
:106F6000012854D1B9F88A0ADFF8F468DFF8F44848
:106F7000002840D150E000BFB9F88A0A00284BD061
:106F8000FEF762FDDFF8E0080088442810D0D9F849
:106F9000F00E00F44170B0F5417F09D1D9F8FC0E34
:106FA000C0F3002000281CBFB9F8840A002804D1CF
:106FB00000F06AFC0120A9F8820A0822DFF8AC0878
:106FC000D9F8281D806B1EF06BFE0015206021682B
:106FD000B8F8BA0588420EDA0020A9F88A0A032018
:106FE000A9F8940A306840F00200306015F072F998
:106FF0000120A9F8820AD9F8C00C0F49002848BF1F
:107000004042884203DBB9F8820A0028B4D0B9F8BC
:107010008A0A08B100F038FC0020A8F840060021D8
:107020004FF4487003F02EFE01B0BDE8F04F03F0BE
:10703000A2BE01B0BDE8F08F5C8F0200CCCCCC00CA
:10704000B0AAAA003333B300A08601002DE9F041B5
:10705000DFF81848DFF81858E06BC5F8940B216C7E
:10706000C5F8981BB5F88A1A0A000CD1DFF8086831
:10707000002130461FF03DFA3046BDE8F0410022C5
:1070800080211FF041BA012940F0A080B5F8641AB0
:1070900041BBDFF8E8171EF0ABFEC5F878044FF4EB
:1070A0008F60D5F8AC1428448847D5F87C04DFF805
:1070B000D0170818D5F87814884204DAB5F87E0A93
:1070C000401CA5F87E0A42F22832D5F8A404C11764
:1070D000A2FB006702FB0177360E46EA0726901BEB
:1070E000A5F8680AB5F8680AB5F86C1ADFF8886779
:1070F000401AA5F86A0A3087B5F8660A4000B087DA
:10710000B5F8660A4000B086B5F8640A012840F078
:10711000A183D5F88C02C5F890024FF43571D5F8EB
:10712000D402C5F8D8024FF44772D5F81C03C5F84D
:10713000200329444FF4237028442A445FF00403B9
:1071400050F8046C066051F8046C0E6052F8046C40
:10715000166050F8086C40F8046C51F8086C41F85F
:10716000046C52F8086C42F8046C50F80C6C40F84F
:10717000086C51F80C6C41F8086C52F80C6C42F831
:10718000086C50F8106C40F80C6C103851F8106C0A
:1071900041F80C6C103952F8106C42F80C6C103A33
:1071A0005B1ECDD1A06BDFF8DC16C5F84C02B5F83C
:1071B000680AC0031EF0D4FDC0F18070C5F89402C7
:1071C000D5F8940BC5F8DC02BDE8F081022940F047
:1071D0006181B5F8640AB8B9D5F86C0CD5F8AC146F
:1071E000C5F878044FF48F6028448847D5F87C04AC
:1071F000DFF88C160818D5F87814884204DAB5F848
:107200007E0A401CA5F87E0AD5F8A01BD5F8842B71
:10721000D5F8A404C5F89C0C5118DFF81C2E914237
:10722000A8BF01F14041B1F1005FCCBF01230023B1
:10723000A5F8703AC5F8A01BDFF8003E5918914236
:10724000A8BF01F14041C5F8A81B8911C5F8A41BCE
:10725000E16BC5F8A01C226CC5F82415C5F8A42C58
:10726000C5F82825616CC5F82C15A16B1EF078FDBA
:10727000DFF8CC1D1EF0BCFDC5F8A8070020C5F83E
:10728000AC07D5F8A40BD5F8B017C5F8A40705F2DC
:107290009C708847D5F89C07D5F81018C5F8FC07EE
:1072A000D5F8A007C5F8000805F2FC708847D5F8A6
:1072B0000408D5F844158012A5F81E05D5F808086D
:1072C0008012A5F82005D5F80C088012A5F8220533
:1072D0004FF4A36028448847B5F8700A01001FD115
:1072E000B5F87C0A012840F0FC81B5F8720A401C10
:1072F000A5F8720A80B205EB40012269A1F8002CC2
:10730000821E4E2A80F0ED81B1F8001CB5F8742A77
:107310008A42C0F0E681A5F8741AA5F8760AE0E181
:10732000012840F09782B5F8641AB5F87C0A012963
:107330000ED101000CD10120A5F87C0A0020A5F88F
:10734000760AA5F8720A40F6FF70A5F8740A14E0F0
:10735000012812D1B5F8760A01000ED00021A5F857
:10736000721A40F6FF71A5F8741AB5F8801A401A1F
:10737000A5F86E0A0020A5F8760AD5F8A00CD5F875
:10738000801C8842B8BFC5F8800CB5F86E0A0100B1
:107390000CD0D5F8841B102280021EF081FCC5F8A9
:1073A000B00BC5F8AC0B0020A5F86E0AD5F8780C28
:1073B000012804DBC5F8740C0020C5F8780CD5F85A
:1073C000740CD5F87C1C411A4FF400001EF010FD1F
:1073D000B5F8641AC5F86C0C012904BFB5F87A1A1F
:1073E000012940F03782D5F88C12C5F890124FF47D
:1073F0003572D5F8D412C5F8D8124FF44773D5F8C2
:107400001C13C5F820132A444FF4237129442B443C
:107410005FF0040451F8046C0E6052F8046C1660BE
:1074200053F8046C1E6051F8086C41F8046C52F873
:10743000086C42F8046C53F8086C43F8046C51F87B
:107440000C6C41F8086C52F80C6C42F8086C53F85C
:107450000C6C43F8086C51F8106C41F80C6C103946
:1074600052F8106C42F80C6C103A53F8106C43F858
:107470000C6C103B641ECDD10021A5F8781AC5F81C
:107480009402D5F8AC1BD5F89C0CC5F84C12C5F885
:10749000DC02DCE1032902BFDFF8D803B0F84006C4
:1074A000012840F0D781D5F8F40CD5F89817C5F825
:1074B0008407D5F8F80CC5F88807D5F87807C5F81B
:1074C0008C0705F284708847D5F8F40CD5F89C1722
:1074D000C5F8E409D5F8F80CC5F8E809D5F8A0070F
:1074E0001FF09CFBC5F8EC091FF05AFB0646D5F8C7
:1074F000EC091FF015FB0746D5F8E40939461EF0E4
:1075000077FC8046D5F8E80931461EF071FC40440E
:10751000C5F8F0093946D5F8E8091EF069FC0746B8
:10752000D5F8E40931461EF063FC381AC5F8F409B1
:10753000D5F89007D5F84819C5F83409D5F8940757
:10754000C5F84C0905F634108847D5F8601905F6DA
:107550004C108847D5F84409D5F8C817C5F8C007B6
:10756000D5F85C09C5F8C407D5F87807C5F8BC0795
:1075700005F2B4708847D5F8B407D5F8F817C5F800
:10758000F007D5F8B807C5F8F40705F2E4708847A6
:10759000D5F8E407C5F8A00CC5F82405D5F8EC0724
:1075A000D5F8E817C5F82C05C5F8A41CC5F82815AA
:1075B000D5F8800BD5F86C15C5F84C0505F24C5084
:1075C0008847D5F85805C5F8C00CC5F868074FF4CA
:1075D000ED60D5F8801728448847D5F8580500286D
:1075E00048BF40424FF080711EF002FCC5F8A8076A
:1075F0000020C5F8AC07D5F87807D5F8B017C5F85E
:10760000A40705F29C708847D5F8D40A00F1807071
:10761000E064D5F89C171EF0EBFBC5F8FC07D5F825
:10762000A017E06C1EF0E4FBC5F8000805F2FC7042
:10763000D5F810188847D5F80408D5F844158012F5
:10764000A5F81E05D5F808088012A5F82005D5F87C
:107650000C088012A5F822054FF4A360284488473F
:10766000D5F8806BA16BDFF85C0D002E48BF764229
:107670001EF0BEFB31461EF0BBFBC5F89C0CD5F8D6
:10768000780700F58000B0F1807FC8BF00F17F402F
:10769000C5F8A40BB0F5000FCCBF01200020A5F861
:1076A000700AB5F8700A010032D1B5F87C0A0128D9
:1076B00017D1B5F8720A401CA5F8720A80B205EB22
:1076C00040012269A1F8002C821E622A3EBFB1F857
:1076D000001CB5F8743A99423CBFA5F8741AA5F895
:1076E000760A0120A5F87A0AD5F8781CD5F8A00CFE
:1076F0008142B8BFC5F8780CD5F8800C002840F15D
:10770000A980C5F87C0C0020C5F8800CBDE8F0818C
:10771000012840F09F80B5F8641AB5F87C0A012969
:107720000ED101000CD10120A5F87C0A0020A5F89B
:10773000760AA5F8720A40F6FF70A5F8740A14E0FC
:10774000012812D1B5F8760A01000ED00021A5F863
:10775000721A40F6FF71A5F8741AB5F8801A401A2B
:10776000A5F86E0A0020A5F8760AD5F8A00CD5F881
:10777000801C8842B8BFC5F8800CB5F86E0A0100BD
:107780000CD0D5F8841B102280021EF089FAC5F8AF
:10779000B00BC5F8AC0B0020A5F86E0AD5F8780C34
:1077A000012804DBC5F8740C0020C5F8780CD5F866
:1077B000740CD5F87C1C411A4FF400001EF018FB25
:1077C000C5F86C0CB5F8640A012804BFB5F87A0A4C
:1077D00001283FD1D5F88C02C5F890024FF43571DD
:1077E000D5F8D402C5F8D80229444FF423702844B0
:1077F0005FF0040250F8043C036051F8043C0B6055
:1078000050F8083C40F8043C51F8083C41F8043C6E
:1078100050F80C3C40F8083C51F80C3C41F8083C4E
:1078200050F8103C40F80C3C103851F8103C41F82E
:107830000C3C1039521EDDD10020A5F8780AD5F88D
:10784000AC0BC5F84C02D5F8740CC5F894020020B6
:10785000A5F87A0ABDE8F0810010270000A0860193
:10786000905E00209812002022210020145D00204C
:107870000000002038430020002C0140E7FB690194
:10788000A470FDFF000094112DE9F043DFF8484D8E
:10789000DFF8487DD4F8B40FC0F30325C0F3031913
:1078A00081B0002138461EF024FE00228021384697
:1078B0001EF02AFEDFF8280DDFF8287D01884BF640
:1078C000FF72114001804FF6FB7138880840388004
:1078D000B4F8860A012812D15FF00000A4F8860AE5
:1078E000A4F88A0A4FF49678D4F89C0EC0F30010DE
:1078F00010B102200CF034F9B8F10108F4D1D4F839
:10790000980EDFF8E48CC0F3400616B1B8F8A00179
:1079100060B1D4F8140FC0F3001010B9B8F8A0018A
:1079200020B9D4F8F00EC0F3002088B9D4F8B40F11
:1079300040F20511884204D0032D08BFB9F1050FAC
:1079400006D1B8F8E20000F57F40FF30C4F8C80E59
:1079500040F20911D4F8B40F88421CBF40F205214F
:1079600088422DD1B8F8FE0750BBC4F8CC01C4F84A
:10797000D001C4F8D401C4F8D801C4F8DC01C4F8BB
:10798000E001C4F8E401C4F8E801C4F8EC01C4F86B
:107990001C02C4F82002C4F82402C4F82C02C4F863
:1079A00028024FF09741D4F87C0B1EF0C1FA1EF06C
:1079B0002BFBC4F830020020C4F83402C4F83802AB
:1079C000D4F89C0EC0F3001000281EBFD4F8B80EE7
:1079D000D4F89C1F81421FD0B8F8CA140A0014D0F2
:1079E000012907D0022902BFD4F8981FC1F3003142
:1079F00000290AD1B8F8D410022911BF0329D4F8FC
:107A0000981F42F62102114206D0B0F57A7F38BFA6
:107A10004FF47A70C4F89C0F002E03BFD4F8F00E18
:107A200000F44070B0F5407F19F038FE94F89C0ED9
:107A300000F00800C4F89C0ED4F8A00EC0F380013A
:107A400041BBD4F8981E21F02001C4F8981EC1F360
:107A5000801161B1D4F8981FD4F8982E41F40061D8
:107A6000C4F8981F022161F38712C4F8982E20F001
:107A7000C000C4F8A00E94F8980EC00703D4DFF835
:107A80006C1B03200880D4F8140F20F48150C4F834
:107A9000140F05E0D4F8980E40F00400C4F8980ED6
:107AA0001CF016FF0020C4F8A40FC4F8A80FC4F8F7
:107AB000AC0FD4F8980E10F0220F05D0D4F8981F10
:107AC00021F40061C4F8981FD4F8A01EDFF8202B21
:107AD00021F02801C4F8A01EDFF8181B0840D4F8D4
:107AE000DC1EC4F8E01EC4F8980E0021C4F8B81ECD
:107AF000D4F8141F1140C4F8141F0021C4F80C1F3F
:107B0000C4F8BC1FC4F8B81FDFF8EC2A116821F0D4
:107B100010011160DFF8E41A0B880C2B08BFB4F8D1
:107B2000983A02D00A2BA8BF0023A4F89A3AB4F8D6
:107B30009C3A0A2B0ADA012B0B8007D1022313602F
:107B4000DFF8082E136843F004031360B4F89A2A90
:107B50000A2A03DB0022A4F89C2A0A80C0F38031A1
:107B600019B120F48040C4F8980E0020C4F8940D98
:107B7000C4F84C0DC4F8580DC4F85C0DC4F8640D7D
:107B8000C4F86C0D4FF08070C4F8D80C0020C4F815
:107B9000240D4FF0A060C4F8D00C0020C4F8140DE0
:107BA000C4F81C0DC4F8180DC4F8200DC4F8040D59
:107BB000C4F8B80CC4F8BC0CC4F8B00CC4F8B40CCD
:107BC000C4F8FC0CC4F8AC0CC4F8A80CC4F8080D3C
:107BD000C4F8100DC4F8000DC4F82C04C4F828042F
:107BE000C4F83404C4F85403C4F84803C4F8440384
:107BF000C4F86C04C4F86404C4F86004C4F8FC035A
:107C0000C4F8F403C4F8F003C4F88C03C4F8840384
:107C1000C4F88003C4F8C403C4F8BC03C4F8B803B0
:107C2000C4F86C0BC4F80C0DC4F88407C4F88807BA
:107C3000C4F88C0704F28470D4F8981788470020A1
:107C4000C4F8A807C4F8AC07C4F8A40704F29C70F1
:107C5000D4F8B01788470020E0656063A063E06453
:107C600020656065A065C4F89C00C4F8A400C4F851
:107C7000B400C4F8B800C4F8BC00C4F8B000E067B1
:107C8000C4F88000E0662067E0632064A060E060E4
:107C9000A061E06120626062A067C4F8E40CC4F8EF
:107CA000E80CC4F8EC0CC4F8F00CC4F8B80EC4F836
:107CB000C00CC4F85805C4F868074FF4ED60D4F858
:107CC000801720448847002020616061C4F8840048
:107CD000C4F88800C4F88C00C4F81408C4F820085C
:107CE000C4F82408C4F82C08C4F83808C4F83C08C0
:107CF000C4F84408C4F85008C4F85408C4F85C0830
:107D0000C4F86808C4F86C08C4F87408C4F880089B
:107D1000C4F88408C4F88C08C4F89808C4F89C080F
:107D2000C4F8A408C4F8B008C4F8B408C4F8BC087F
:107D3000C4F8C808C4F8CC08C4F8D408C4F8E008EB
:107D4000C4F8E408C4F8EC08C4F8F808C4F8FC085F
:107D5000C4F80409C4F81009C4F81409C4F81C09CB
:107D6000C4F82809C4F82C09C4F8C007C4F8C4072B
:107D7000C4F8BC0704F2B470D4F8C81788470020D0
:107D8000C4F8D807C4F8DC07C4F8D40704F2CC70F0
:107D9000D4F8E01788470020C4F8F007C4F8F407C7
:107DA00004F2E470D4F8F81788470020C4F8A80556
:107DB000C4F8BC05C4F8B805C4F8C405C4F8D805AF
:107DC000C4F8D405C4F8E005C4F8F405C4F8F00517
:107DD000C4F8FC05C4F81006C4F80C06C4F818066C
:107DE000C4F82C06C4F82806C4F83406C4F84806BB
:107DF000C4F84406C4F85006C4F86406C4F8600623
:107E0000C4F86C06C4F88006C4F87C06C4F888067A
:107E1000C4F89C06C4F89806C4F8A406C4F8B806CA
:107E2000C4F8B406C4F8C006C4F8D406C4F8D00632
:107E3000C4F8DC06C4F8F006C4F8EC06C4F8F8068A
:107E4000C4F80C07C4F80807C4F81407C4F82807D6
:107E5000C4F82407C4F8180EC4F8200EC4F8240E81
:107E6000C4F8280EC4F8300EC4F8340EC4F8380E26
:107E7000C4F83C0EC4F8400EC4F8440EC4F8480ED2
:107E8000C4F84C0EC4F8500EC4F8540EC4F8580E82
:107E9000C4F85C0EC4F8640EC4F8680EC4F86C0E26
:107EA000C4F8700EC4F8740EC4F8780EC4F87C0ED2
:107EB000C4F8800EC4F8A80DC4F8AC0DC4F8B00D19
:107EC000C4F8000EC4F8040EC4F8080EC4F80C0E72
:107ED000C4F8D00DC4F8E00DC4F8B40DC4F8B80D62
:107EE000C4F8BC0DC4F8C00DC4F8C40DC4F8E40D4A
:107EF000C4F8E80DC4F8EC0DC4F8F00DC4F8F80DA2
:107F0000C4F8F40DC4F8140EC4F87005C4F8840560
:107F1000C4F88005C4F88C05C4F8A005C4F89C0515
:107F2000C4F8380FC4F83C0FC4F8600FC4F82C0F25
:107F3000C4F8300FC4F8340FC4F8640FC4F8680FE5
:107F4000C4F86C0FC4F8700FC4F8740FC4F8780F3D
:107F5000C4F87C0FC4F8800FC4F8840FC4F8400F35
:107F6000C4F8440FC4F8480FC4F84C0FC4F8500FBD
:107F7000C4F8540FC4F8580FC4F85C0FD4F8280F95
:107F800020F01E00C4F8280F0020C4F8900FC4F899
:107F90009000C4F8980DC4F8600BC4F8380BC4F80E
:107FA000440BC4F8480BC4F84C0BC4F8340BC4F8A9
:107FB000FC09C4F80C0AC4F8080AC4F8140AC4F886
:107FC000240AC4F8200AC4F8AC09C4F8BC09C4F8EF
:107FD000C009C4F8B809C4F8C809C4F8D809C4F875
:107FE000DC09C4F8D409C4F8EC0AC4F89404C4F851
:107FF0009804C4F89C04C4F8A004C4F87C040120CC
:10800000A4F8840A0020C4F8000BC4F8FC0A1CF091
:108010004EFF1EF06FFF0020A4F8A80AF9F795FDA7
:1080200038884FF6BF710840388001B00020A4F8AE
:108030005E0ABDE8F083000001000040A5B8AA2A4E
:108040006B9A270170B5DFF8A055DFF88C45B5F8BD
:10805000F400012804BFD4F8DC0E012800F04781A9
:10806000B5F8D400042818BF052800F0408100218D
:10807000C4F86C1BC4F8781BC4F8701BC4F8741BDC
:10808000DFF878150A880A2AA8BF0022A4F89C2ADB
:10809000B4F89A2A0A2A0CDA012A0DD1DFF85865B9
:1080A00002233360DFF8A4381E6846F004061E6021
:1080B00002E00022A4F89A2A0A804FF6FF36DFF881
:1080C000501CC96CD4F8BC2EC4F8F81FC4F8C02EDC
:1080D000D4F8DC1EC4F8E01ED4F8D41EC4F8B01ED8
:1080E000D4F8D81EC4F8B41EDFF8F8140B88334057
:1080F0000B800021C4F8181ED4F8F41ED4F8983E62
:10810000C1F3C0010029D4F8981F0CBF41F40051FD
:1081100021F40051C4F8981F5E0AD4F8141F46EAEF
:1081200013230B4343EA510343EAD11343EA1123D8
:10813000D4F8986F5B0963F3451621F00201022819
:10814000C4F8986FC4F8141F2ADBB5F8DA30D4F8F5
:10815000D06EB34224D2B5F8DC300BB3022818BF7E
:10816000032812D1B5F8CA04012808D0022802BF9A
:10817000D4F8980F43F62003184206D110E0D4F843
:10818000980F42F6200318420AD00020C4F8B00F1E
:1081900094F8280FC0075CBF41F00200C4F8140F28
:1081A000D4F80C0F40F04000C4F80C0FB5F854069A
:1081B000C103D0031DF0D4FDD4F8E01E012908BF8F
:1081C0004042C4F8A00DC4F84C05D4F8B00EA4F891
:1081D0006405D4F8B40EA4F86605B5F8D40001001F
:1081E0001CBF012806282AD0B5F8B004012818BF02
:1081F00003280DD1D4F8982FC2F3401212B9B5F864
:10820000CA242AB9D4F80C2F42F01002C4F80C2F5B
:10821000002818BF022812D1D4F8140FC0F3400070
:1082200038B1B5F85406C103B5F8DA00C0031DF043
:1082300097FDD4F8E01E012902D1404200E0002061
:10824000C4F858050020C4F8380BC4F8440BC4F82F
:10825000480BC4F84C0B1CF00DF8D4F85805DFF8A7
:10826000601CC4F8C00CD4F82C0D81FB0001000E7A
:1082700040EA0120C4F8DC0CB5F8CA04012819D082
:10828000022802BFD4F8980F43F62101084217D004
:108290004FF4A360D4F8481520448847D4F89C0EC6
:1082A00040F01000C4F89C0ECD484188C1F30E0187
:1082B000418070BDD4F8980F42F621010842E7D101
:1082C000B4F8860A002802BFD4F80C0FC0F30010DF
:1082D0000028DDD1B5F8D4000228D9DBB4F8620A51
:1082E000B0F57A7FD4DA0120A4F8AA0ADCE7D4F842
:1082F000A00E20F08800C4F8A00E70BDF0B5DFF825
:10830000106AB54DB06BD5F8281D81B008221DF05C
:10831000C7FCDFF8B04B001520600522F16B084662
:108320001DF0BEFC0746306C052201461DF0B8FC6E
:10833000C719706C052201461DF0B2FCDFF8886B8E
:10834000C01930604FF4C00120F046FA30601EF0D2
:10835000B1FB3060C000C5F80C0BDFF8701BDFF814
:10836000707B1DF045FDC5F8080B0B2230684FF0FF
:1083700048611DF095FC3060D5F87011DFF8540BA2
:108380001DF036FD3168BB680822C91A1DF088FC53
:10839000B9684018B8600322D5F8381D1DF080FC7C
:1083A00078600722D5F8381DB8681DF079FC0014F4
:1083B000F8600A21B0FBF1F0388001B020687880C5
:1083C000F0BD00005839B40070B5834D864CD5F827
:1083D0009C0EC0F30010002840F0A080B4F8D40038
:1083E000022806DBB4F85416B4F8EC001DF0B8FC13
:1083F00001E04FF08070C5F8780D3220B4F85416C3
:10840000DFF8D46A1DF0ACFCC5F87C0DB4F814019B
:108410000106DFF8C80A1DF0EBFCC5F8740D4FF03B
:10842000C841B4F81A0100061DF09AFCC5F8800D89
:108430004FF0C841B4F81E0100061DF091FCC5F8CC
:10844000840D4FF0C841B4F8220100061DF088FCED
:10845000C5F8880D4FF0C841B4F8260100061DF09C
:108460007FFCC5F88C0D4FF0C841B4F82A01000616
:108470001DF076FC30614FF0C841B4F82E010006C3
:108480001DF06EFC70614FF0C841B4F83001000679
:108490001DF066FC01464FF080701DF0A9FCC5F888
:1084A000900DB4F85406C103B4F81801C0031DF0D0
:1084B00057FCB061B4F85406C103B4F81C01C00302
:1084C0001DF04EFCF061B4F85406C103B4F820016D
:1084D000C0031DF045FC3062B4F85406C103B4F883
:1084E0002401C0031DF03CFC7062B4F85406C103C3
:1084F000B4F82801C0031DF033FCB062B4F8540690
:10850000C103B4F82C01C0031DF02AFCF062B4F8DA
:108510005416B4F8EC001DF023FC3063B4F8D4001A
:10852000022818BF03280DD1B4F830014FF0C8411C
:1085300000061DF015FC01464FF080701DF058FC40
:10854000C5F8900DB4F8D400062808D1D5F8FC077A
:1085500001461DF04DFC0646D5F8000807E0D5F8A9
:10856000A80701461DF044FC0646D5F8AC070146B5
:108570001DF03EFC80191EF029F80646DFF8900732
:10858000DFF85C19806B1DF0EBFB31461DF030FC11
:10859000DFF84469011331600822B4F84416490534
:1085A0001DF07EFBC012B063B26BF06B411C706BB0
:1085B000F16310186429706308D34FF4C8311DF0BB
:1085C00045FDC5F8B40D00207063F063D5F8B40D17
:1085D0008012A5F8920A70BD00000020002C014016
:1085E0005C5C0020985C0020384300204C20002078
:1085F000BDDFFFFFEDEFFFFF44210020242100201D
:10860000F0B5DFF8E048DFF8E058B4F81A010100EF
:1086100081B01CD0B4F81821DFF8D018C00322B9FB
:108620000B221DF03DFB064612E00B221DF038FB2D
:108630000646B4F81811D5F8B80E884208D21DF0D5
:108640008FFB014630461DF0D3FB064600E00026B6
:10865000B4F81211D5F8C00C0A0024D10028D5F8BE
:108660007C2D48BF4042824207DB0146D5F8740D9D
:108670001DF0BEFBD5F87C1D99E0D5F8781D884229
:1086800080F20981891A801A1DF06AFBDFF84878A8
:10869000F860D5F8741DC1F180711DF0A9FBD5F803
:1086A000741D0818F9E0012973D1B4F816110629D0
:1086B00010D10028D5F87C1D48BF4042814212DA13
:1086C000D5F8781D884280F2E6801DF049FB1DF048
:1086D0007DFF1CE005292FD10028D5F87C1D48BF5F
:1086E000404281420CDB0146D5F8740D1DF080FB41
:1086F000D5F87C1D1DF034FBDFF8DC174860CCE0BA
:10870000D5F8781D884280F2C6801DF029FB074607
:10871000D5F8C00CD5F8781D002848BF40421DF0A0
:108720001FFB39461DF064FBDFF8AC77796888429F
:10873000B8BF0846B860B0E00028D5F8781D48BF3B
:10874000404288420CDA1DF00BFB071210224FF456
:10875000481138461DF0A4FA00140004C00B02E0D2
:108760004FF480376420B4F81611012908BFDFF8F0
:1087700080170AD0022908BFDFF8781705D003292F
:108780000CBFDFF87417DFF87417085A381A0002A4
:1087900083E0DFF84477B969002848BF404281424E
:1087A00008DB0146D5F8800D1DF022FBB9691DF0EC
:1087B000D7FA72E0FA69824210DB411AD5F8840DCB
:1087C000D5F8802D801A1DF013FBF969BA69891A52
:1087D0001DF0C6FAD5F8801D08185EE0396A81429E
:1087E00010DB811AD5F8880DD5F8842D801A1DF07C
:1087F000FFFA396AFA69891A1DF0B2FAD5F8841DB0
:1088000008184AE07A6A824210DB411AD5F88C0DCA
:10881000D5F8882D801A1DF0EBFA796A3A6A891A20
:108820001DF09EFAD5F8881D081836E0B96A814215
:108830000FDB811A3869D5F88C2D801A1DF0D8FA13
:10884000B96A7A6A891A1DF08BFAD5F88C1D081856
:1088500023E0FA6A82420DDB411A78693A69801A8C
:108860001DF0C6FAF96ABA6A891A1DF079FA3969EF
:10887000081812E0396B81420DDB811A7869C0F16A
:1088800080701DF0B5FA396BFA6A891A1DF068FA22
:108890007969081801E04FF08070B042B4F83411E3
:1088A000B8BF3046012941D1B4F8D41002293DDBCC
:1088B000C5F8440EDFF848060168B4F844061DF018
:1088C0004FFADFF840161DF093FAC5F8680ED5F898
:1088D000441E1DF08DFAD5F8441E401AC5F8640EEA
:1088E000C5F850064FF4CA60D5F868162844884782
:1088F000D5F86406D5F88416C5F86C0605F26C60E8
:108900008847D5F8440ED5F880160818D5F8901D7C
:1089100048BF002081FB0001000E40EA0120B0F1B9
:10892000807F11DD4FF0807001B0F0BD4FF080719D
:10893000C5F8681E0021C5F8641ED5F8901D81FB9E
:108940000001000E40EA012001B0F0BD48210020E6
:10895000DFF89005B0F8D41001B9704710B5DFF812
:108960008845D4F8981EC1F3001100295AD1D4F8D3
:10897000981FC1F3401119B9B0F8CA14002951D198
:10898000D4F8B81FB0F8B824914210D2D4F80C2F04
:10899000012060F30512D4F8EC0EC4F80C2FC0F3DC
:1089A000402000283ED0481CC4F8B80F10BDD4F8B1
:1089B0000C1FC1F30011C9B1D4F8141FC1F3400159
:1089C00041B1B0F85416B0F8DA00C903C0031DF085
:1089D000C7F900E00020C4F85805D4F8E00E0128DB
:1089E00004D1D4F858054042C4F85805D4F80C0F07
:1089F00020F01000C4F80C0F0020C4F8600DC4F87B
:108A0000680DC4F89C04C4F89804C4F89404C4F82D
:108A1000A004C4F8A404C4F87804C4F8580D0120D4
:108A2000C4F8640D10BD30B5DFF8B854DFF8B844B1
:108A3000B5F8BC04012881B042D1F8F753FFD4F84F
:108A4000EC0A022840F0A280D4F8BC0FB5F8BA14A2
:108A5000884221D294F8981EC9071DD494F8141F97
:108A600011F0300F18D1D4F80C1FD4F8D02E41F0EB
:108A70003001C4F80C1F0021C4F8B81FB5F8B214B7
:108A80008A4228BFC4F8B81ED4F8EC1EC1F34021B6
:108A900000297BD0401C77E0D4F80C0F20F01000A8
:108AA000C4F80C0F0020C4F89C04C4F89804C4F85F
:108AB0009404C4F8A004C4F8A404C4F8780444E0FE
:108AC000D4F8981EC1F30010002845D0B5F8B224A0
:108AD000D4F8B80E82423FD3D4F8BC0FB5F8BA34FC
:108AE00098421FD2C9071DD494F8141F11F0300FFB
:108AF00018D1D4F8101F21F4C071C4F8101FD4F895
:108B00000C1F41F03001C4F80C1FD4F8D01E914264
:108B100028BFC4F8B82ED4F8EC1EC1F34021A9B385
:108B2000401C31E0D4F8100F40F08000C4F8100F62
:108B3000C0F3002050B30020A4F8A20AD4F80C0F10
:108B400020F01000C4F80C0F0020C4F8BC0F01B0D6
:108B5000BDE83040FEF798BEC1F3C00050B1B5F893
:108B6000D400022806DAD4F80C0FC0F3001008B1C4
:108B7000FEF78AFE0020A4F8A20AD4F80C0F20F019
:108B80003000C4F80C0F0020C4F8BC0F01B030BD99
:108B900010B5D54CD4F8980EC0F3001048B1D148A8
:108BA000D4F8B81EB0F8B204884223D3BDE8104010
:108BB00039E7D4F8980FC0F3401018B9C948B0F895
:108BC000CA04B8B9D4F80C0FC0F3401058B1C54866
:108BD000B0F8D40038B9FEF757FED4F80C0F20F0E7
:108BE0001000C4F80C0FFFF7B3FE0020C4F8EC0A25
:108BF000C4F8BC0F10BD70B5BA4CB4F8BC04012861
:108C000025D0B4F8B404652807DB6420A4F8B404C4
:108C1000642140F25A2002F035F8B4F8B604652811
:108C200007DB6420A4F8B604642140F25B2002F064
:108C300029F8B4F8B204B0F5FA7F08DD4FF4FA7001
:108C4000A4F8B204014640F2592002F01BF8B4F82F
:108C500046068102B4F8CC0080021DF081F8064679
:108C6000B4F8B004012818BF03280ED1B4F8B40436
:108C7000DFF8501D162280021DF012F80146304622
:108C80001DF0B6F8B4F8B81403E0B4F85816DFF8DD
:108C9000380D954DC5F8F40AC5F8D81F1622B4F85A
:108CA000B604DFF8201D80021CF0FAFF01463046B2
:108CB0001DF09EF8C5F8F80A914800684105B4F81F
:108CC000920640051DF04CF84FF000711DF090F831
:108CD000DFF8881D0860D5F89C0EC0F30010B0B115
:108CE000B5F8860A98B9B4F8B004012804BFBDE805
:108CF0007040FFF72DBE022804BFBDE87040FFF7AB
:108D000092BE032804BFBDE87040FFF741BF70BDAD
:108D1000145D00202DE9F041DFF8440DDFF8446DCB
:108D2000406B714CDFF8BC81C104706988B00D22C2
:108D30001CF0B6FFD4F8281D08221CF0B1FF3188C2
:108D40003269718000153080891830884018002100
:108D500031614008B8F8C6148842C0F29A80B8F869
:108D6000D420022A04DAB8F8BE24022A00F0918046
:108D7000B8F8DC24012A27D1451A4FF0C86128052C
:108D80001CF0EEFF002D44BF0020C4F8BC03C4F863
:108D90009C030020C4F898034FF46670D4F8CC13F9
:108DA00020448847D4F8C40308224FF4C8011CF0BB
:108DB00077FF00140B2838BF0A20F0604FF461677A
:108DC00078436421B0FBF1F5B8F8DC04D0B9B8F809
:108DD000C80401460B290FDB332904DADFF8441DF0
:108DE000B1FBF0F70AE05B2906DADFF8382DC1F1B4
:108DF0006401B2FBF1F701E048F6A0477843642133
:108E0000B0FBF1F5BD4228BF7D1EDFF81C6D781E5A
:108E1000B0853587D4F8141FC1F3C02100294BD188
:108E2000ADF8040009210020ADF80010ADF80600EF
:108E300020210120ADF802108DF808006946304667
:108E40001DF02CFA6020ADF80C00ADF81250012096
:108E5000ADF80E0003A90220ADF814000020ADF813
:108E6000180030461DF0A5FA082130461DF085FB9C
:108E7000012130461DF070FB012130461DF02FFB13
:108E8000D4F8140F40F40060C4F8140F08B0BDE823
:108E9000F081DFF8946C0220B08500203087D4F890
:108EA000140F20F40060C4F8140F0020C4F8C403A9
:108EB000C4F8BC03C4F8B80308B0BDE8F0810000F2
:108EC00047E1FA0098120020DC630020E7FB69010B
:108ED0002861002033333300105F0020AE470100CB
:108EE000B6F3BD0138430020000000200AD7A300DC
:108EF000BCCE020824CF02088CCF0208F4CF0208AF
:108F000094120020900F6A014FF6FE712DE9F04394
:108F1000DFF8187CDFF8608D3888DFF8605DDFF8F7
:108F2000609D0840388081B0D8F8B40FC0F30321A9
:108F3000A962C0F3031100F00F00E9622863B9F8D9
:108F4000DE40B9F8E2071CF065FF064620461CF03B
:108F500061FF014630461CF06DFFC8F87C0B41F202
:108F6000883120461CF0FCFE6861B9F8F417D8F887
:108F7000200F01290CBF20F4006040F40060C8F805
:108F8000200FB9F8960109281CBFB9F898110529D6
:108F900040F0D283D8F8B41F40F2091291421CBFAE
:108FA00040F2052291422ED0A96A032905D1E96A2F
:108FB00009291CBF296B052925D0B9F89E11022962
:108FC00010D1092804D1D8F8F41EC1F34011D1B949
:108FD000B9F8981105291AD1D8F8F41EC1F3401137
:108FE00000290FE0032912D1092808D1D8F8F41E6E
:108FF000C1F3401119B1398841F001013980B9F844
:109000009811052903D1398841F001013980B9F857
:10901000D4176A882B6D01291CBFB9F8D277012FAC
:1090200054D1B9F8207340F2991404FB07FC64246E
:10903000BCFBF4FCB9F8CC4504FB0CFC6424BCFB81
:10904000F4FCDFF8404C246864453DD20A2F3BDB3A
:10905000D8F8EC7EC7F3400707B1521C92B2022A3F
:1090600035DBB9F8CA75002287B3012F0AD1DFF8C2
:10907000187C3C68C4F38036CEB944F480440123A4
:109080003C6016E0022F05D1DFF8004C6A62012334
:1090900022800EE0032F04D1B9F8E0706F62012343
:1090A00007E0042F03D1AF6D6F62012301E0012BB4
:1090B0000DD1092804BF6F6A2F66B9F89871052F82
:1090C00005D16F6A6F6602E06B6AAB6500232B65A2
:1090D0006A800229AA886B6D1CBFB9F8D277022F6B
:1090E00054D1B9F82C7340F2991404FB07FC6424A2
:1090F000BCFBF4FCB9F8CC4504FB0CFC6424BCFBC1
:10910000F4FCDFF88C4B246864453DD20A2F3BDB2E
:10911000D8F8EC7EC7F3400707B1521C92B2022A7E
:1091200035DBB9F8CA75002287B3012F0AD1DFF801
:10913000587B3C68C4F38036CEB944F480440123A4
:109140003C6016E0022F05D1DFF8404B6A62012334
:1091500022800EE0032F04D1B9F8E0706F62012382
:1091600007E0042F03D1AF6D6F62012301E0012BF3
:109170000DD1092804BF686A2866B9F89801052846
:1091800005D1686A686602E0686AA86500236B65B5
:10919000AA80286D184340F0D282D8F8EC0EC0F3B4
:1091A0004000002800F04B8101292ED1B9F820039E
:1091B0004FF07A5100051CF0D3FD68634FF07A51EF
:1091C000B9F8240300051CF0CBFDA8630A21B9F807
:1091D00028031CF0C5FD0746DFF8A80A006840F622
:1091E000FF711CF0BDFD39461CF002FEA96B6A6BD5
:1091F00028648A4230D0904233DB8142B8BF4FF0BE
:10920000807042DB891A801A3DE0022933D1B9F817
:109210002C034FF07A5100051CF0A2FD68634FF05B
:109220007A51B9F8300300051CF09AFDA8630A21B1
:10923000B9F834031CF094FD0746DFF8540A0068BF
:1092400040F6FF711CF08CFD39461CF0D1FDA96B76
:109250006A6B28648A4202D14FF4000015E0904204
:1092600001DA002011E08142B8BF4FF080700CDBC2
:10927000891A801A07E0032918BF042906D1E86D6E
:109280004FF07A51C0031CF06BFDE863E86B0822D5
:109290004FF07A711CF004FD0014E8642880D8F8BF
:1092A000100FC0F3C00028B9B9F844084FF07A5144
:1092B0000005A8E0B9F8D207010005D1B9F8D80730
:1092C0004FF07A5100059EE001282DD1D8F8200FEB
:1092D000C0F3C020002840F09980B9F820034FF077
:1092E0007A5100051CF03CFD68634FF07A51B9F8E3
:1092F000240300051CF034FDA863DFF8981CDFF898
:109300008409006880041CF02BFDA96B6A6BA864BB
:109310008A425DD0904260DB8142B8BF4FF08070DE
:1093200073DB891A801A6EE002282CD1D8F8200F3E
:10933000C0F3C020002869D1B9F82C034FF07A514E
:1093400000051CF00DFD68634FF07A51B9F8300349
:1093500000051CF005FDA863DFF8381CDFF83009B4
:10936000006880041CF0FCFCA96B6A6BA8648A424C
:109370002ED0904231DB8142B8BF4FF0807044DB89
:10938000891A801A3FE0032831D1D8F8200FC0F3A2
:10939000C02000283AD1B9F838034FF07A510005BF
:1093A0001CF0DEFC68634FF07A51B9F83C0300050D
:1093B0001CF0D6FCA863DFF8DC1BDFF80C0D00689E
:1093C00080041CF0CDFCA96B6A6BA8648A4202D1B0
:1093D0004FF4000019E0904201DA002015E08142CC
:1093E000B8BF4FF0807010DB891A801A0BE0042898
:1093F00002BFD8F8200FC0F3C020002806D1E86DC6
:109400004FF07A51C0031CF0ABFC6864D8F8100F21
:10941000C0F3C00010B9B9F844080FE0B9F8D2079A
:1094200010B9B9F8D80709E0686C1FF01DFADFF829
:109430009C1C1CF07DFD1CF0E7FD80B2A86198F833
:10944000980E10F0010002D0B9F8A01151B1D8F86F
:10945000141FC1F3001100291CBFB9F8A021002A74
:1094600000F01281D8F8DC0E032800F06881E8696A
:10947000B9F8FC178842C0F062810020E8614FF41F
:109480007A71B9F85C080028B9F80A0846D11CF0CE
:1094900067FCC8F8F0016421B9F8F6071CF060FC1D
:1094A000C8F8B801B9F8F817080008BF002008D0BC
:1094B000B9F8FC071CF054FC0146D8F8B8011CF0C0
:1094C00097FCC8F8BC01B9F8FC17B9F8FA071CF00A
:1094D00047FC0146D8F8B8011CF08AFCC8F8C00166
:1094E000DFF8280DC8F8C8014FF08070C8F8C40133
:1094F000B9F8DC27E86B696C002A0EBF0A46024601
:109500000846C8F8B401C8F8B0214FF4D870D8F8AC
:10951000FC1140448847D8F8EC0145E01CF020FCE1
:10952000C8F83C026421B9F8F6071CF019FCC8F829
:109530000802B9F8F817080008BF002008D0B9F8E9
:10954000FC071CF00DFC0146D8F808021CF050FC8A
:10955000C8F80C02B9F8FC17B9F8FA071CF000FCBF
:109560000146D8F808021CF043FCC8F81002DFF8E6
:109570009C0CC8F818024FF08070C8F81402B9F8B3
:10958000DC27E86B696C002A0EBF0A4602460846D3
:10959000C8F80402C8F800224FF40070D8F8481246
:1095A00040448847D8F8380280122862A86A032805
:1095B00013D1E86A092810D0286B05280DD12C6A30
:1095C000A86E002C05D480FB0446A40B44EA864414
:1095D0001BE0614280FB010113E02C6AB9F8DE2038
:1095E000002C08D4E617A2FB040102FB0611800B35
:1095F00040EA814409E06442E617A2FB040102FB51
:109600000611800B40EA81404442B9F8FE0740BB96
:10961000B9F8E2170846844214DB11B3D8F89C1E4F
:10962000C1F30011E9B9B9F89E1105291CBF06293B
:10963000012916D0032902BFD8F8F41EC1F3401146
:1096400000290ED00446D8F87C1B4FF097401CF040
:109650006FFC1CF0D9FCC8F8EC01C8F83802C8F857
:109660003002B9F8E807A042A6BF4042844204464F
:109670006C62B9F89601092808BF2C66B9F8980100
:1096800005285CD16C665AE0002804BFB9F8A00137
:10969000002805D0002952D1B9F8A00100284ED0E9
:1096A000D8F89C0EC0F30010002848D1C8F8CC01AF
:1096B000C8F8D001C8F8D401C8F8D801C8F8DC014E
:1096C000C8F8E001C8F8E401C8F8E801C8F8EC01FE
:1096D000C8F81C02C8F82002C8F82402C8F82C02F6
:1096E000C8F828024FF09740D8F87C1B1CF020FCEB
:1096F0001CF08AFCC8F830020020C8F83402C8F810
:109700003802A86A032807D1E86A092804D0286B20
:10971000052808BF002001D0B9F8E2076862B9F84F
:109720009601092804BF686A2866B9F898010528D7
:1097300005D1686A686602E000202865686501B0A6
:10974000DFF840050068A9F85608DFF8440500680E
:10975000A9F85808DFF870090068A9F85A08A8683D
:10976000A9F89602E868A9F898022869A9F89A0267
:10977000BDE8F083F0B5DFF80045D4F89C0EC0F3E7
:109780000010002881B000F01781DFF8F454B5F81C
:10979000D40001001CBF0128032805D0022804BF03
:1097A000B5F81201032808D1D4F8C01700294CBF1E
:1097B00048420846D4F8C41707E0D4F8C417002973
:1097C0004CBF48420846D4F8C017DFF8446A002965
:1097D00048BF49421DF022FAC4F830074FF4E66052
:1097E000D4F8481720448847D4F8440708224FF497
:1097F00080611CF055FAD4F8081E4018F16A491C23
:10980000FF2904D90012C4F80C0E00210020F162D7
:10981000C4F8080E4FF46111D4F80C0E1CF05EFC75
:109820008012C4F8000ED4F80C0E1FF02FF8C4F804
:10983000040E6421306B1CF009FC3060D4F8041E67
:109840001CF04CFC70600A21B5F846061CF0FEFBCB
:10985000014630681CF0FAFBB060D4F8C01CDFF899
:10986000B409002948BF4942814206DB1CF078FA5E
:10987000B16808221CF014FAB060D4F8CC1DB068AE
:109880001CF02CFCF0606421B5F8EC051CF0DEFB4C
:10989000B5F8D41002290EDAB26840F267218A4284
:1098A00009DB8242A8BF002007DAA0F26621801AF5
:1098B0001CF0CCFB01E04FF480603061B4F8920AF8
:1098C000716880021CF00AFC01464FF440601CF0F5
:1098D00005FC0746B5F8480604211CF0B7FB014615
:1098E00038461CF0FBFB0746D4F8301DD4F8EC0DCD
:1098F0006FF001021CF0D4F9D4F8101E1CF0EEFB3E
:10990000014638461CF0A2FB70614FF42061D4F888
:10991000CC0D1CF0E3FB71698142C8BF0146716147
:10992000706931691CF0DAFB07463069F168C0F5EF
:1099300080601CF0D3FBC019B061D4F8CC1D1CF0C2
:1099400085FB0146D4F8EC0D08221CF0A9F901466C
:1099500016224FF080701CF0A3F9C4F84C0704F2F3
:109960004C70D4F864178847D4F8601708224FF475
:1099700080601CF095F9F1694018316AF061491C6A
:10998000FF2931621BD94FF47A2100121CF0A6FB8B
:109990008012B0F5FA6F88BF4FF4FA60706201B0C0
:1099A000B5F8421648434FF47A71B0FBF1F0B0625B
:1099B0000020F0613062F0BDDFF85418886201B019
:1099C000F0BD00005C8F02006666660070B5AC4DAD
:1099D000B5F8D400022818BF03283ED1B5F83E01DF
:1099E000012802BFA44CB4F8860A002835D1B5F886
:1099F000400690BB1EF062FF40F2735190FBF1F104
:109A000040F2735202FB110000F24466C4F8506D3C
:109A100030461CF0F5F901464FF07E501CF00AFA72
:109A20000146DFF8F407C4F8D41C90FBF6F0C4F844
:109A300018054FF097401CF07BFA1CF0E5FAB5F8DA
:109A400054660246C317A6FB020106FB03116422FB
:109A500000231BF013F8C4F86C0770BDF8610020F8
:109A6000145D00203412002010B58548B0F8D410E1
:109A700008001CBF0129062942D1DFF8A047D4F80D
:109A80009C0EC0F3001000283AD0D4F894070629A1
:109A900003D1002808D5404206E00028D4F8641F0E
:109AA00048BF40421CF05CF9C4F870054FF4AE604A
:109AB000D4F8881520448847D4F82C0F401CC4F8EB
:109AC0002C0F0822D4F884054FF4C8211CF0E8F8C4
:109AD000D4F86C1F01EB2030D4F82C1FC4F86C0FA5
:109AE00020291ED340110021B0F5967FC8BF4FF446
:109AF0009670C4F82C1FC4F8680FC4F86C1F10BD12
:109B0000DFF818470020C4F87005C4F88405C4F8CD
:109B10008005C4F8640FC4F8680FC4F86C0FC4F86B
:109B20002C0F10BD407E050000040040985C002012
:109B300070B5DFF8EC46524D2068B5F86C1941B9A4
:109B4000B5F8720900B90120B5F87019012908BFEC
:109B5000404220604FF47A711CF002F9DFF8BC66D5
:109B6000C6F8400F002848BF4042C6F8440FB5F879
:109B70007C0910B9B5F8820960604FF47A716068A9
:109B80001CF0EEF8C6F8500FD6F8DC1DD6F8440FDE
:109B90001CF02EF920620822B5F85416C9031CF0F7
:109BA0007FF8C0136061B5F88C0948B9B5F88E0923
:109BB000B5F8DE1048434FF47A7190FBF1F0A060E5
:109BC000B5F88A09012818BF032803D16169A26882
:109BD000914200D2A1686162B5F8901949B9B5F80F
:109BE0009219B5F8DE2051434FF47A7291FBF2F1ED
:109BF000E160022818BF032803D16169E06881424F
:109C000000D2E168A16296F8280F00F00500012853
:109C100013D1D6F89C0EC0F30010002814BFD6F85C
:109C2000E00ED6F8DC0E81B209B9606A04E080B2B9
:109C300001280CBFA06A00202061A069B5F898191E
:109C400009B9B5F89C0900B90120A0614FF47A71F7
:109C50001CF086F8C6F8580FB5F8A219E06909B9E2
:109C6000B5F8A60900B90120E0614FF47A711CF043
:109C700077F8C6F85C0F70BD00000020F45D00208E
:109C80003843002078100020905E0020645C0020A3
:109C900000110020F0B5DFF88C45B4F8D4000100C5
:109CA0001CBF0128062881B040F06A81FFF7DCFE66
:109CB000FFF73EFFB4F8D400DFF86055062800F047
:109CC0006081D5F8980ED5F8141F820B42EA503205
:109CD00042EA511242EA911242EA113242EA513109
:109CE000D5F8282F61F30412C5F8282FD5F8281FBE
:109CF000C1F30012002A40F01481B4F86069D5F86D
:109D0000302FD5F8343F012E02D0022E14D05AE065
:109D1000CA076DD4D5F89C2E41F00101C5F8281F63
:109D2000C2F300121AB141F00801C5F8281FD5F896
:109D3000281F21F0020159E0B4F86269D5F8F47ED9
:109D400006EB8606B6B2C7F30017F7B90023CF07B4
:109D500050D495F8EC7EFF074CD5521C964249D260
:109D6000D5F89C2E41F00101C5F8281FC2F300125E
:109D70001AB141F00801C5F8281F0022D5F8281FA4
:109D800021F00201C5F8281F34E00022CF0731D5A9
:109D900095F8EC7EFF072DD55B1C9E422AD2490820
:109DA000D5F89C3E4900C5F8281FC3F300131BB12A
:109DB00041F00201C5F8281FD5F8281F21F008013D
:109DC000C5F8281F15E0CA0712D54908D5F89C2EFA
:109DD0004900C5F8281FC2F300121AB141F0020170
:109DE000C5F8281FD5F8281F21F00801C5F8281F3D
:109DF00000220023D5F89C1EC5F8343FC5F8302F4B
:109E0000C1F3001179B3D5F8281FCA07C0F30010B9
:109E100024D50028C1F3800018D028B921F008000B
:109E200040F00200C5F8280F95F8280F00F0050053
:109E3000012840F08B80B4F88009B0F57A7F1FD0FC
:109E4000D5F8606F002E13D5764211E00028EBD0D4
:109E5000042060F34301C5F8281FE5E70028E3D19B
:109E600021F00400DEE7D5F8280F20F00E006BE0AB
:109E7000D5F8880F864203DBD5F88C1F884202DBB9
:109E8000D5F8500F11E08E42A8BF00200DDA091A54
:109E9000D5F8500F1BF064FF0146D5F8880F301A33
:109EA0001BF0A6FFD5F8501F081AC5F8540FD5F8B7
:109EB000541FD5F8580F401A44F289118842B8BF90
:109EC0000846D5F8441F8842C8BF0846C5F8440F65
:109ED00095F8EC0EC0071CD5B4F8640900EB8001BE
:109EE00089B201201BF03CFFD5F8441FD5F84C2F58
:109EF000C5F8480F8A420CD004DA8018C5F84C0F18
:109F0000814203E0101AC5F84C0F8842B8BFC5F86B
:109F10004C1FD5F84C0FD5F8541F0818C5F87C0F06
:109F200014E0C80734D54908D5F89C0E4900C5F897
:109F3000281FC0F3001018B141F00200C5F8280F27
:109F4000D5F8280F20F00C00C5F8280FB4F8A001B0
:109F5000F0B195F8280FC00744BFD5F8400F00288E
:109F600016D5D5F8DC0E20B90120C5F8DC0E01B0FD
:109F7000F0BD01280CD10020C5F8DC0E01B0F0BD09
:109F8000A64D0020C5F8280FC5F8300FC5F8340FCE
:109F900001B0F0BD0000FC3F70B58CB004A81CF00F
:109FA0008BFA0020ADF810002020ADF8120004A9B3
:109FB0009A4C9D4DD4F81805401EADF8140040F29F
:109FC00005560020ADF8160001208DF8180028462F
:109FD0001CF064F968461CF078FA7020ADF80000B7
:109FE000ADF806600120ADF8020069460420ADF826
:109FF00004000220ADF808000820ADF80A00002097
:10A00000039028461CF095F9ADF80660694628468D
:10A010001CF0CFF9ADF80660694628461CF003FA3B
:10A02000082128461CF0A2FA082128461CF0A5FAAF
:10A03000082128461CF0A9FA012128461CF08CFAB8
:10A040004FF40060ADF81C004FF48060ADF81E00C6
:10A050000020ADF82000D4F89C0DB0F5AF7F06D9F4
:10A0600000EBC0006421B0FBF1F0A03006E000EB93
:10A07000C00188006421B0FBF1F04030ADF822004F
:10A0800007A94FF48050ADF824000020ADF8260059
:10A09000ADF8280028461CF0FFF9202128461CF0C6
:10A0A0007BFA802128461CF08DFA01228021284667
:10A0B0001CF02AFA012128461CF011FA0121284639
:10A0C0001CF017FA0CB070BD8411002000007A4417
:10A0D00070B58CB004A81CF0EFF90020ADF81000AA
:10A0E0002020ADF8120004A94C4C4F4DD4F81805AF
:10A0F000401EADF8140040F205560020ADF81600E1
:10A1000001208DF8180028461CF0C8F868461CF09D
:10A11000DCF97020ADF80000ADF806600020ADF865
:10A120000200ADF8040069460220ADF808000820DE
:10A13000ADF80A000020039028461CF0FAF8012030
:10A14000ADF80200ADF806600420ADF804006946E1
:10A1500028461CF02EF9ADF80660694628461CF02A
:10A1600062F9082128461CF001FA082128461CF053
:10A1700004FA082128461CF008FA012128461CF0A0
:10A18000EBF94FF40060ADF81C004FF48060ADF8BF
:10A190001E000020ADF82000D4F89C0DB0F5AF7F74
:10A1A00006D900EBC0006421B0FBF1F0A03006E05E
:10A1B00000EBC00188006421B0FBF1F04030ADF845
:10A1C000220007A94FF48050ADF824000020ADF81C
:10A1D0002600ADF8280028461CF05EF9202128460C
:10A1E0001CF0DAF9802128461CF0ECF901228021CC
:10A1F00028461CF089F9012128461CF070F901213C
:10A2000028461CF076F90CB070BD000033333300E3
:10A21000505F00208FC2F500005125020000002091
:10A22000B45F002038430020002C01402DE9F041AC
:10A23000012104201EF0FAFB012108201EF0F6FB8C
:10A24000012110201EF0F2FB012120201EF0EEFB68
:10A25000012140201EF0EAFB012101201EF0E6FB57
:10A26000DFF89C47082120461CF092FBDFF894574A
:10A270004FF4004128461CF08BFB4FF480412846E8
:10A280001CF086FB4FF4005128461CF081FBDFF8E0
:10A2900078674FF4006130461CF07AFBDFF86C778A
:10A2A000802138461CF074FB4FF4007138461CF0D6
:10A2B0006FFBDFF85C875320A8F8680008F168019D
:10A2C000022088F86A00002088F86B0038461CF0ED
:10A2D000F1FA41F62850A8F8680008F16801022058
:10A2E00088F86A00042088F86B0038461CF0E2FA0F
:10A2F0000320A8F8680008F16801022088F86A00C5
:10A30000002088F86B0028461CF0D4FA4FF6E07065
:10A31000A8F8680008F16801032088F86A00102096
:10A3200088F86B0028461CF0C5FA4FF64140A8F8A3
:10A33000680008F16801022088F86A00042088F8A3
:10A340006B0020461CF0B6FA01224FF4604128460B
:10A350001CF022FB3620A8F8680008F168010220F2
:10A3600088F86A00002088F86B0020461CF0A2FAEA
:10A370004FF46270A8F8680008F16801032088F8BB
:10A380006A00142088F86B0020461CF093FA40F60F
:10A39000FF00A8F8680008F16801022088F86A0048
:10A3A000142088F86B0030461CF084FA01224FF428
:10A3B000006130461CF0F0FA0022FF2130461CF00C
:10A3C000EBFA4FF47740A8F8680008F16801022022
:10A3D00088F86A00042088F86B0030461CF06AFA9E
:10A3E00044F2FF00A8F8680008F16801022088F82C
:10A3F0006A00042088F86B00DFF818061CF05AFA8F
:10A400002846BDE8F04101224FF47C511CF0C4BA4B
:10A4100070B501217D201EF009FB01214FF4006081
:10A420001EF004FBDFF8F045DFF8E45520461BF092
:10A430005DFE05F140001CF03FF80020A5F840004B
:10A4400005F140012020A5F8420040F2055648F6EB
:10A45000A040A5F844000020A5F84600012085F89A
:10A46000480020461BF01AFF28461CF02EF87020EA
:10A470002880EE800120688029460420A8800220E0
:10A480002881082068810020E86020461BF051FFE9
:10A49000EE80294620461BF08CFFEE8029462046A0
:10A4A0001BF0C1FF082120461CF060F8082120465F
:10A4B0001CF063F8082120461CF067F801212046B3
:10A4C0001CF04AF80121DFF85405DFF848651CF05C
:10A4D00070FA05F168001CF04CFA4FF47C50A5F8B6
:10A4E000680005F16801182085F86B00032085F8E5
:10A4F0006A0030461CF0DEF94FF4285130461CF05B
:10A5000050FA05F168001CF034FA4FF40040A5F849
:10A51000680005F16801042085F86B0030461CF0E6
:10A52000C9F94FF4006028844FF4806068840020EB
:10A53000A884DFF8EC040068B0F5AF7F06D900EB23
:10A54000C0006421B0FBF1F0A03006E000EBC001D8
:10A5500088006421B0FBF1F04030E88405F120016F
:10A560004FF48050288500206885A88520461BF080
:10A5700093FF202120461CF00FF8802120461CF07C
:10A5800021F82046BDE8704001211BF0A8BFF0B5BE
:10A5900081B04FF400401EF001FA01214FF4007029
:10A5A0001EF044FA01214FF480601EF03FFADFF8FC
:10A5B0007444DFF87454DFF8746420461EF06AFABD
:10A5C00028461EF067FA012120461EF0B6FA012146
:10A5D00028461EF0B2FA30461EF0A6FA4FF4A0202C
:10A5E00030604FF4602701203071B7600020707137
:10A5F000F06031460420307420461EF077FA0120C6
:10A600003071B76000207071F06031460420307402
:10A6100028461EF06BFA20461EF0A1FA20461EF0D6
:10A62000A3FA0028FAD128461EF099FA28461EF00F
:10A630009BFA0028FAD120461EF09BFA20461EF015
:10A640009DFA0028FAD128461EF093FA28461EF0FB
:10A6500095FA0028FAD1042120461EF0D5FA0023ED
:10A660000122002120461EF0A6FA00230222082122
:10A6700020461EF0A0FA00230322092120461EF0E6
:10A680009AFA00230422062120461EF094FA0021A3
:10A6900020461EF081FA012120461EF083FA012196
:10A6A00020461EF070FA042120461EF0BFFA042155
:10A6B00028461EF0A9FA00230122012128461EF097
:10A6C0007AFA002302220C2128461EF074FA002395
:10A6D00003220B2128461EF06EFA002304220E21CD
:10A6E00028461EF068FA012128461EF05BFA012177
:10A6F00028461EF048FA204601B0BDE8F04001228D
:10A700004FF490611EF022BA70B5012144F20500A9
:10A710001EF08CF9BD4E4FF4806130461CF038F9C4
:10A72000BB4C4FF40070A4F8680004F168010120EC
:10A7300084F86A004FF48065182084F86B00304676
:10A740001CF0B8F8012084F86A00A4F868500420CE
:10A7500084F86B0004F1680130461CF0ABF8B44E8D
:10A7600030461DF031FF04F110001DF0CDFF4FF415
:10A770009650206125834FF48050A08204F110018F
:10A780000020E082A0830C20608330461DF064FF2F
:10A790003046BDE8704001211DF0C2BF30B581B028
:10A7A00001214FF400301EF04AF9984D042128464B
:10A7B0001CF0EEF8082128461CF0EAF8944C04201E
:10A7C000A4F8680004F16801012084F86A001820E8
:10A7D00084F86B0028461CF06DF80820A4F8680087
:10A7E00004F16801012084F86A00042084F86B00F9
:10A7F00028461CF05FF88F4D28461DF0E5FE04F159
:10A8000010001DF081FF4FF41650206104F110017B
:10A810004FF48050A0820020E0824FF480602083BB
:10A820000020A0830C20608328461DF015FF2846D9
:10A8300001B0BDE8304001211DF072BF10B501210B
:10A8400004201EF0F3F8724C3020A4F8680004F1E4
:10A850006801002084F86B006C481CF02BF8012183
:10A860004FF000501EF0EBF81EF0F6F904F1300046
:10A870001EF015FA00202063606304F1300102200D
:10A88000E06300201EF0F7F904F1300110201EF003
:10A89000F2F9012100201EF008FA012110201EF01B
:10A8A00004FA002100201EF019FA012100201EF0F8
:10A8B00008FABDE81040012110201EF002BA30B5A0
:10A8C00081B0012102201EF0BAF8012104201EF0FF
:10A8D000ADF84F4C584D48F6A040A4F8600004F184
:10A8E0005C010020E065A4F862004FF080401BF09E
:10A8F000D5FC6020A4F84C0004F14C010120A4F820
:10A900004E000020A4F852000220A4F8540028466B
:10A910001BF04FFD082128461BF02FFE0121284681
:10A920001BF01AFE8020A4F8680004F168010320DF
:10A9300084F86A00182084F86B0034481BF0BAFFD2
:10A94000012101201EF07BF84FF080401BF0CEFB70
:10A9500040F69F70A4F8600004F15C010820A4F8A0
:10A960005C000020A4F86200A4F85E004FF0804074
:10A970001BF094FC01214FF080401BF016FE0122D9
:10A9800001214FF080401BF0BFFD01B0BDE8304019
:10A9900001214FF080401BF0A2BD10B54FF4A06024
:10A9A0001EF0BAF9254C182020700020607001209C
:10A9B000A070E07020461EF0B4F912202070002034
:10A9C00060700220A0700120E07020461EF0A9F9FE
:10A9D0001C202070012060700220A0700120E07017
:10A9E00020461EF09EF92620207001206070A07085
:10A9F000E0702046BDE810401EF093B90000000052
:10AA000000100140000C014000140140000801400A
:10AA1000885D002000180140002C0140C000160095
:10AA20009C0D00200024014000280140EC60002023
:10AA300000380140004400400004004078610020DC
:10AA400000B581B0FFF7F2FBFFF7E2FCFFF79FFDD7
:10AA5000FFF75AFEFFF7A2FEFFF7F0FEFFF72FFF0A
:10AA600001B05DF804EB98E710B5DFF89C494FF4AE
:10AA7000007120461BF08CFF092009F052F880215C
:10AA800020461BF085FF092009F04BF84FF4807138
:10AA900020461BF07DFF092009F043F82046BDE861
:10AAA00010404FF480711BF075BF70B504460D4621
:10AAB000092009F036F8280022D0DFF84C69600040
:10AAC000A4B2B4F5004F044604DA802130461BF0EE
:10AAD00061FF03E0802130461BF05AFF092009F096
:10AAE00020F84FF4807130461BF052FF092009F026
:10AAF00018F84FF4807130461BF04CFF6D1EDED10C
:10AB000070BD000070B504460D46092009F009F833
:10AB1000280027D0DFF8F0684FF4807130461BF032
:10AB200037FF092008F0FDFF802130461BF030FF81
:10AB3000802130461BF02CFF092008F0F2FF802115
:10AB400030461BF01EFF6400012808BF44F00104DA
:10AB50004FF4807130461BF01DFF092008F0E1FF23
:10AB60006D1ED9D1A0B270BD10B5092008F0D9FF73
:10AB7000DFF894484FF4007120461BF00BFF0920CA
:10AB800008F0CFFF4FF4807120461BF001FF092031
:10AB900008F0C7FF4FF4007120461BF0F9FE0920B2
:10ABA00008F0BFFF4FF4807120461BF0F3FE092030
:10ABB00008F0B7FF802120461BF0EAFE80212046E6
:10ABC0001BF0E6FE092008F0ACFF802120461BF0B8
:10ABD000D8FE0028EED02046BDE810404FF40071AA
:10ABE0001BF0D8BE30B540F63401884281B046DA59
:10ABF00040F214518842DFF8142835DA1523DFF8C3
:10AC0000101800F041FD00F11704DFF8FC574FF475
:10AC1000007128461BF0BCFE092008F082FF80214D
:10AC200028461BF0B5FE092008F07BFF4FF4807129
:10AC300028461BF0ADFE092008F073FF4FF4807129
:10AC400028461BF0A7FE2001A0F500400C2180B291
:10AC5000FFF72BFF10210020FFF754FF0446FFF7FA
:10AC600083FF204601B030BD1523DFF8A81700F0A0
:10AC70001BFC00F11704A4B2B4F5806FC5D100200D
:10AC800001B030BD70B50D46DFF88C1721F81050BB
:10AC900040F63401884261DA40F214518842DFF80C
:10ACA0006C275CDA1523DFF8681700F0EDFC00F183
:10ACB0001704DFF854674FF4007130461BF068FE4C
:10ACC000092008F02EFF802130461BF061FE09208C
:10ACD00008F027FF4FF4807130461BF059FE092021
:10ACE00008F01FFF4FF4807130461BF053FE0C211B
:10ACF0004FF44050FFF7D9FE092008F012FFFFF78C
:10AD000033FF4FF4007130461BF042FE092008F07B
:10AD100008FF802130461BF03BFE092008F001FFB0
:10AD20004FF4807130461BF033FE092008F0F9FE25
:10AD30004FF4807130461BF02DFE200100F580405D
:10AD40000C2180B2FFF7B1FE092008F0EAFE1021C5
:10AD50002846FFF7AAFEBDE8704005E770BD152341
:10AD6000DFF8B01600F0A0FB00F11704A4B2B4F5B0
:10AD7000806F9ED170BD10B5DFF88C464FF4007126
:10AD800020461BF005FE092008F0CBFE802120465E
:10AD90001BF0FEFD092008F0C4FE4FF48071204630
:10ADA0001BF0F6FD092008F0BCFE4FF48071204630
:10ADB0001BF0F0FD0C210020FFF777FEBDE81040EE
:10ADC000D2E600002DE9F04FDFF85016DFF83C9690
:10ADD000DFF83C76002481B00C804E464FF0160818
:10ADE00035883888A8425BD301F0A2FAA4B204EBFC
:10ADF00044008000DFF8281601444989C90549D478
:10AE0000DFF81C1631F800A0DFF81806DFF8081686
:10AE1000A0F800A0ADB2284621F810A040F63401F9
:10AE2000884237DA40F21451884208DA15234A463C
:10AE3000DFF8DC1500F028FC00F1170B0BE0152300
:10AE40004A46DFF8D01500F02FFB17301FFA80FBC1
:10AE5000BBF5806F1ED0FFF707FE0C214FF440506A
:10AE6000FFF723FE092008F05CFEFFF77DFEFFF7E9
:10AE7000FBFD4FEA0B1000F580400C2180B2FFF77C
:10AE800014FE092008F04DFE10215046FFF70DFE7C
:10AE9000FFF76AFE6D1C3888641CA9B28842A3D2F1
:10AEA000BF1CB61CB8F101089AD101B0BDE8F08F03
:10AEB0002DE9F04FDFF85485DFF8541585B01523E0
:10AEC000424640F2EC4000F0DFFB04464FF40071D4
:10AED000DFF834051BF05CFD092008F022FE80211C
:10AEE000DFF824051BF054FD092008F01AFE4FF48A
:10AEF0008071DFF814051BF04BFD092008F011FEEE
:10AF00004FF48071DFF800051BF044FD200147F687
:10AF10009062801A0C2180B2FFF7C7FD102100203B
:10AF2000FFF7F0FD0446FFF71FFEDFF8FC04DFF833
:10AF3000E414029004801523424640F60A0000F013
:10AF4000B3FA00F1170400260025A4B2B4F5806F0F
:10AF50002ED04FF40071DFF8B0041BF019FD09206A
:10AF600008F0DFFD8021DFF8A0041BF011FD0920AF
:10AF700008F0D7FD4FF48071DFF88C041BF008FD5A
:10AF8000092008F0CEFD4FF48071DFF87C041BF03F
:10AF900001FD2001A0F500400C2180B2FFF785FDE6
:10AFA00010210020FFF7AEFD0446FFF7DDFD00E0B5
:10AFB00000240298A0F83C4640F2D2410298B0F832
:10AFC0003C06884200F0A880DFF85014DFF84044C7
:10AFD0000D801620CDF80080019040F2145940F603
:10AFE000340A009807882088B8424FDB01F0A0F9A6
:10AFF000B6B206EB4601DFF82804890030F801B04C
:10B00000DFF82004DFF81014A0F800B0384621F86B
:10B0100010B0504534DA484508DA15234246DFF8C7
:10B02000F01300F031FB00F117050BE01523424649
:10B03000DFF8E01300F038FA00F11705ADB2B5F50E
:10B04000806F1DD0FFF710FD0C214FF44050FFF72B
:10B050002CFD092008F065FDFFF786FDFFF704FDD4
:10B06000280100F580400C2180B2FFF71EFD092069
:10B0700008F057FD10215846FFF717FDFFF774FD44
:10B080007F1C2088761CBFB2B842AFDA4FF4FA605A
:10B0900008F025FD0098801C0090A41C0198401E1B
:10B0A00001909ED101F044F9DE4940F2D24008807F
:10B0B00015230299A1F83C064246D64940F60A00FB
:10B0C00000F0F2F900F11704A4B2B4F5806F1ED0BD
:10B0D000FFF7CAFC0C214FF44050FFF7E6FC0920B3
:10B0E00008F01FFDFFF740FDFFF7BEFC200100F553
:10B0F00080400C2180B2FFF7D8FC092008F011FD38
:10B10000102140F2D240FFF7D0FCFFF72DFD4FF4A5
:10B11000FA6008F0E4FC4EE102980088884200F0F2
:10B120004D81BB480090CDF804801620039040F27A
:10B13000145940F6340A0198078800980088B842EC
:10B14000C0F2D78001F0F4F80C2F18BF0D2F00F0DB
:10B15000C88002980088002840F081800B2F1CBF17
:10B1600040F23A30874204D0672F1CBF682FE52F8A
:10B1700032D13846504529DA484507DA1523424688
:10B18000A34900F081FA00F117040AE015234246B2
:10B19000A04900F089F900F11704A4B2B4F5806F5A
:10B1A00014D0FFF761FC2001A0F500400C2180B213
:10B1B000FFF77BFC10210020FFF7A4FC0446FFF7FB
:10B1C000D3FC954820F8174001258AE092480024D6
:10B1D00020F81740012584E0B6B206EB4600800057
:10B1E0008F490C5A8F488C490480384621F810400A
:10B1F000504532DA484507DA15234246844900F0C3
:10B2000043FA00F117050AE015234246814900F090
:10B210004BF900F11705ADB2B5F5806F1DD0FFF702
:10B2200023FC0C214FF44050FFF73FFC092008F0AD
:10B2300078FCFFF799FCFFF717FC280100F5804028
:10B240000C2180B2FFF731FC092008F06AFC1021C4
:10B250002046FFF72AFCFFF787FC012541E0B6B244
:10B2600006EB460080006E490C5A6E486A4904801D
:10B27000384621F81040504533DA484507DA15239F
:10B280004246634900F000FA00F1170B0AE015236B
:10B290004246604900F008F917301FFA80FBBBF501
:10B2A000806F1ED0FFF7E0FB0C214FF44050FFF7FA
:10B2B000FCFB092008F035FCFFF756FCFFF7D4FB38
:10B2C0004FEA0B1000F580400C2180B2FFF7EDFB38
:10B2D000092008F026FC10212046FFF7E6FBFFF7C7
:10B2E00043FC009800887F1C761CBFB2B842BFF6B2
:10B2F00029AF4FF4FA6008F0F2FB0098801C009030
:10B300000198801C01900398401E03907FF413AFB6
:10B310005DB105F083FB05F053FC05F0C3FE05F0BD
:10B32000FBFF04F0CFFE00F075FB029940F2D24023
:10B33000088015234246364940F2EC4000F0A4F95B
:10B3400004464FF4007130481BF022FB092008F03E
:10B35000E8FB80212C481BF01BFB092008F0E1FBD7
:10B360004FF4807128481BF013FB092008F0D9FB2B
:10B370004FF4807124481BF00DFB0C214FF440501A
:10B38000FFF793FB092008F0CCFBFFF7EDFBFFF77D
:10B390006BFB200100F5824070300C2180B2FFF77A
:10B3A00084FB092008F0BDFB102140F2D240FFF7DA
:10B3B0007CFBFFF7D9FB1949642008804FF400712A
:10B3C00011481BF0E5FA092008F0ABFB80210E487C
:10B3D0001BF0DEFA092008F0A4FB4FF480710A4844
:10B3E0001BF0D6FA092008F09CFB4FF48071064848
:10B3F0001BF0D0FA0C210020FFF757FB05B0BDE889
:10B40000F04FFFF7B1BB000000100140D4910208DB
:10B410007C910208A89102083843002004210020F2
:10B420000092020806210020104D002070B5DFF8C0
:10B43000E04CB4F8AC00B4F8AA60B4F8AE500128FF
:10B440001CBFB4F8B000012827D1DFF8C80C006891
:10B45000C0F3402000B1761CB6B2B6F5967F0BDD86
:10B46000DFF8B40C00680026C0F3001010B1DFF85C
:10B47000B01E0E8006F0F0FAB4F8B000012808BF44
:10B480006D1CADB2652D09DB00250026A4F8B05077
:10B49000A4F8AE50A4F8AA6070BD0026A4F8AE507F
:10B4A000A4F8AA6070BD00002DE9F04F06461846CA
:10B4B00064253346A946B3FBF5F335469BB2B5FB8D
:10B4C000F9F581B01C46ADB2162C09FB1565DFF805
:10B4D00054AEDFF854EE009528BF15244FF0000C51
:10B4E00064B314F0030609D03EF8027B3AF802BBBD
:10B4F000A7EB0B077F1C761EBC44F5D1A4081DD01A
:10B500003EF8026B3AF8027BF61B761CB4443EF818
:10B51000026B3AF8027BF61B761CB4443EF8026BD1
:10B520003AF8027BF61B761CB4443EF8026B3AF8FC
:10B53000027BF61B761C641EB444E1D1AC441FFAB6
:10B540008CF4DFF8E8AD04EB44040AEB8404A47A3D
:10B55000E40748BF40F2E93000F19380984238BFD9
:10B5600003464FF0000C6BB313F0030000F00980AA
:10B5700031F8026B32F8024B341B641C401EA444A9
:10B58000F6D1980800F01E8031F8026B32F8024BB9
:10B59000341B641CA44431F8026B32F8024B341B98
:10B5A000641CA44431F8026B32F8024B341B641C57
:10B5B000A44431F8026B32F8024B341B641C401E69
:10B5C000A444E1D10021002D58D009FB03F2CE465E
:10B5D00090B2B0FBFEFE1FFA8EFEB0FBF9F0BEF19A
:10B5E000160F94B280B228BF4FF0150E09FB104021
:10B5F0000024BEF1000FDFF82C3DDFF82C8D30D099
:10B600001EF0030600F00A8038F8027B33F802BB14
:10B61000A7EB0B077F1C3C19761EF5D15FEA9E0E47
:10B6200000F01F8038F8026B33F8027BF61B761CA3
:10B63000341938F8026B33F8027BF61B761C341988
:10B6400038F8026B33F8027BF61B761C341938F895
:10B65000026B33F8027BF61B761C3419BEF1010E27
:10B66000E0D1001980B200EB40030AEB8300807A3E
:10B67000C00758BF491C521C6D1EA8D101EB0C001D
:10B6800080B201B0BDE8F08FF0B464250446B4FB8D
:10B69000F5F4A4B2A34238BF1C460346B3FBF5F34E
:10B6A0009BB205FB1300002364B314F0030508D01C
:10B6B00031F8026B32F8027BF61B761CF3186D1E14
:10B6C000F6D1A40800F01E8031F8025B32F8026B5C
:10B6D000AD1B6D1CEB1831F8025B32F8026BAD1B31
:10B6E0006D1CEB1831F8025B32F8026BAD1B6D1C60
:10B6F000EB1831F8025B32F8026BAD1B6D1CEB18D6
:10B70000641EE1D1F0BCC01880B2704710B5DFF8FC
:10B71000944DB4F8C80101282CD102216A20FFF70A
:10B72000B1FA0121CB20FFF7ADFA0221CC20FFF7BF
:10B73000A9FA0121CF20FFF7A5FA01214FF49E704D
:10B74000FFF7A0FA3A2140F23D10FFF79BFA3421AF
:10B750004FF49F70FFF796FA022140F23F10FFF777
:10B7600091FA08214FF4A070FFF78CFA002140F203
:10B77000411001E1022835D102216A20FFF782FA47
:10B780000121CB20FFF77EFA0221CC20FFF77AFAC5
:10B790000221CF20FFF776FA0021D020FFF772FABE
:10B7A00038214FF49E70FFF76DFA392140F23D10B9
:10B7B000FFF768FA37214FF49F70FFF763FA3A21D9
:10B7C00040F23F10FFF75EFA08214FF4A070FFF738
:10B7D00059FA002140F24110FFF754FA002140F2DB
:10B7E000AF10C9E0032835D102216A20FFF74AFAD9
:10B7F0000421CB20FFF746FA0121CC20FFF742FAC3
:10B800000121CF20FFF73EFA0021D020FFF73AFABE
:10B8100038214FF49E70FFF735FA032140F23D10B6
:10B82000FFF730FA04214FF49F70FFF72BFA052140
:10B8300040F23F10FFF726FA08214FF4A070FFF7FF
:10B8400021FA002140F24110FFF71CFA002140F2DA
:10B85000AF1091E004284ED102216A20FFF712FABE
:10B8600000217020FFF70EFA00217120FFF70AFA7D
:10B870000021CB20FFF706FA0021CC20FFF702FAC7
:10B880000021CF20FFF7FEF90121D020FFF7FAF9C0
:10B890000121E020FFF7F6F90F214FF49E70FFF72A
:10B8A000F1F90D2140F23D10FFF7ECF90E214FF4B4
:10B8B0009F70FFF7E7F9362140F23F10FFF7E2F9FA
:10B8C00008214FF4A070FFF7DDF9002140F241108C
:10B8D000FFF7D8F9002140F2AF10FFF7D3F9B4F821
:10B8E000E200DFF8B01D00F57F40FF300860DFF8B0
:10B8F000A81D086010BD052842D102216A20FFF76B
:10B90000C1F90921CB20FFF7BDF90021CC20FFF7B9
:10B91000B9F90021CF20FFF7B5F90021D020FFF7BA
:10B92000B1F901214FF49E70FFF7ACF93A2140F2D2
:10B930003D10FFF7A7F934214FF49F70FFF7A2F9EC
:10B94000022140F23F10FFF79DF908214FF4A0704B
:10B95000FFF798F9002140F24110FFF793F9002119
:10B9600040F2AF10FFF78EF9012140F2E930FFF706
:10B9700089F9022140F2EA30BDE81040FFF782B9B0
:10B9800010BD40F22A33984200D07047DFF80C0D0A
:10B9900000B50068032881B03AD1012A41F27070E5
:10B9A0001DD1814208D14FF4E67140F22230FFF7F9
:10B9B00069F94FF4E1610BE041F28830814227D10F
:10B9C0004FF4BE7140F22230FFF75CF940F2B451FF
:10B9D00001B05DF804EB40F22530FFF753B9814226
:10B9E00008D1DFF8C00A4FF4E671A0F844164FF40E
:10B9F000E1610BE041F28830814209D1DFF8A40A0D
:10BA00004FF4BE71A0F8441640F2B451A0F84A16A3
:10BA100001B000BD30B5DFF88C4AB4F8CA01012886
:10BA200081B000F07283022820D1B4F8D00003283E
:10BA3000C0F26B83DFF8680C0168C1F38022002A32
:10BA400040F0638341F48061016040F22A31DFF805
:10BA5000C046A4F8861040F2DD20FFF713F940F24B
:10BA60000231A4F8861040F2632049E303286DD127
:10BA7000DFF89C460020A4F8860000216A20FFF72A
:10BA800001F942F60411A4F886106F20FFF7FAF8C6
:10BA90000F20A4F886000F217220FFF7F3F80F2083
:10BAA000A4F886000F217320FFF7ECF80120A4F81A
:10BAB000860001217720FFF7E5F80A20A4F8860028
:10BAC0000A214FF44B70FFF7DDF80020A4F8860040
:10BAD00000219F20FFF7D6F80120A4F8860001215D
:10BAE000CB20FFF7CFF80120A4F886000121D02059
:10BAF000FFF7C8F80020A4F88600002140F2E120FA
:10BB0000FFF7C0F80020A4F88600002140F2DB40D7
:10BB1000FFF7B8F81920A4F88600192140F2363052
:10BB2000FFF7B0F840F6C415A4F88650294640F255
:10BB3000CE40FFF7A7F8A4F88650294640F2D3403C
:10BB4000FFF7A0F8002140F25F20D9E2042823D1BA
:10BB5000B4F8D000032812DBDFF8440B0168C1F30E
:10BB6000802262B941F48061016040F22A31DFF83D
:10BB7000A005A0F8861040F2DD20FFF783F8002131
:10BB80007020FFF77FF8012140F2BE20FFF77AF81E
:10BB9000192140F2BF20B3E2052818D1DFF8000BCD
:10BBA0000168C1F38022002A00F0AF8221F4806195
:10BBB0000160B4F8D0000328C0F2A782DFF8500576
:10BBC00040F22A31A0F8861040F2DD2098E20628E3
:10BBD00040F0AD8049F6404529466F20FFF752F806
:10BBE00029467120FFF74EF829467620FFF74AF8DC
:10BBF00001217720FFF746F84FF47A619920FFF78B
:10BC000041F800219F20FFF73DF803214FF49E707B
:10BC1000FFF738F8042140F23D10FFF733F8052113
:10BC20004FF49F70FFF72EF80F214FF4A070FFF72D
:10BC300029F842F210714FF4FC70FFF723F843F635
:10BC4000982140F2F910FFF71DF844F620614FF4F7
:10BC5000FD70FFF717F846F2A81140F2FB10FFF74E
:10BC600011F847F230514FF4FE70FFF70BF848F629
:10BC7000B80140F2FD10FFF705F829464FF4FF70B8
:10BC8000FFF700F8502140F20720FEF7FBFF50219C
:10BC90004FF40270FEF7F6FF502140F20920FEF744
:10BCA000F1FF502140F20A20FEF7ECFF502140F254
:10BCB0000B20FEF7E7FF50214FF40370FEF7E2FF81
:10BCC000502140F20D20FEF7DDFF642140F21620E6
:10BCD000FEF7D8FF642140F21720FEF7D3FF64215E
:10BCE0004FF40670FEF7CEFF642140F21920FEF7F4
:10BCF000C9FF642140F21A20FEF7C4FF642140F21C
:10BD00001B20FEF7BFFF64214FF40770FEF7BAFF58
:10BD1000012140F2BE20FEF7B5FF45F6C05140F2CA
:10BD20002530FEF7AFFF294640F22A30E8E1072828
:10BD30006ED1F74C0020A4F8860000216A20FEF79F
:10BD4000A1FF42F21071A4F886106F20FEF79AFF4F
:10BD50002820A4F8860028217220FEF793FF2820CF
:10BD6000A4F8860028217320FEF78CFF0120A4F898
:10BD7000860001217720FEF785FF0A20A4F88600BF
:10BD80000A214FF44B70FEF77DFF0020A4F88600D7
:10BD900000219F20FEF776FF0120A4F886000121F4
:10BDA000CB20FEF76FFF0120A4F886000121D020F0
:10BDB000FEF768FF0020A4F88600002140F2E12091
:10BDC000FEF760FF0020A4F88600002140F2DB406F
:10BDD000FEF758FF1920A4F88600192140F23630EA
:10BDE000FEF750FF4FF4FA60A4F88600014640F2D7
:10BDF000CE40FEF747FF40F6C415A4F8865029460A
:10BE000040F2D340FEF73EFF002140F25F2077E191
:10BE1000082840F00F8149F6404529466F20FEF77B
:10BE200031FF29467120FEF72DFF32217220FEF7E7
:10BE300029FF50217320FEF725FF29467620FEF7C3
:10BE400021FF01217720FEF71DFF00219F20FEF733
:10BE500019FF0121D020FEF715FF03214FF49E703A
:10BE6000FEF710FF042140F23D10FEF70BFF052105
:10BE70004FF49F70FEF706FF072140F23F10FEF7D8
:10BE800001FF0F214FF4A070FEF7FCFE42F210718B
:10BE90004FF4FC70FEF7F6FE43F6982140F2F910DD
:10BEA000FEF7F0FE44F620614FF4FD70FEF7EAFE67
:10BEB00046F2A81140F2FB10FEF7E4FE47F23051C3
:10BEC0004FF4FE70FEF7DEFE48F6B80140F2FD10BA
:10BED000FEF7D8FE29464FF4FF70FEF7D3FE32215D
:10BEE00040F20720FEF7CEFE32214FF40270FEF73B
:10BEF000C9FE322140F20920FEF7C4FE322140F291
:10BF00000A20FEF7BFFE322140F20B20FEF7BAFEF8
:10BF100032214FF40370FEF7B5FE322140F20D20BE
:10BF2000FEF7B0FE502140F21620FEF7ABFE502186
:10BF300040F21720FEF7A6FE50214FF40670FEF7E0
:10BF4000A1FE502140F21920FEF79CFE502140F244
:10BF50001A20FEF797FE502140F21B20FEF792FEBA
:10BF600050214FF40770FEF78DFE45F6C055294667
:10BF700040F22530FEF786FE41F2883140F22A3049
:10BF8000FEF780FE042140F25F20FEF77BFE8F214A
:10BF900040F26120FEF776FE03214FF41970FEF7A0
:10BFA00071FE002140F26E20FEF76CFE4FF44871E6
:10BFB0008C20FEF767FE4FF47A618E20FEF762FE5A
:10BFC0004FF4FA519020FEF75DFE4FF47A51922023
:10BFD000FEF758FE29469420FEF754FE4FF4FA412E
:10BFE0009620FEF74FFE02218D20FEF74BFE0C211E
:10BFF0008F20FEF747FE1A219120FEF743FE3C21D9
:10C000009320FEF73FFE52219520FEF73BFE612173
:10C010009720FEF737FEFA214FF42570FEF732FE27
:10C02000B4F8E200DFF86C1600F57F40FF300860DE
:10C0300001B030BD092868D100217020FEF722FE32
:10C040000221CA20FEF71EFE0121CB20FEF71AFEB8
:10C050000421CC20FEF716FE0121CF20FEF712FEB0
:10C060000221D020FEF70EFE0D214FF49670FEF750
:10C0700009FE052140F22D10FEF704FE0F214FF4BA
:10C080009E70FEF7FFFD102140F23D10FEF7FAFD15
:10C0900021214FF49F70FEF7F5FD032140F23F1080
:10C0A000FEF7F0FD04214FF4A070FEF7EBFD0F2129
:10C0B0004FF49E70FEF7E6FD00214FF4FC70FEF792
:10C0C000E1FD40F6C415294640F2F910FEF7DAFD0D
:10C0D00029464FF4FD70FEF7D5FD41F2883140F25C
:10C0E000FB10FEF7CFFD002140F26520FEF7CAFDF0
:10C0F000012140F22340FEF7C5FD012140F2264018
:10C1000001B0BDE83040FEF7BDBD01B030BD00005C
:10C1100080200020EC0E00209C0E0020DFF8040D93
:10C12000B0F8701000EB4100B0F86010022900F088
:10C130009280102900F0A380122900F08480192930
:10C1400079D0242967D030296DD0402953D078295F
:10C1500000F08980792956D07F2900F0BC808029A1
:10C1600000F08580822972D0832900F09080862992
:10C1700000F09980882900F08680892900F09B8052
:10C180008C2900F0A4808E2900F09180902972D033
:10C19000912900F0BC80922951D0992947D0A1293A
:10C1A0007DD0A32900F0AB80A42930D0A72900F0CE
:10C1B0009E80AF2900F09780B02930D0BF2900F0D1
:10C1C0009A80C02913D0C12900F08980C62962D085
:10C1D000C72974D0C82900F09680DC2900F09B8024
:10C1E000E32970D0F8293AD0F92908D070477D2189
:10C1F000A0F860107047FD21A0F860107047602122
:10C20000A0F860107047E021A0F8601070473E2150
:10C21000A0F860107047BE21A0F8601070477A2126
:10C22000A0F860107047FA21A0F8601070476321F1
:10C23000A0F860107047E321A0F8601070475B2100
:10C24000A0F860107047DB21A0F8601070475F21F4
:10C25000A0F860107047DF21A0F8601070477021CF
:10C26000A0F860107047F021A0F8601070477F219F
:10C27000A0F8601070477B21A0F860107047FB2188
:10C28000A0F8601070477721A0F8601070474F2128
:10C29000A0F8601070471D21A0F8601070476E2153
:10C2A000A0F8601070471F21A0F860107047172198
:10C2B000A0F8601070476721A0F8601070470D214A
:10C2C000A0F8601070474C21A0F86010704737212B
:10C2D000A0F8601070478021A0F8601070476D21B1
:10C2E000A0F8601070470621A0F8601070470E217A
:10C2F000A0F8601070470221A0F8601070474E212E
:10C30000A0F8601070477521A0F8601070476B218D
:10C31000A0F8601070474621A0F860107047000038
:10C320005A0A0020D49102087C9102080092020867
:10C3300070B5DFF8F04A5B49B4F89E00B1F84A13D3
:10C3400009B1010002D0022840F0AB80DFF8185C90
:10C35000402128461CF00EFA002800F0A280DFF8E9
:10C360000C0C0078B4F87060012840F08480062E30
:10C370000FD1DFF8FC1B0988B4F8820001290CBF3B
:10C3800000F07F0040F08000A4F88200B4F8821032
:10C3900066E0FFF7C3FEB4F88400B0F5A57F04BFE4
:10C3A000B4F8A400012857D1D4F8C400C0F3800029
:10C3B000002851D00020A4F86200DFF8B80B006814
:10C3C000C1074CBF04210121A4F862108207B4F810
:10C3D00062104CBF41F0400141F02001A4F862100E
:10C3E0000021A4F8641041074CBF04210121A4F8E6
:10C3F00064100207B4F864104CBF41F0400141F0F2
:10C400002001A4F864100021A4F86610C1064CBFF6
:10C4100004210121A4F866108206B4F866104CBF0E
:10C4200041F0400141F02001A4F866100021A4F879
:10C43000681041064CBF04210121A4F868100006D1
:10C44000B4F868104CBF41F0400041F02000A4F85F
:10C450006800FF20A4F86A0004EB4600B0F8601002
:10C4600028461CF07FF9B4F87000401CA4F8700056
:10C4700080B2072811E0052E0EBFB4F8821004EB3D
:10C480004600B0F8601028461CF06CF9B4F8700053
:10C49000401CA4F8700080B20628A4BF0020A4F8B5
:10C4A000700070BD3843002070B50D46DFF8C84AF3
:10C4B000E0B9012120461AF06DFA022120461AF057
:10C4C00069FA042120461AF065FA082120461AF07C
:10C4D00061FA102120461AF05DFA202120461AF058
:10C4E00059FA402120461AF055FACCE0012813D120
:10C4F000DFF8886A802130461AF04AFA4021304637
:10C500001AF048FA202130461AF044FA4FF48071AC
:10C5100030461AF03FFA40E0022813D1DFF85C6A97
:10C52000802130461AF036FA402130461AF030FAAF
:10C53000202130461AF02EFA4FF4807130461AF05E
:10C5400029FA2AE0032813D1DFF8306A8021304627
:10C550001AF020FA402130461AF01CFA2021304609
:10C560001AF016FA4FF4807130461AF013FA14E0FC
:10C57000042818D1DFF8046A802130461AF00AFA3C
:10C58000402130461AF006FA202130461AF002FA0D
:10C590004FF4807130461AF0FBF94FF400713046C9
:10C5A0001AF0F8F919E0052817D1DFF8D0698021D1
:10C5B00030461AF0EFF9402130461AF0EBF920210D
:10C5C00030461AF0E7F94FF4807130461AF0E2F97C
:10C5D0004FF4007130461AF0DBF9ED43E80704D55B
:10C5E000012120461AF0D4F903E0012120461AF077
:10C5F000D1F9A80704D5022120461AF0C9F903E0B1
:10C60000022120461AF0C6F9680704D50421204605
:10C610001AF0BEF903E0042120461AF0BBF92807FE
:10C6200004D5082120461AF0B3F903E0082120467A
:10C630001AF0B0F9E80604D5102120461AF0A8F93E
:10C6400003E0102120461AF0A5F9A80604D5202100
:10C6500020461AF09DF903E0202120461AF09AF9AD
:10C66000680604D5402120461AF092F903E04021E3
:10C6700020461AF08FF9280605D52046BDE87040FF
:10C6800080211AF085B92046BDE8704080211AF05B
:10C6900081B90000C40E0020C80E0020E86100200F
:10C6A000100F0020F0B5DFF87C47B4F8B20081B07D
:10C6B00001281EBFDFF8B4080078012824D1DFF874
:10C6C000B858012128461AF065F9022128461AF0C7
:10C6D00061F9042128461AF05DF9082128461AF06C
:10C6E00059F9102128461AF055F9202128461AF048
:10C6F00051F9402128461AF04DF9284601B0BDE80D
:10C70000F04080211AF046B9D4F8BC00C0B9B4F8A2
:10C7100062100120FFF7C8FED4F8C000401C0228B8
:10C72000C4F8C0000CD3B4F862100020FFF7BCFEC0
:10C73000D4F8BC00401CC4F8BC000020C4F8C00001
:10C74000D4F8BC00012818D1B4F864100220FFF717
:10C75000ABFED4F8C000401C0228C4F8C0000CD3C3
:10C76000B4F864100020FFF79FFED4F8BC00401C12
:10C77000C4F8BC000020C4F8C000D4F8BC000228F3
:10C7800018D1B4F866100320FFF78EFED4F8C0006D
:10C79000401C0228C4F8C0000CD3B4F86610002076
:10C7A000FFF782FED4F8BC00401CC4F8BC00002097
:10C7B000C4F8C000D4F8BC00032818D1B4F868103D
:10C7C0000420FFF771FED4F8C000401C0228C4F812
:10C7D000C0000CD3B4F868100020FFF765FED4F851
:10C7E000BC00401CC4F8BC000020C4F8C000D4F851
:10C7F000BC00042818D1B4F880100520FFF754FEBF
:10C80000D4F8C000401C0228C4F8C0000CD3B4F80F
:10C8100080100020FFF748FED4F8BC00401CC4F88C
:10C82000BC000020C4F8C000D4F8BC00DFF84857B2
:10C83000052867D14FF4007128461AF0A9F84FF483
:10C84000806128461AF0A4F8DFF830674FF4806161
:10C8500030461AF09FF84FF4006130461AF098F80D
:10C860004FF4805130461AF093F8D4F8C000401CC1
:10C870000228C4F8C00045D30020C4F8C0004FF41B
:10C88000806128461AF07DF880B9B4F89600401C03
:10C8900080B2042806D11121A4F890100121A4F837
:10C8A0008E1004E0052802DB052000E00020A4F83B
:10C8B00096004FF4007128461AF063F8B4F890100F
:10C8C00050B9B4F89800401C80B2042805D100206B
:10C8D0003321A4F8980004E00020A4F89800080090
:10C8E00005D0DFF89C06008808B9012001E000218E
:10C8F0000020A4F88E00A4F89010D4F8BC00401CCE
:10C90000C4F8BC00D4F8BC00062840F0A8804FF45E
:10C91000007128461AF03CF84FF4806128461AF05E
:10C9200037F8DFF858664FF4806130461AF030F877
:10C930004FF4006130461AF02DF84FF48051304624
:10C940001AF026F8D4F8C000401C0228C4F8C00031
:10C95000C0F085800020C4F8C0004FF480612846F4
:10C960001AF00FF898BBB4F89200401C80B204286B
:10C9700014BF1428772127D01E2829DB0D216F280A
:10C980000ADA0346B3FBF1F39BB201FB1301F9B9D9
:10C990007721A4F890101BE040F2051398420ADAC0
:10C9A0000346B3FBF1F39BB201FB130181B978217C
:10C9B000A4F890100CE00646B6FBF1F6B6B201FB07
:10C9C000160129B918467921A4F8901000E000203A
:10C9D000A4F892004FF40071284619F0D2FFB4F881
:10C9E000902060BBB4F89400401C80B2042818BFAB
:10C9F00014280BD01E2823DB0D216E2808DA0346ED
:10CA0000B3FBF1F39BB201FB1301C9B9662217E036
:10CA100040F20513984208DA0346B3FBF1F39BB2E8
:10CA200001FB130161B967220AE00746B7FBF1F782
:10CA3000BFB201FB170119B91846682200E00020B7
:10CA4000A4F89400A4F89020B4F8900010B101204C
:10CA5000A4F88E00D4F8BC00401CC4F8BC00D4F884
:10CA6000BC00072867D14FF40071284619F090FFE9
:10CA70004FF48061284619F08BFFDFF800654FF412
:10CA80008061304619F084FF4FF40061304619F0A0
:10CA90007FFF4FF48051304619F07CFFD4F8C0007E
:10CAA000401C0228C4F8C00045D30020C4F8C000D0
:10CAB0004FF48061284619F064FF80B9B4F89A00F9
:10CAC000401C80B2042806D12221A4F89010012134
:10CAD000A4F88E1004E0052802DB052000E0002009
:10CAE000A4F89A004FF40071284619F04AFF90B953
:10CAF000B4F89C00401C80B2042805D14421A4F85D
:10CB00009010A4F89C000EE0052807DB0121052009
:10CB1000A4F8AC1002E00020A4F8AC00A4F89C003B
:10CB2000B4F8900010B10120A4F88E00D4F8BC0035
:10CB3000401CC4F8BC00D4F8BC00082804D3002072
:10CB4000C4F8BC00C4F8C000DFF8240D008818B990
:10CB5000A4F89000A4F88E0001B0F0BD30B5DFF865
:10CB6000085481B0012128461BF004FE70B902214F
:10CB700028461BF0FFFD48B9042128461BF0FAFDAA
:10CB800020B9082128461BF0F5FD38B128461BF0D6
:10CB9000EDFDDFF8CC1900F0FF000860DFF8C409F4
:10CBA000A04CB0F84A0388B1B4F89E0070B92021B7
:10CBB00028461BF0DFFD48B128461BF0D7FD00F0EA
:10CBC000FF00A4F890000120A4F88E00DFF8982957
:10CBD0001288B4F89000142A014609DBDFF88C298A
:10CBE000128852B1B4F88E20012A06D1442917D0F8
:10CBF0000022A4F88E20A4F8A220572918BF582993
:10CC00000ED1A4F8A2000020DFF8682CA4F8900050
:10CC1000A4F88E005729107000F0028100F004F98A
:10CC2000B4F88E00DFF84859012845D10020A4F857
:10CC30008C00A4F88A00A4F88E000021B4F89000BB
:10CC4000A4F89010A4F8A200332812BF4428B4F826
:10CC5000A4100C290ED1DFF8202C00211160DFF880
:10CC60001C2C116821F004011160DFF8141C0988E4
:10CC7000A4F8A410672818BF682803D0782818BF24
:10CC8000792807D12868C0F3001018B1B4F8A400BF
:10CC90000C2801D000F0C8F8DFF8E81B002008607D
:10CCA000DFF8D80B0068C0F38000002840F09A80BD
:10CCB000DFF8C41B086095E0B4F8A200672818BF2D
:10CCC000682803D0782818BF792814D12868C0F3C1
:10CCD000001080B1B4F8A4000C280CD1DFF8A81B18
:10CCE000DFF8A00B0978C90702D50168491C01606B
:10CCF00000680B2805D30020DFF8881BA4F8A200E9
:10CD00000860DFF8740BB4F8A42001680C2A1CD169
:10CD1000DFF8742B1278D20748BF491C332905D39A
:10CD2000DFF8582B136843F0040313603C2913D336
:10CD3000DFF8482B136823F0040313600021DFF8A9
:10CD4000402B1288A4F8A42006E0DFF8302B1368EB
:10CD500023F00403002113600160B4F88A00401C32
:10CD600080B2C9280BDBDFF8241B0A680020C2F35D
:10CD7000403222B10B68022262F34E330B60A4F8FA
:10CD80008A00B4F88C00401CA4F88C0080B2B0F586
:10CD90007A7F27DD0020A4F88C002868C0F30010FB
:10CDA000002804BFB4F8A4100C2904D1DFF8D01A6D
:10CDB0000988A4F8A410B4F8A410012908D1D4F863
:10CDC000C420C2F380031BB142F48072C4F8C420B3
:10CDD000002808BF002905D1D4F8C40040F4007031
:10CDE000C4F8C400B4F8A200672818BF682803D0AC
:10CDF000782818BF79280ED12868C0F3001050B1E8
:10CE0000B4F8A4000C2806D1DFF87C0A0078C0072B
:10CE100048BF00F009F801B0BDE83040FEF706BB9E
:10CE200001B030BD80200020DFF8380730B5B0F801
:10CE3000D410544C062981B00DD15149098851B103
:10CE4000B4F8A210442915D0D4F8C810C1F3801149
:10CE5000002900F08780B4F8A210582918BF57297C
:10CE600008D14249012008700020DFF8081A087034
:10CE700001B030BDDFF8183A00224FF49671A4F8E3
:10CE8000A8101A800121DFF80C3A1A70DFF8083A6E
:10CE90001A70B0F80C0500B90021DFF8000A018013
:10CEA000DFF8FC190A80B4F8A200112808BF03F0CB
:10CEB00047F8B4F8A200222808BF03F071F9B4F8CB
:10CEC000A200332804D10020A4F88A0004F0A2FCB8
:10CED000B4F8A200442808BF04F02EFDB4F8A25014
:10CEE000452D03BF01200021A4F8AE100020A4F8B6
:10CEF000B000662D08BF05F08DF9672D08BF05F05D
:10CF000089F9682D08BF05F085F9772D08BF04F071
:10CF10001FFE782D08BF04F01BFE792D08BF04F01A
:10CF200017FE882D08BF06F0D1FBB4F8A200BB287D
:10CF300001BFDFF870190968C1F3400100290AD167
:10CF4000DFF8642901211180DFF860190A88531E77
:10CF50009B41DB0F0B80CC2804D101B0BDE83040F1
:10CF600006F02EBC01B030BD00380140580A002048
:10CF7000DC6400204062002000140140000C0140ED
:10CF8000860A002080200020F0B581B0044606F01B
:10CF90008FFC2046DFF81859002600F0EBFADFF886
:10CFA000D0050068B5F8A420DFF8B815C0F300106C
:10CFB000002800F0A081B5F8A8304FF48370084431
:10CFC000002B04BFB0F8C630012B1AD10F2A18D09D
:10CFD000D5F8C460022363F3420640F63403A5F893
:10CFE0008430C5F8C4600122B0F8623FA5F8723001
:10CFF00090F8B23F03F00F03072B0AD1A5F87E206B
:10D0000007E0130003D1DFF8AC180E68C4E0012A72
:10D010005ED1D5F8C430C3F340064EB1B5F8847084
:10D0200040F634018F423E4650DB7E1C0221B4E0C4
:10D03000C3F38003002B3ED0B5F884703B46B3F5B4
:10D04000577F08BFB0F8B26514D040F24B16B34218
:10D0500008BFB0F890610DD0B3F5A67F08BFB0F857
:10D06000926107D040F24D16B3420CBFB0F8946104
:10D07000B5F87260A7F63407282F1AD201EB4307E0
:10D08000B7F850705FEA076C44BF31F81310A5F889
:10D09000721007F00F010F290BD0F90609D5B5F86A
:10D0A0007210B1F57A7FAEBFA1F2E73640F2E733F6
:10D0B0005E1A032171E00221C5F8C410D5F8C8102A
:10D0C000B5F8846041F00401C5F8C810022164E09D
:10D0D000022A03D169886E8C891C5EE0032A03D181
:10D0E000A988AE8C891C58E0042A03D1E988EE8C0B
:10D0F000891C52E0052A03D129892E8D891C4CE018
:10D10000062A03D169896E8D891C46E0072A03D15E
:10D11000A989AE8D891C40E0082A03D1E989EE8DEA
:10D12000891C3AE0092A03D1298A2E8E891C34E011
:10D130000A2A03D1698A6E8E891C2EE00B2A03D13C
:10D14000A98AAE8E891C28E00C2A15D1DFF8301789
:10D1500009888B1E082B0AD205EB410131F8021C0D
:10D16000022904D1DFF8301C0E68112115E0DFF828
:10D170002C1C0E68122110E00D2A08BF13210CD0C0
:10D180000E2A08BF142108D00F2A08BF152104D089
:10D19000DFF820170E6800220121DFF8043C196037
:10D1A0002100A5F8A4204CD00088B5F8A4100228CE
:10D1B00008BF022900F09D8000F00302032A40F01E
:10D1C0009380032900F09580002200F00703DFF828
:10D1D000D47B042B08BF02293A8000F0A3814207C8
:10D1E00008D50322104205D0032903D13A88012A29
:10D1F00040F0B281072B08BF042900F0938100F0B2
:10D200000F02082A08BF022900F08C8100070FD501
:10D21000012B1CBF022B042B02D1032900F08281B9
:10D22000032B1CBF052B062B02D1042900F07A81A9
:10D230000F2A08BF052900F075810020DFF8681B60
:10D240000880B5F8A400012805D0B5F8A40010B1F5
:10D250000020A5F874002146304600F02DFBDFF8D1
:10D260001406017822001AD0DFF81C261268C2F3D7
:10D2700040021AB1BD4A128802B9491CC9B20A2932
:10D280001CBFB5F89E20012A09D1DFF8203B002100
:10D290001970B5F87420042AA8BFA5F8741001709D
:10D2A000204601F0B5FAB5F85A00B5F85810B5F8AF
:10D2B0005620B5F85430B5F85260B5F85070A5F85E
:10D2C0006070002CA5F86260A5F86430A5F86620AF
:10D2D000A5F86810A5F86A0000F04081B5F85C0078
:10D2E000A5F86C0001B0F0BD022A08BF02297FF446
:10D2F0006BAF012269E7B5F8A800002801BF4FF421
:10D3000083700818B0F8C630012B1AD10F2A18D034
:10D31000D5F8C460022363F3420640F63403A5F84F
:10D320008430C5F8C4600122B0F8623FA5F87230BD
:10D3300090F8B20F00F00F0007280BD1A5F87E205F
:10D3400008E0100004D1DFF8540A06683220D5E066
:10D35000012A60D1D5F8C400C0F340034BB1B5F841
:10D36000847040F6340087423E4652DB7E1C3320F8
:10D37000C4E0C0F38000002840D0B5F884703B467C
:10D380004FF483700844B3F5577F08BFB0F8B26517
:10D3900014D040F24B16B34208BFB0F890610DD0E4
:10D3A000B3F5A67F08BFB0F8926107D040F24D16E2
:10D3B000B3420CBFB0F89461B5F87260A7F63400C0
:10D3C000282819D201EB4300B0F85000070644BFEB
:10D3D00031F81330A5F8723000F00F030F2B0BD08B
:10D3E000C00609D5B5F87200B0F57A7FAEBFA0F2DD
:10D3F000E73640F2E7331E1A34207FE00220C5F8FA
:10D40000C400D5F8C800B5F8846040F00400C5F841
:10D41000C800332072E0022A05D168886E8C022889
:10D420005DDA63206AE0032A05D1A888AE8C022861
:10D4300055DA632062E0042A05D1E888EE8C0228E0
:10D440004DDA63205AE0052A05D128892E8D02285D
:10D4500045DA632052E0062A05D168896E8D0228DC
:10D460003DDA63204AE0072A05D1A889AE8D02285B
:10D4700035DA632042E0082A05D1E889EE8D0228DA
:10D480002DDA63203AE0092A05D1288A2E8E022857
:10D4900025DA632032E00A2A06D1688A6E8E0228D5
:10D4A0001ADB288A343029E00B2A06D1A88AAE8EEE
:10D4B000022811DB688A343020E00C2A06D1E88A81
:10D4C000EE8E022808DBA88A343017E00D2A08D136
:10D4D000288B2E8F022801DA63200FE0E88A34308F
:10D4E0000CE00E2A08BF462008D00F2A08BF4720AC
:10D4F00004D0DFF8A808066832200022DFF8A03840
:10D5000018602000A5F8A4203FF49BAE4FF4837070
:10D510000844408800F00701042904BFB5F8A4209E
:10D52000022A04D1DFF88018012008808DE6420726
:10D5300006D50322104203D0B5F8A4000328F1D089
:10D54000072904BFB5F8A40004287FF476AEDFF8FD
:10D5500058180120088078E601206FE601B0F0BD80
:10D56000AC0E002038430020900A00206C200020E0
:10D570009C0E0020DFF818CCDFF8182CDCF800C077
:10D580000021CCF3001CBCF1000FDFF80C3C00F0D4
:10D59000B180B3F80601C30706D5DFF8003C1B686D
:10D5A000538401210223538083070AD5DFF8F03B1F
:10D5B0001B68491C02EB410CACF82030032322F815
:10D5C000113043070AD5DFF8DC3B1B88491C02EB0E
:10D5D000410CACF82030042322F8113003070AD59F
:10D5E000DFF8C43B1B68491C02EB410CACF820304F
:10D5F000052322F81130C3060AD5DFF8B03B1B889B
:10D60000491C02EB410CACF82030062322F8113003
:10D6100083060AD5DFF8983B1B88491C02EB410CB6
:10D62000ACF82030072322F8113043060AD5DFF882
:10D63000843B1B68491C02EB410CACF820300823EA
:10D6400022F8113003060AD5DFF86C3B1B68491C31
:10D6500002EB410CACF82030092322F81130C3054D
:10D660000AD5DFF8583B1B68491C02EB410CACF8AB
:10D6700020300A2322F8113083050AD5DFF8403B19
:10D680001B68491C02EB410CACF820300B2322F83C
:10D69000113043050AD5DFF82C3B1B68491C02EB0F
:10D6A000410CACF820300C2322F8113003050AD5C8
:10D6B000DFF8143B1B68491C02EB410CACF820302E
:10D6C0000D2322F8113010F480500ED0DFF8FC3A10
:10D6D0001B6803EB830C491C4FEA4C0302EB410C23
:10D6E000ACF820300E2322F811300A29C0F2B6809F
:10D6F0000923B4E038B1B3F808015FEAC07C0AD569
:10D70000401EA3F8080193F80801C00703D50121C2
:10D71000002050845180B3F8080183070AD5DFF850
:10D7200078361B68491C02EB410CACF82030022310
:10D7300022F8113043070AD5DFF86C3A1B68491C00
:10D7400002EB410CACF82030052322F8113003071E
:10D750000AD5DFF8583A1B88491C02EB410CACF89B
:10D760002030062322F81130C3060AD5DFF8403AEC
:10D770001B88491C02EB410CACF82030072322F82F
:10D78000113083060AD5DFF82C3A1B68491C02EBDE
:10D79000410CACF82030082322F8113043060AD59A
:10D7A000DFF8183A1B68491C02EB410CACF820303A
:10D7B0000A2322F8113003060AD5DFF8043A1B6861
:10D7C000491C02EB410CACF820300B2322F811303D
:10D7D000C3050AD5DFF8EC391B68491C02EB410C84
:10D7E000ACF820300C2322F81130830510D5DFF877
:10D7F00074CCDCF800C0491C02EB4103BCF1000F03
:10D8000048BFCCF1000CA3F820C00E2322F8113041
:10D81000430508D5491C02EB410C0023ACF820302D
:10D82000032322F81130030508D5491C02EB410CF3
:10D830000023ACF82030032322F8113010F480507C
:10D8400008D0491C02EB410C0023ACF82030032324
:10D8500022F811300829A8BF072300DA0B46A2F8E6
:10D86000A030DFF8042C1060DFF8000C0160704776
:10D870008E0A00202E650020B4630020140F0020C3
:10D88000980A0020C0630020EC0E0020980E0020B3
:10D89000E2640020E6640020E4640020DE640020EE
:10D8A000E0640020A00E0020F4640020F264002058
:10D8B00080200020B80E00202DE9F0470D4680465C
:10D8C000284600F0DBFDDFF8CC98DFF8D404002612
:10D8D000A9F8A6600068052818BF37280BD00828CB
:10D8E00018BF3A2807D03E2818BF0C2803D00728B5
:10D8F00018BF39284ED1290025D042F21071884531
:10D90000C0F29180B9F8A620521C0A23A9F8A620DB
:10D9100098FBF3F88845A1BF521CA9F8A62098FBF4
:10D92000F3F88845C0F27F80521CA9F8A62098FB26
:10D93000F3F88845A1BF521CA9F8A62098FBF3F87C
:10D940008845DFDA6FE0B8F57A7F6CDBB9F8A610AE
:10D95000491C0A22A9F8A61098FBF2F8B8F57A7FBC
:10D96000A1BF491CA9F8A61098FBF2F8B8F57A7F78
:10D9700059DB98FBF2F8491CB8F57A7FA9F8A61094
:10D9800051DB98FBF2F8491CB8F57A7FA9F8A6108C
:10D99000DCDA48E0290023D0DFF8D41A884542DBDE
:10D9A000B9F8A620521C0A23A9F8A62098FBF3F880
:10D9B0008845A1BF521CA9F8A62098FBF3F888451A
:10D9C00031DB521CA9F8A62098FBF3F88845A1BFCB
:10D9D000521CA9F8A62098FBF3F88845E0DA22E06B
:10D9E00042F2107188451EDBB9F8A620521C0A23AA
:10D9F000A9F8A62098FBF3F88845A1BF521CA9F806
:10DA0000A62098FBF3F888450DDB521CA9F8A62048
:10DA100098FBF3F88845A1BF521CA9F8A62098FBF3
:10DA2000F3F88845E0DA012801D102261AE012282D
:10DA300018BF3228F9D0052818BF3728F5D00E288E
:10DA400018BF4028F1D0102801D101260AE0422851
:10DA500018BF0F28F9D0032812BF342899F87E0088
:10DA600000F00306DFF82807DFF8084A0068C0F373
:10DA70000010002804BFB9F8A400002840F0D680A8
:10DA8000D9F8C47007F40470B0F5047F7CD1DFF8D6
:10DA90000807B0F896110A0018BF05290AD1B0F896
:10DAA0009E11022901BFDFF8D0190968C1F34011A6
:10DAB000002915D1B0F8981100294ED1B0F89E0177
:10DAC00001281CBF052806280AD0022818BF0328F1
:10DAD00001BFDFF8A4090068C0F3401000283CD162
:10DAE000B9F8740001000AD1FF212A00A9F85210E8
:10DAF000A9F85410A9F8561018BFA9F85810012811
:10DB00000BD1FF212800A9F85210A9F8541038D0E1
:10DB1000A9F85610A9F85A104FE0022807D1FF21A2
:10DB20002800A9F852102AD0A9F8541010E00328B0
:10DB300005D1FF21280020D0A9F8521006E00428C2
:10DB40003BD1280039D0FF21A9F85410A9F856106C
:10DB5000A9F85810A9F85A102FE028000AD0FF2180
:10DB6000A9F85210A9F85410A9F85610A9F858109D
:10DB7000A9F85A10FF21A9F85210A9F85410A9F8D1
:10DB80005610A9F8581018E0B9F8A60009EB400A99
:10DB900028003146404608D000F00AF99AF85600AD
:10DBA00000F07F00AAF8560007E000F011FB9AF899
:10DBB000540000F07F00AAF85400DFF81C0C006845
:10DBC000C0F3401018B187F01000C9F8C400002D50
:10DBD000278800F0DD80D9F8C400C0F34000002899
:10DBE00000F0C280D9F8C800C0F34010002840F00F
:10DBF000B880B9F8A4000027010000F0C980DFF860
:10DC0000D82BDFF8D81B1268C2F340121AB10A8869
:10DC100082F001020A800988002940F0B480314670
:10DC2000404600F0C5F82780BDE8F087B9F8A400A9
:10DC3000012802BFD9F8C47007F48270B0F5827F62
:10DC40006DD1DFF8940B0068C0F3401018B187F075
:10DC50002000C9F8C400B9F88400B0F5577F1CBF94
:10DC600040F24B1290426FD0B0F5A67F1CBF40F23D
:10DC70004D12904268D0B0F5637F1EBFD9F8C42022
:10DC8000C2F34012002A5FD0DFF80C2502EB4001FE
:10DC900091F85010090603D5A0F63400282853D374
:10DCA000B9F87400290021D0010004BFFF21A9F8B0
:10DCB0005A10012804D1FF20A9F8580027888AE7C4
:10DCC000022804D1FF20A9F85600278883E70328FB
:10DCD00003D1FF20A9F8540079E7042801D0278850
:10DCE00079E7FF20A9F85200278874E7010004BFF4
:10DCF000FF21A9F85810012806D1FF20A9F85600E5
:10DD000027882780BDE8F0870228E2D0032804BFD7
:10DD1000FF20A9F8520027882780BDE8F087DFF8A8
:10DD2000C00A0068C0F3800070B12788FF21002D71
:10DD3000A9F85210A9F85410A9F85610A9F85810CB
:10DD400026D0A9F85A1046E72788002D31464046CC
:10DD500002D000F02DF83EE700F03AFA2780BDE847
:10DD6000F087B9F8A40018B900272780BDE8F0872C
:10DD7000DFF8640A0068C0F3401048B187F001077B
:10DD80002780BDE8F087012804BFFF20A9F85A00CA
:10DD90002780BDE8F0870000D8620020D00E002068
:10DDA000D0630020EA640020F0640020580A0020BC
:10DDB000F0B4DFF8E023DFF82C4AB2F8803042F20A
:10DDC0001075A84231DB294690FBF1F105FB1100EB
:10DDD0004FF47A7590FBF5F605FB1600642590FB71
:10DDE000F5F5642707FB15005527A2F8507034F8A5
:10DDF0001110A2F8521034F81610A2F8541034F88A
:10DE00001510A2F856100A2190FBF1F134F81150C8
:10DE1000A2F8585001EB8105A0EB450034F8100042
:10DE2000A2F85A00A2F85C3094E1FF26B0F57A7FA0
:10DE300032DB4FF47A7190FBF1F14FF47A7505FB08
:10DE40001100642590FBF5F5642707FB15005527A5
:10DE5000A2F85070A2F8526034F81110A2F85410D1
:10DE600034F81510A2F856100A2190FBF1F134F89D
:10DE70001150A2F8585001EB8105A0EB450034F891
:10DE80001000A2F85A00A2F85C30B2F8740004281E
:10DE900040F06081C0205BE1B2F8A450642862DBEE
:10DEA000642790FBF7F74FF0640C0CFB17004FF062
:10DEB000550CA2F85260A2F85460A2F850C034F891
:10DEC0001760A2F856600A2690FBF6F634F8167032
:10DED000A2F85870032906EB8607A0EB470034F838
:10DEE0001000A2F85A00A2F85C3004BFC020A2F8CB
:10DEF0005400012D0BD1D2F8C410C1F3800131B10F
:10DF0000B2F87410032904BFC021A2F85410DFF83E
:10DF1000D8180968C1F3001139B92B0001BFB2F854
:10DF20007430032BC023A2F85430012D0DD1D2F848
:10DF3000C400C0F3800040B1B2F87400042804D1DA
:10DF4000C020A2F85200A2F85400002902BF002D00
:10DF5000B2F87400042840F0FD80C020A2F85200FE
:10DF6000A2F85400F6E00A286FDBA2F85260A2F88B
:10DF70005460A2F856605527A2F850700A2690FB0C
:10DF8000F6F634F81670A2F85870022906EB8607E8
:10DF9000A0EB470034F81000A2F85A00A2F85C3059
:10DFA00008BFC02004D0032904D1C020A2F8540027
:10DFB000A2F85600012D11D1D2F8C410C1F380018E
:10DFC00061B1B2F87430022B08BFC02104D0032B1A
:10DFD00004D1C021A2F85410A2F85610DFF8081896
:10DFE0000968C1F3001171B92B000CD1B2F874307B
:10DFF000022B08BFC02304D0032B04D1C023A2F8F6
:10E000005430A2F85630012D0FD1D2F8C400C0F31D
:10E01000800050B1B2F87400042806D1C020A2F8E4
:10E020005200A2F85400A2F85600002902BF002DA9
:10E03000B2F87400042840F08D80C020A2F852008D
:10E04000A2F85400A2F8560084E05527A2F85070B8
:10E05000A2F85260A2F85460A2F85660A2F8586084
:10E06000012934F81000A2F85A00A2F85C3008BF69
:10E07000C02004D0022905D1C020A2F85600A2F881
:10E08000580008E0032906D1C020A2F85800A2F8E1
:10E090005400A2F85600012D1BD1D2F8C410C1F3D0
:10E0A0008001B1B1B2F87430012B03D1C021A2F8C4
:10E0B00058100EE0022B03D1C021A2F8581006E040
:10E0C000032B06D1C021A2F85810A2F85410A2F8D0
:10E0D0005610DFF814170968C1F30011B1B92B000D
:10E0E00014D1B2F87430012B08BFC0230CD0022B1E
:10E0F00003D1C023A2F8583006E0032B06D1C02379
:10E10000A2F85830A2F85430A2F85630012D11D19F
:10E11000D2F8C400C0F3800060B1B2F874000428E3
:10E1200008D1C020A2F85800A2F85400A2F8560066
:10E13000A2F85200002902BF002DB2F87400042892
:10E1400008D1C020A2F85800A2F85400A2F8560046
:10E15000A2F85200D2F8C400C0F34000B0B1B2F847
:10E1600084000A2809DAB2F8A400012807D1C020E7
:10E17000A2F85400A2F8580005E0642806DAB2F8C4
:10E18000A400012802D1C020A2F85400F0BC7047BE
:10E190009C0E00208020002038430020D462002004
:10E1A000805F0020920A002094120020F45D00207D
:10E1B00088120020B4620020DC6200200C5E002087
:10E1C000C8620020C0620020785F0020680F002035
:10E1D000F0B4DFF81826DFF80C46B2F88030B0F55E
:10E1E0007A7F2ADB4FF47A7190FBF1F14FF47A7564
:10E1F00005FB1100642590FBF5F5642606FB150070
:10E200005526A2F8506034F81110A2F8521034F8D4
:10E210001510A2F854100A2190FBF1F134F81150B6
:10E22000A2F8565001EB8105A0EB450034F8100030
:10E23000A2F85800A2F85A30F6E0FF25642845DB22
:10E24000642690FBF6F6642707FB16005527A2F814
:10E250005250A2F8507034F81650A2F854500A25C3
:10E2600090FBF5F534F81560A2F85660032905EB2C
:10E270008506A0EB460034F81000A2F85800A2F87A
:10E280005A3004BFC020A2F85200B2F8A4000128FE
:10E290000BD1D2F8C410C1F3800131B1B2F87410BF
:10E2A000032904BFC021A2F85210DFF83C15096809
:10E2B000C1F30011002902BF0028B2F8740003283E
:10E2C00040F0B280C020A2F85200ADE00A284FDB37
:10E2D000A2F85250A2F854505526A2F850600A25D0
:10E2E00090FBF5F534F81560A2F85660022905EBAD
:10E2F0008506A0EB460034F81000A2F85800A2F8FA
:10E300005A3008BFC02004D0032904D1C020A2F88D
:10E310005200A2F85400B2F8A400012811D1D2F89A
:10E32000C410C1F3800161B1B2F87410022908BFB2
:10E33000C02104D0032904D1C021A2F85210A2F8B0
:10E340005410DFF8A4140968C1F30011002908BFB4
:10E35000002869D1B2F87410022908BFC02004D087
:10E36000032961D1C020A2F85200A2F854005BE05A
:10E370005526A2F85060A2F85250A2F85450A2F8C4
:10E380005650012934F81000A2F85800A2F85A306B
:10E3900008BFC0200ED0022905D1C020A2F8560027
:10E3A000A2F8540008E0032906D1C020A2F85200C8
:10E3B000A2F85400A2F85600B2F8A400012817D120
:10E3C000D2F8C410C1F3800191B1B2F874100129E0
:10E3D00008BFC0210AD0022908BFC02104D00329E8
:10E3E00006D1C021A2F85210A2F85410A2F856107B
:10E3F000DFF8F4130968C1F30011002908BF0028F1
:10E4000012D1B2F87410012908BFC0200AD0022925
:10E4100008BFC02004D0032906D1C020A2F85200B2
:10E42000A2F85400A2F85600D2F8C400C0F340008D
:10E43000B0B1B2F884000A2809DAB2F8A4000128C1
:10E4400007D1C020A2F85400A2F8560005E06428C5
:10E4500006DAB2F8A400012802D1C020A2F85400C4
:10E46000F0BC7047B45F0020AC0E0020F8620020C2
:10E47000A0860100EC640020F40E002070B4DFF8E8
:10E480007043DFF868132468B1F8B420B1F8B630EF
:10E490000028C4F3400400F0BB80ACB1521C92B21F
:10E4A000FA2A07DBB1F8820040F002000022A1F84E
:10E4B000820010E07E2A0EDBB1F882004FF6FD7577
:10E4C0002840A1F8820006E0B1F8820040F0020086
:10E4D000A1F882000022C748B0F89051032D18BF60
:10E4E000042D05D0B0F89201032818BF042818D1D4
:10E4F00018001EBF5B1E98B2002806D1B1F882003A
:10E500004FF6F7752840A1F88200BB480088012823
:10E510000DD1B1F8820040F00800A1F8820032234A
:10E5200005E0B1F8820040F00800A1F88200AE4892
:10E530000068C0F300100028B1F8820015D040F048
:10E540001000AE4CA1F8820024682CB94FF6FB7481
:10E55000204040F0200036E1012C40F036814FF69B
:10E56000DF74204040F004002DE14FF6EF752840A5
:10E57000994DA1F882002D68C5F340052DB1D1F861
:10E58000C45085F08005C1F8C4509D4D2E68D1F867
:10E59000C450C5F3C01576B94FF6FB763040A1F8EC
:10E5A00082001DB140F00400A1F88200B1F88200A1
:10E5B00040F0200017E0012E0ED14FF6DF763040FC
:10E5C000A1F882001DB140F02000A1F88200B1F84E
:10E5D000820040F0040006E040F02400A1F8820030
:10E5E0001DB140F01000A1F882008648007810F0BC
:10E5F000850F01BF7A480068C0F30010002800F0C2
:10E60000E480002C40F0E180002D00F0DE80D6E0B8
:10E610005CB1B1F8800040F09000A1F88000B1F842
:10E62000820040F00A00A1F882006F4D76482D6804
:10E63000C5F30015002D46D0704C246804604FF6D9
:10E640007F75B1F880402C40A1F880404FF6F775F7
:10E65000B1F882402C40A1F88240B1F8A4402500D6
:10E660006DD00C2C0CD1694C2488250067D0A51ED8
:10E67000082D05D201EB440434F8024C022C5ED183
:10E68000B1F8804044F01004A1F88040B1F8824015
:10E6900044F00204A1F88240D1F8C440C4F340051C
:10E6A000002D1EBFD1F8C850C5F34015002D53D022
:10E6B000B1F8805045F02005A1F88050B1F88250A3
:10E6C00045F0040554E04E4D2D6805604D4D2D7804
:10E6D00015F0850F01BF424D2D68C5F30015002DC3
:10E6E0001DD0E4B93C4C2468C4F340042CB1D1F8EB
:10E6F000C44084F40064C1F8C440D1F8C440C4F3F9
:10E70000C02464B1B1F880404FF67F752C40A1F869
:10E7100080404FF6F775B1F882402C4009E0B1F81F
:10E72000804044F08004A1F88040B1F8824044F079
:10E730000804A1F88240B1F8A440002CA0D1B1F89F
:10E7400080404FF6EF752C40A1F880404FF6FD75E4
:10E75000B1F882402C409DE7B1F880504FF6DF764B
:10E760003540A1F880504FF6FB76B1F88250354025
:10E77000A1F88250006878B101281AD016480068C4
:10E78000C0F3400018B184F08000C1F8C400D1F893
:10E79000C400C0F3C01060B1B1F880004FF6BF7480
:10E7A0002040A1F880004FF6EF74B1F882002040BD
:10E7B00009E0B1F8800040F04000A1F88000B1F815
:10E7C000820040F01000A1F88200A1F8B630A1F854
:10E7D000B42070BC70470000EC0E0020EE640020F6
:10E7E000140F0020882F01089C0E0020802000209C
:10E7F000A00E00203843002056200020E00E00200C
:10E80000DC0E0020980E0020AC0E0020980A00209C
:10E81000DFF8801C30B50968DFF87C4CC1F30011CB
:10E820000029B4F8A41081B000F083860A0000F03B
:10E830008C86012900F08186022940F0A482658837
:10E84000002800F05981012D22D15520A4F8500054
:10E850008920A4F852008E20A4F85400BF20A4F808
:10E860005600C020A4F85800B4F88000A4F85A005C
:10E870000020DFF8281E042D088000F03781052DC8
:10E8800000F03481DFF8181E0020088001B030BD90
:10E89000022D00F0DD80032D0CD18820A4F8520059
:10E8A000B4F8A6000228C0F2A980DFF8F01D01200C
:10E8B0000880E4E7042D06D1C120A4F852006D20A1
:10E8C000A4F85200D4E7052D0DD1E320A4F852009E
:10E8D000B4F8A6000128CBD194F85A0000F07F00CC
:10E8E000A4F85A00FDE0062D1DD1B4F8A60060B1D1
:10E8F0008320A4F852000020DFF8A01D088000202B
:10E90000DFF89C1D088001B030BDB4F85800FF2826
:10E9100004BFC020A4F8580094F8580000F07F000D
:10E92000A4F85800E4E7072D03D18920A4F8520089
:10E930009EE7082D00F08C80092D02D104F06BFBBE
:10E9400096E70A2D13D1B4F8A60008B14E20D0E7FF
:10E95000B4F85800FF2804BFC020A4F8580094F869
:10E96000580000F07F00A4F858004E20C1E70B2D9E
:10E9700042D1DFF8300D0068012818BF052824D0E7
:10E98000022815D15520A4F850008320A4F8520085
:10E99000AF20A4F85400F920A4F85600FF20A4F8F2
:10E9A0005800A4F85A00B4F88000A4F85C005FE7AF
:10E9B00003284DD15520A4F850008320A4F852001C
:10E9C000AF20A4F85400A420E6E75520A4F8500096
:10E9D000A320A4F85200E320A4F854008620A4F851
:10E9E00056000620A4F85800FF20A4F85A00B4F8F6
:10E9F0008000A4F85C003BE70C2D0AD1B4F8A60017
:10EA000004EB400090F8561001F07F01A0F856107A
:10EA100067E00D2D12D1B4F8A60000287FF46BAF8B
:10EA2000B4F85800FF280CD1C020A4F8580094F87E
:10EA3000580000F07F00A4F8580019E70E2D7FF46D
:10EA400017AF94F8580000F07F00A4F858000FE7C3
:10EA5000B4F8A600012806D194F85A0000F07F000F
:10EA6000A4F85A003DE002280CD194F85A0000F0B6
:10EA70007F00A4F85A0094F8580000F07F00A4F832
:10EA800058002EE0032812D194F85A0000F07F00BD
:10EA9000A4F85A0094F8580000F07F00A4F8580039
:10EAA00094F8560000F07F00A4F8560019E00428FE
:10EAB00017D194F85A0000F07F00A4F85A0094F897
:10EAC000580000F07F00A4F8580094F8560000F0B9
:10EAD0007F00A4F8560094F8540000F07F00A4F8DA
:10EAE0005400032D7FF4C4AE012005E7DFF8B01B0E
:10EAF0000120088001B030BD012D14D15520A4F8AB
:10EB0000500001B08920A4F852008E20A4F85400CF
:10EB1000BF20A4F85600C020A4F85800B4F8800024
:10EB2000A4F85A0030BD022D00F0DE80032D08D17C
:10EB30008820A4F85200B4F8A600022880F2AC8520
:10EB4000A5E0042D04D1C120A4F8520001B030BDCD
:10EB5000052D0FD1E320A4F85200B4F8A600012837
:10EB600040F09A8594F8580000F07F00A4F858000F
:10EB700001B030BD062D14D1B4F8A60060B9B4F8C8
:10EB80005600FF2804BFC020A4F8560094F8560091
:10EB900000F07F00A4F856008320A4F8520001B0D2
:10EBA00030BD072D04D18920A4F8520001B030BD3A
:10EBB000082D00F09980092D04D101B0BDE8304046
:10EBC00004F029BA0A2D14D1B4F8A60060B9B4F83B
:10EBD0005600FF2804BFC020A4F8560094F8560041
:10EBE00000F07F00A4F85600A320A4F8520001B062
:10EBF00030BD0B2D49D1DFF8AC0A0068012818BFE1
:10EC000005282DD0022814D15520A4F8500001B0B9
:10EC10008320A4F85200AF20A4F85400F920A4F8EF
:10EC20005600FF20A4F85800B4F88000A4F85A0059
:10EC300030BD032858D15520A4F8500001B08320DE
:10EC4000A4F85200AF20A4F85400A420A4F8560061
:10EC5000FF20A4F85800B4F88000A4F85A0030BD92
:10EC60005520A4F8500001B0A320A4F85200E320DE
:10EC7000A4F854008620A4F85600AF20A4F8580049
:10EC8000B4F88000A4F85A0030BD0C2D0BD1B4F8B4
:10EC9000A60004EB400090F8541001F07F01A0F8AA
:10ECA000541001B030BD0D2D13D1B4F8A6000028CA
:10ECB00040F0F284B4F85600FF2829D1C020A4F80F
:10ECC000560001B094F8560000F07F00A4F85600FA
:10ECD00030BD0E2D40F0E08494F8560000F07F0027
:10ECE000A4F8560001B030BDB4F8A600012807D141
:10ECF00094F8580000F07F00A4F8580001B030BD2F
:10ED000002280DD194F8580000F07F00A4F85800B4
:10ED100001B094F8560000F07F00A4F8560030BD12
:10ED2000032813D194F8580000F07F00A4F858008D
:10ED300001B094F8560000F07F00A4F8560094F853
:10ED4000540000F07F00A4F8540030BD042840F0C7
:10ED5000A38494F8580000F07F00A4F8580001B094
:10ED600094F8560000F07F00A4F8560094F8540080
:10ED700000F07F00A4F8540094F8520000F07F00E7
:10ED8000A4F8520030BD03295DD1A588B0B3012D90
:10ED90003FF45BAD022D3FF45BAE032D3FF47DAD40
:10EDA000042D3FF489AD052D3FF48FAD062D05D11F
:10EDB000B4F8A60000287FF49BADA6E5072D3FF42C
:10EDC000B4AD082D3FF444AE092D3FF4B7AD0A2D84
:10EDD00005D1B4F8A60000287FF4B8ADB8E50B2D36
:10EDE0003FF4C7AD0C2D3FF409AE0D2D7FF426AED8
:10EDF000B4F8A60000287FF47EAD11E6012D3FF4A3
:10EE00007DAE022D3FF470AF032D3FF491AE042D83
:10EE10003FF499AE052D3FF49DAE062D3FF4ACAE08
:10EE2000072D3FF4C0AE082D3FF45EAF092D3FF42F
:10EE3000C4AE0A2D3FF4C8AE0B2D3FF4DCAE0C2D52
:10EE40003FF425AF2FE704295DD1E588B0B3012D4C
:10EE50003FF4FBAC022D3FF4FBAD032D3FF41DADA1
:10EE6000042D3FF429AD052D3FF42FAD062D05D11E
:10EE7000B4F8A60000287FF43BAD46E5072D3FF42B
:10EE800054AD082D3FF4E4AD092D3FF457AD0A2DE4
:10EE900005D1B4F8A60000287FF458AD58E50B2D35
:10EEA0003FF467AD0C2D3FF4A9AD0D2D7FF4C6AD39
:10EEB000B4F8A60000287FF41EADB1E5012D3FF4A3
:10EEC0001DAE022D3FF410AF032D3FF431AE042DE3
:10EED0003FF439AE052D3FF43DAE062D3FF44CAE68
:10EEE000072D3FF460AE082D3FF4FEAE092D3FF430
:10EEF00064AE0A2D3FF468AE0B2D3FF47CAE0C2DB2
:10EF00003FF4C5AECFE605295DD12589B0B3012D0B
:10EF10003FF49BAC022D3FF49BAD032D3FF4BDAC01
:10EF2000042D3FF4C9AC052D3FF4CFAC062D05D11F
:10EF3000B4F8A60000287FF4DBACE6E4072D3FF42C
:10EF4000F4AC082D3FF484AD092D3FF4F7AC0A2D45
:10EF500005D1B4F8A60000287FF4F8ACF8E40B2D36
:10EF60003FF407AD0C2D3FF449AD0D2D7FF466AD98
:10EF7000B4F8A60000287FF4BEAC51E5012D3FF4A3
:10EF8000BDAD022D3FF4B0AE032D3FF4D1AD042D45
:10EF90003FF4D9AD052D3FF4DDAD062D3FF4ECADCA
:10EFA000072D3FF400AE082D3FF49EAE092D3FF42F
:10EFB00004AE0A2D3FF408AE0B2D3FF41CAE0C2D11
:10EFC0003FF465AE6FE606295DD16589B0B3012DCA
:10EFD0003FF43BAC022D3FF43BAD032D3FF45DAC61
:10EFE000042D3FF469AC052D3FF46FAC062D05D11F
:10EFF000B4F8A60000287FF47BAC86E4072D3FF42C
:10F0000094AC082D3FF424AD092D3FF497AC0A2DA4
:10F0100005D1B4F8A60000287FF498AC98E40B2D35
:10F020003FF4A7AC0C2D3FF4E9AC0D2D7FF406ADF9
:10F03000B4F8A60000287FF45EACF1E4012D3FF4A3
:10F040005DAD022D3FF450AE032D3FF471AD042DA4
:10F050003FF479AD052D3FF47DAD062D3FF48CAD29
:10F06000072D3FF4A0AD082D3FF43EAE092D3FF42F
:10F07000A4AD0A2D3FF4A8AD0B2D3FF4BCAD0C2D73
:10F080003FF405AE0FE607295DD1A589B0B3012D88
:10F090003FF4DBAB022D3FF4DBAC032D3FF4FDABC3
:10F0A000042D3FF409AC052D3FF40FAC062D05D11E
:10F0B000B4F8A60000287FF41BAC26E4072D3FF42B
:10F0C00034AC082D3FF4C4AC092D3FF437AC0A2D05
:10F0D00005D1B4F8A60000287FF438AC38E40B2D35
:10F0E0003FF447AC0C2D3FF489AC0D2D7FF4A6AC5A
:10F0F000B4F8A60000287FF4FEAB91E4012D3FF4A4
:10F10000FDAC022D3FF4F0AD032D3FF411AD042D05
:10F110003FF419AD052D3FF41DAD062D3FF42CAD88
:10F12000072D3FF440AD082D3FF4DEAD092D3FF42F
:10F1300044AD0A2D3FF448AD0B2D3FF45CAD0C2DD2
:10F140003FF4A5ADAFE508295FD1E589C0B3012D36
:10F150003FF47BAB022D3FF47BAC032D3FF49DAB22
:10F16000042D3FF4A9AB052D3FF4AFAB062D06D11E
:10F17000B4F8A60000287FF4BBABFFF7C6BB072D91
:10F180003FF4D3AB082D3FF463AC092D3FF4D6AB6D
:10F190000A2D06D1B4F8A60000287FF4D7ABFFF7FC
:10F1A000D7BB0B2D3FF4E5AB0C2D3FF427AC0D2D59
:10F1B0007FF444ACB4F8A60000287FF49CAB2FE4A5
:10F1C000012D3FF49BAC022D3FF48EAD032D3FF497
:10F1D000AFAC042D3FF4B7AC052D3FF4BBAC062D0E
:10F1E0003FF4CAAC072D3FF4DEAC082D3FF47CADF4
:10F1F000092D3FF4E2AC0A2D3FF4E6AC0B2D3FF4B1
:10F20000FAAC0C2D3FF443AD4DE5092960D1258AB8
:10F21000C8B3012D3FF419AB022D3FF419AC032DF7
:10F220003FF43BAB042D3FF447AB052D3FF44DAB12
:10F23000062D06D1B4F8A60000287FF459ABFFF7DD
:10F2400064BB072D3FF471AB082D3FF401AC092DD1
:10F250003FF474AB0A2D06D1B4F8A60000287FF461
:10F2600075ABFFF775BB0B2D3FF483AB0C2D3FF453
:10F27000C5AB0D2D7FF4E2ABB4F8A60000287FF4F7
:10F280003AABFFF7CDBB012D3FF438AC022D3FF474
:10F290002BAD032D3FF44CAC042D3FF454AC052DA5
:10F2A0003FF458AC062D3FF467AC072D3FF47BAC20
:10F2B000082D3FF419AD092D3FF47FAC0A2D3FF422
:10F2C00083AC0B2D3FF497AC0C2D3FF4E0ACEAE49B
:10F2D0000A2960D1658AC8B3012D3FF4B6AA022D70
:10F2E0003FF4B6AB032D3FF4D8AA042D3FF4E4AAB3
:10F2F000052D3FF4EAAA062D06D1B4F8A600002891
:10F300007FF4F6AAFFF701BB072D3FF40EAB082DE3
:10F310003FF49EAB092D3FF411AB0A2D06D1B4F892
:10F32000A60000287FF412ABFFF712BB0B2D3FF4B1
:10F3300020AB0C2D3FF462AB0D2D7FF47FABB4F806
:10F34000A60000287FF4D7AAFFF76ABB012D3FF47F
:10F35000D5AB022D3FF4C8AC032D3FF4E9AB042D2F
:10F360003FF4F1AB052D3FF4F5AB062D3FF404ACB3
:10F37000072D3FF418AC082D3FF4B6AC092D3FF42F
:10F380001CAC0A2D3FF420AC0B2D3FF434AC0C2DFB
:10F390003FF47DAC87E40B2960D1A58AC8B3012D69
:10F3A0003FF453AA022D3FF453AB032D3FF475AA4B
:10F3B000042D3FF481AA052D3FF487AA062D06D11E
:10F3C000B4F8A60000287FF493AAFFF79EBA072D91
:10F3D0003FF4ABAA082D3FF43BAB092D3FF4AEAA96
:10F3E0000A2D06D1B4F8A60000287FF4AFAAFFF7D3
:10F3F000AFBA0B2D3FF4BDAA0C2D3FF4FFAA0D2D83
:10F400007FF41CABB4F8A60000287FF474AAFFF7C1
:10F4100007BB012D3FF472AB022D3FF465AC032D09
:10F420003FF486AB042D3FF48EAB052D3FF492AB39
:10F43000062D3FF4A1AB072D3FF4B5AB082D3FF4EB
:10F4400053AC092D3FF4B9AB0A2D3FF4BDAB0B2DE6
:10F450003FF4D1AB0C2D3FF41AAC24E40C2962D15B
:10F46000DFF85C1C09888A1E082A6ED204EB410171
:10F4700031F8021C022968D100283FF435ACB4F8F9
:10F48000A60001280AD194F85A0000F07F00A4F8E1
:10F490005A0041E09C0E00208020002002280CD160
:10F4A00094F85A0000F07F00A4F85A0094F858002D
:10F4B00000F07F00A4F858002EE0032812D194F841
:10F4C0005A0000F07F00A4F85A0094F8580000F0A9
:10F4D0007F00A4F8580094F8560000F07F00A4F8CC
:10F4E000560019E0042817D194F85A0000F07F0064
:10F4F000A4F85A0094F8580000F07F00A4F85800CF
:10F5000094F8560000F07F00A4F8560094F85400D8
:10F5100000F07F00A4F8540000206049088001B08A
:10F520005F49088030BD0E2958D00F2900F0A68011
:10F53000A9E00A0009D0012924D1D4F8C410C1F3EC
:10F540004002A2B9C1F3800141B118B101B0BDE8D8
:10F5500030402EE301B0BDE8304092E30221C4F810
:10F56000C410D4F8C81041F00401C4F8C81020B188
:10F5700001B0BDE8304003F0D1BC01B0BDE830407F
:10F5800003F016BD022908BF65881AD0032908BFF9
:10F59000A58816D0042908BFE58812D0052908BF20
:10F5A00025890ED0062908BF65890AD0072908BF1A
:10F5B000A58906D0082908BFE58902D009290BD101
:10F5C000258A0028284603D001B0BDE830406BE012
:10F5D00001B0BDE83040D1E10E294DD1B4F8801022
:10F5E00030B35520A4F8500055227020A4F85200E2
:10F5F000A4F860201F207022A4F85400A4F8622010
:10F600005B201F22A4F85600A4F8642070205B221F
:10F61000A4F85800A4F86620FF207022A4F85A002D
:10F62000A4F86820A4F86A00A4F86C1001B030BDFA
:10F630005520A4F85000A4F85A10F820A4F852005D
:10F64000A4F86A108620A4F8540001B09220A4F80F
:10F650005600F820A4F858005520A4F86000F820BF
:10F66000A4F862008620A4F864009220A4F8660042
:10F67000F820A4F8680030BD0F2904D101B0BDE81E
:10F68000304003F02FBD10B100F093FA01E000F01C
:10F69000F8FA0020A4F8A40001B030BDEA6400200C
:10F6A000F0640020C462002000B5012881B0DFF8BA
:10F6B000D01A1CD15520A1F850008920A1F8520081
:10F6C0008E20A1F85400BF20A1F85600C020A1F858
:10F6D0005800B1F88000A1F85A000020DFF8A41A01
:10F6E00008800020DFF8A01A088001B000BD0228C1
:10F6F00000F0C480032809D18822A1F85220B1F873
:10F70000A620022AC0F217810120E7E704280FD1C2
:10F71000C120A1F8520001B06D20A1F852000020D4
:10F72000DFF8601A08800120DFF85C1A088000BD4D
:10F73000052811D1E322A1F85220B1F8A620012A10
:10F7400000F0A080DFF83C1A002008800120DFF8DC
:10F75000381A088001B000BD062817D1B1F8A600FC
:10F7600018B18320A1F85200B7E7B1F85800FF287C
:10F7700004BFC020A1F8580091F8580000F07F00A5
:10F78000A1F858008320A1F85200A6E7072803D16A
:10F790008920A1F85200A0E708286FD0092802D1DB
:10F7A00003F039FC99E70A2817D1B1F8A60018B17F
:10F7B0004E20A1F8520090E7B1F85800FF2804BF8E
:10F7C000C020A1F8580091F8580000F07F00A1F87F
:10F7D00058004E20A1F852007FE70B2840F0A98086
:10F7E000DFF8A8291268012A18BF052A16D155206A
:10F7F000A1F85000A320A1F85200E320A1F8540082
:10F800008620A1F856000620A1F85800FF20A1F894
:10F810005A00B1F88000A1F85C005EE7022A15D119
:10F820005520A1F850008320A1F85200AF20A1F884
:10F830005400F920A1F85600FF20A1F85800A1F8C3
:10F840005A00B1F88000A1F85C0046E7032A15D100
:10F850005520A1F850008320A1F85200AF20A1F854
:10F860005400A420A1F85600FF20A1F85800A1F8E8
:10F870005A00B1F88000A1F85C002EE7B1F8A6208C
:10F88000012A17D191F85A2002F07F02A1F85A20DC
:10F8900003283FF439AFDFF8EC280021042818BF13
:10F8A000052811807FF41DAFDFF8DC1801200880E7
:10F8B00001B000BD022A0CD191F85A2002F07F025B
:10F8C000A1F85A2091F8582002F07F02A1F85820A0
:10F8D000DEE7032A12D191F85A2002F07F02A1F844
:10F8E0005A2091F8582002F07F02A1F8582091F890
:10F8F000562002F07F02A1F85620C9E7042AC7D19A
:10F9000091F85A2002F07F02A1F85A2091F858206D
:10F9100002F07F02A1F8582091F8562002F07F02F1
:10F92000A1F8562091F8542002F07F02A1F854204B
:10F93000AEE70C280AD1B1F8A62001EB420191F8FC
:10F94000562002F07F02A1F85620A1E70D2812D11F
:10F95000B1F8A60000287FF4C0AEB1F85800FF2827
:10F9600004BFC020A1F8580091F8580000F07F00B3
:10F97000A1F85800B1E60E28F6D0AEE60128DFF86F
:10F98000001813D15520A1F850008920A1F8520089
:10F990008E20A1F85400BF20A1F85600C020A1F885
:10F9A0005800B1F88000A1F85A007047022800F012
:10F9B0009980032808D18820A1F85200B1F8A60048
:10F9C000022880F2F580D3E0042808BFC12000F0AF
:10F9D000CA8005280ED1E320A1F85200B1F8A60094
:10F9E000012840F0E58091F8580000F07F00A1F870
:10F9F00058007047062813D1B1F8A60060B9B1F8D5
:10FA00005600FF2804BFC020A1F8560091F8560008
:10FA100000F07F00A1F856008320A1F85200704743
:10FA2000072808BF892000F09E8008285AD009289E
:10FA300008BF03F0F0BA0A2813D1B1F8A60060B9E4
:10FA4000B1F85600FF2804BFC020A1F8560091F875
:10FA5000560000F07F00A1F85600A320A1F8520044
:10FA600070470B2840F08280DFF8200700680128EB
:10FA700018BF052813D15520A1F85000A320A1F8E4
:10FA80005200E320A1F854008620A1F85600AF20D0
:10FA9000A1F85800B1F88000A1F85A007047022878
:10FAA0000AD15520A1F850008320A1F85200AF20C0
:10FAB000A1F85400F9200BE0032813D15520A1F838
:10FAC00050008320A1F85200AF20A1F85400A420D8
:10FAD000A1F85600FF20A1F85800B1F88000A1F865
:10FAE0005A007047B1F8A600012806D191F85800D5
:10FAF00000F07F00A1F858007047022806D191F865
:10FB0000580000F07F00A1F858004BE0032812D104
:10FB100091F8580000F07F00A1F8580091F85600C5
:10FB200000F07F00A1F8560091F8540000F07F002B
:10FB3000A1F85400704704283AD191F8580000F019
:10FB40007F00A1F8580091F8560000F07F00A1F85E
:10FB5000560091F8540000F07F00A1F8540091F88D
:10FB6000520000F07F00A1F8520070470C280AD123
:10FB7000B1F8A60001EB400090F8541001F07F01AD
:10FB8000A0F8541070470D280AD1B1F8A60078B932
:10FB9000B1F85600FF2805D1C020A1F8560001E0B9
:10FBA0000E2805D191F8560000F07F00A1F856000C
:10FBB0007047DFF8CC05B0F8A410012946D1D0F881
:10FBC000C430C3F38003002B1CBFB0F88430B3F5FE
:10FBD000A57F3BD0DFF8B8C50023ACF8003090F823
:10FBE0007E3013F003030CD1B0F8A630012B2DD1D9
:10FBF00000EB430393F858C00CF07F0CA3F858C0F7
:10FC000024E0012B09D1B0F8A630FBB990F85830A8
:10FC100003F07F03A0F8583018E0022B0AD1B0F8A7
:10FC2000A63000EB430393F856C00CF07F0CA3F80A
:10FC300056C00BE0032B09D1B0F8A63000EB43030C
:10FC400093F854C00CF07F0CA3F854C0DFF844358F
:10FC50001B68C3F300139BB10C2901BFDFF83825E3
:10FC60001268C2F38002002A00D049B9B0F8A63069
:10FC700000EB430393F8560000F07F00A3F8560012
:10FC80007047F0B5DFF8F844B4F8A400B4F8846025
:10FC90000546012D81B040F09280D4F8C410C1F324
:10FCA0008001002900F08B80B6F5A57F50D1FF219F
:10FCB000DFF8E824A4F852101268A4F85410D3070F
:10FCC0004CBFEF23DF23A4F852309707B4F852302B
:10FCD000A4F858104CBF4FF6FB774FF6FD773B402A
:10FCE000A4F85230A4F8561053074CBFEF23DF237B
:10FCF000A4F854301707B4F854304CBF4FF6FB77D4
:10FD00004FF6FD773B40A4F85430D3064CBFEF23A9
:10FD1000DF23A4F856309706B4F856304CBF4FF6A0
:10FD2000FB774FF6FD773B4051064CBFEF21DF21BB
:10FD3000A4F858101206B4F85810A4F856304CBF66
:10FD40004FF6FB724FF6FD721140A4F8581036E0E2
:10FD500094F87E1011F003010CD1B4F8A61001291B
:10FD60002DD104EB410191F8562002F07F02A1F859
:10FD7000562024E0012909D1B4F8A610F9B994F865
:10FD8000561001F07F01A4F8561018E002290AD19C
:10FD9000B4F8A61004EB410191F8542002F07F0260
:10FDA000A1F854200BE0032909D1B4F8A61004EB04
:10FDB000410191F8522002F07F02A1F85220DFF8B1
:10FDC000D4130968C1F3001199B10C2D01BFDFF8FC
:10FDD000C8130968C1F38001002900D048B9B4F8FC
:10FDE000A61004EB410191F8540000F07F00A1F847
:10FDF0005400A6F6340028281CD2012D1AD1DFF8B1
:10FE0000500D00EB4600B0F8500000F00F010F2934
:10FE100004D1B4F8720000F01BF80BE0C00609D55D
:10FE2000B4F8720040F2E7318842ACBFFF20BF2037
:10FE3000A4F8520040F65C00864207DB012D05D194
:10FE4000B4F8720001B0BDE8F04001E001B0F0BDCF
:10FE5000B0F5805FCA490FF2C80224DBC31200EB81
:10FE600013531B13A0EB033032F81330A1F85230B8
:10FE70004FEAE01C00EB1C6C4FEA2C2C32F81C30D3
:10FE8000A1F85430A0EB0C20C31000EB13731B112E
:10FE900032F813C0A1F856C0A0EB031032F81000DE
:10FEA000A1F858007047FF23FF281CDDA1F852304D
:10FEB0004FEAE01C00EB1C6C4FEA2C2C32F81C3093
:10FEC000A1F85430A0EB0C20C31000EB13731B11EE
:10FED00032F813C0A1F856C0A0EB031032F810009E
:10FEE000A1F8580070471028A1F85230A1F85430FA
:10FEF0000EDBC31000EB13731B1132F813C0A1F813
:10FF000056C0A0EB031032F81000A1F8580070475B
:10FF1000A1F8563032F81000A1F8580070470000E0
:10FF2000C000F900A400B000990092008200F8001F
:10FF30008000900088008300C600A10086008E002B
:10FF400010B5DFF8CC0A016829B10021016000205A
:10FF5000DFF8C01A0860DFF8C04A2068172808BF19
:10FF600011F0DAF9DFF8EC2B85481268B0F8A4102C
:10FF7000C2F34002002A40F08180864A1268C2F330
:10FF800000127AB30C2921D0491CB0F8A020DFF868
:10FF9000C83B89B2921C91421A60C0F2868000214F
:10FFA0000022C0F8C420D0F8C82022F00402C0F813
:10FFB000C820A0F8A41078490A68D30705D55208CC
:10FFC00052000A606421A0F8841010BD0021DFF8FF
:10FFD0008C2B116070490A6822F004020A603849CB
:10FFE0000988E6E72268142A1CBF152A162A09D0B8
:10FFF000062A2FD10F2927D1DFF8642B0621118083
:020000040801F1
:10000000012133E00F2915D1DFF8541B0A800021AC
:100010000122C0F8C420D0F8C82022F00402C0F8A1
:10002000C8200A00C5D1D0F8C42042F40072C0F83C
:10003000C420BEE7491CB0F8A020DFF81C3B89B201
:10004000921C91421A600FDBDFF8141B09882160B3
:100050000F21DDE7491CB0F8A020DFF8FC3A89B297
:10006000921C91421A60D2DA0129D1D10222C0F841
:10007000C420D0F8C82042F00402D0E70F29DFF8EE
:10008000E03A0ED12268012A18BF1A8007D11988D8
:100090002160D0F8C81041F00401C0F8C810012157
:1000A00006E0198821600F217AE701297FF478AFF3
:1000B0000222C0F8C420D0F8C82042F0040276E73B
:1000C000980A002000B581B0FAF77CFE3349002081
:1000D0000860DFF8901A0860DFF88C1A0860DFF813
:1000E0008C1A0860DFF8881A0860DFF8881A086040
:1000F000DFF8841A0860DFF8841A0860DFF8801AD5
:100100000860DFF8801A0860DFF87C1A0860DFF802
:100110007C1A0860DFF8781A086000F051FD184971
:10012000DFF8703AA020A1F884000020DFF8681AF8
:100130000880DFF8681A0880DFF8641A08804FF634
:10014000FF70DFF8901AB1F8E22082181A60DFF829
:10015000543A1A60B1F89E31B1F83621022B1BBF18
:10016000B1F8381100298018801ADFF83C1A0860AD
:1001700001B0DFF8380A016821F00901016000BD13
:1001800080200020EA640020F0640020C462002087
:10019000E86400209C0E0020140F00204062002024
:1001A0002DE9F04FDFF8089A0020A9F8740081B01B
:1001B000D9F8C800C0F38001002900F046814FF053
:1001C000640E4FF48271C9F8C41020F00401B9F82C
:1001D0008400DFF8005ADFF8DC69DFF8DC79C9F861
:1001E000C8108446BCFBFEFE1FFA8EFEBEF1160F41
:1001F00028BF4FF0150E0246642435F81230A9F8D6
:100200007230BCFBF4FC1FFA8CFCBEF1000F04FB47
:100210001C2C4FF0000834D01EF0030400F00B80BB
:1002200037F802AB36F802BBAAEB0B0A0AF1010A57
:10023000641ED044F4D15FEA9E0E22D037F8024B00
:1002400036F802ABA4EB0A04641CA04437F8024B56
:1002500036F802ABA4EB0A04641CA04437F8024B46
:1002600036F802ABA4EB0A04641CA04437F8024B36
:1002700036F802ABA4EB0A04641CBEF1010EA044E4
:10028000DCD10CEB0806DFF8D078B6B23E6006EBA6
:1002900046077E00DFF8FC7D3E60A0F63400DFF804
:1002A0001C7907EB460728287E88A9F87660FC8829
:1002B000BE88A9F87A403C89A9F87C407F8914D28D
:1002C00005EB4200B0F85000044604F00F0EBEF1FA
:1002D0000F0F0AD0C0064CBF40F2CE7640F2E73690
:1002E00004F00F00072808BF012740F2BE20824219
:1002F000A9F87E7017D1B5F8D00003280ED1B5F853
:10030000CE00382806DBA9F87860A9F8883001B05B
:10031000BDE8F08F0120A9F87600F4E7F3DAB5F82C
:10032000CE004C28EEE7B2F5377F0DD1B5F8D000FE
:10033000032803DA7820A9F87600E4E7E3D14FF444
:100340009670A9F87600DEE7992A25D1B5F8D00095
:1003500003280ED1B5F8CE0040F23A718842D2DBC4
:1003600041F27070A9F87800A9F8883001B0BDE8B2
:10037000F08FC8DAB5F8CE00B0F5B97FC3DB40F234
:100380003A718842ECDA42F22830A9F87800A9F8EC
:10039000883001B0BDE8F08F40F25920824210D180
:1003A000B5F8BC040128AED1B5F8D4000228AADB08
:1003B00041F28830A9F87800A9F8883001B0BDE88A
:1003C000F08F40F25A20824219BF40F25B208242F5
:1003D000B5F8BC04012804D1B5F8D4000228A8BFA0
:1003E0006426682AA9F8786009D1DFF8AC0C0068A7
:1003F000C9F8CC00A9F8883001B0BDE8F08F672AB1
:10040000F3D06C2A0CD1C1F3001000287FF47DAF2B
:100410000020A9F88830A9F8720001B0BDE8F08F7B
:10042000652A0AD00C2A18BF0D2A7FF46EAFDFF8B8
:100430006C0C0078C0073FF568AF0020A9F8883041
:10044000A9F8720001B0BDE8F08FB9F8A410012935
:1004500040F0DB820221C9F8C41040F00403B9F86F
:100460008400B9F87210C9F8C8300246642A38D13D
:10047000DFF86057288B814215D1DFF8206C376890
:100480006A8B47F0010142F2B827BA4205D10C222B
:10049000A9F88420A9F8720004E00D20A9F88400CE
:1004A000A9F872203160B5F8D600012840F0AD827D
:1004B000B9F87200B0F5EC6F1CBFB5F8D8108842DF
:1004C00006D143F01000C9F8C80001B0BDE8F08FB4
:1004D000C3F30010002840F098826420A9F884003B
:1004E0008DE2652A25D140F2DF72914209D143F0B5
:1004F0004000C9F8C80001B00A20A9F88400BDE88E
:10050000F08F0129C3F380120CD1002A00F077820A
:1005100023F04000C9F8C80001B06420A9F88400A5
:10052000BDE8F08F002A40F07082002900F06D8253
:1005300065E2B9F888508D4200F0678213F05004EC
:10054000DFF8586B04D1DFF88C56B5F8D65035B9C2
:100550000C2A18BF0D2A02D03578ED071ED5376852
:10056000FD0740F149820C2A18BF0D2A40F0448251
:10057000DFF8605624B9B5F8D670002F40F04582F8
:10058000A02A08BF012935D1DFF8147B3F68C7F3E3
:1005900000177FBB01B0BDE8F04F93E50E2AE7D10D
:1005A000C3F38010002800F03082012940F02D8232
:1005B000002140F2E320FAF765FB4FF43170A9F80F
:1005C00084000020A9F886000021B9F88400FAF719
:1005D00059FBFAF7D0FBB9F88400401CA9F8840055
:1005E00080B2B0F5357FECDB0E20A9F8840001B0B5
:1005F000BDE8F08F99F87E7007F03004DFF8587589
:100600003C60DFF89C7A3F68C7F30017B7B36CBB58
:10061000A9F88610FAF736FBFAF7ADFBB9F88400B3
:1006200040F2853188420FD101210022002311437D
:10063000194316D140F28631884240F0F480DFF849
:10064000B01C01200880FAE0002140F2873290427D
:1006500008BF0122EAD00022B0F5627FE6D1012373
:10066000E5E7DFF88C1C01200880DCE00F20A9F80A
:10067000A4000220DFF898130860D4E0002C18BF13
:10068000102C64D0202C03D1C3F38013002B5ED137
:1006900040F263239A4273D1B5F8D020032A6FDB6E
:1006A000A9F88610FAF7EEFAB9F8840040F2213181
:1006B000884203D100F0B2F900F02EFEB9F88400B0
:1006C000682818BF67280BD100F0A8F900F078FA65
:1006D00000F0E8FC00F020FEDFF8181C0020088085
:1006E000B9F88400E52808BFFBF794F9B9F884004D
:1006F000F4F74CFCB9F88400E42808BFFBF706F8CF
:10070000B9F88400E62804BFB5F8CC01012804D16B
:1007100006214FF46270FAF7B5FAB9F88410B9F807
:10072000720040F22A32914202BFDFF8CC1B096806
:10073000032922D141F2707188420ED14FF4E67143
:1007400040F22230FAF79EFA4FF4E16111E0B2F57F
:10075000487FA5D125F8121071E041F28831884216
:100760000BD14FF4BE7140F22230FAF78BFA40F20F
:10077000B45140F22530FAF785FAFAF7FCFA05E0B1
:100780000F20A9F8A4000120A1490860B9F884004D
:10079000CB280CD1DFF8642B00211160DFF8602B2F
:1007A0001160DFF8602B1160DFF85C2B1160CB2843
:1007B00018BFCC2803D0CF2818BFCA280DD1DFF826
:1007C000EC130A6822F009020A603168DFF83C2B5A
:1007D00021F48061316000211160B0F5FA7F06D10B
:1007E000DFF8C813086820F00900086027E0D02867
:1007F00018BFCA28F4D040F22331884204D1DFF870
:10080000101B002008801AE040F2263188421CBFED
:1008100040F227318842F2D0B0F54A7F1CBF40F247
:1008200029318842EBD0B9F88400DB2807D1DFF802
:10083000E40AB9F87210026861F34922026002F01A
:1008400097FAB9F8840040F28532904214D101221F
:10085000002300271A433A4303D140F286329042E4
:1008600003D1DFF88C3A01221A803268D30714D5FD
:100870000C280ED10D2010E0002240F28733984260
:1008800008BF0123E5D00023B0F5627FE1D1012745
:10089000E0E75108490064203160A9F8840040F67F
:1008A0008401B9F88400884206D199F8721089074A
:1008B00044BF0021A9F8A81083280DD10020A9F871
:1008C00086000021E120FAF7DDF9B9F88610E22070
:1008D000FAF7D8F9FAF74FFAB9F8840071284FF609
:1008E000FF7106D1B5F8E220AA4B8A181A60AD4B09
:1008F0001A609B280FD1B5F89E61B5F83631AA4A27
:10090000022E08BFCB1815D0B5F83861002E0CBFE9
:10091000CB18CB1A13609C280DD1B5F89E21022A62
:1009200009D0B5F83861B5F836319F4A002E0CBFB2
:10093000CB18CB1A1360CF2816D1B5F8E220954B0F
:100940008A181A60974B1A60B5F89E61B5F836316F
:10095000954A022E08BFC91805D0B5F83851002DA8
:100960000CBFC918C91A11606B2805D1D9F8C81075
:1009700021F05001C9F8C810CB2804BFB9F87200A3
:100980000A2808D10821DFF8200D16F001F8DFF859
:100990001C1D56200880B9F88400C8280ED1B9F86B
:1009A0007200032818BF042808D10821DFF8F80CCA
:1009B00015F0EEFFDFF8F41C56200880B9F884002B
:1009C000C9280ED1B9F87200032818BF042808D12D
:1009D0000821DFF8D40C15F0DBFFDFF8D01C56201F
:1009E0000880B9F88400D0280FD1DFF8C41C00209B
:1009F0000860DFF8C01C07E07808400030600F2076
:100A0000A9F8A40001200249086001B0BDE8F08FF8
:100A100098620020D4630020940A00202DE9F04160
:100A20004B4DDFF8D408B5F8D060DFF8DC2D066058
:100A3000012EDFF8640613680168B5F8424618BF56
:100A4000022E40D1B5F8CE80DFF8C06D01270A250F
:100A5000D6F828C0D6F800E0E04508BF3946BEFB0E
:100A6000F5FEA64505D2AE46BCFBFEFEA64528BF58
:100A70003B4607F1010E376DB84508BF7146BCFB18
:100A8000F5FCA44505D2AC46B7FBFCFCA44528BF49
:100A900073460EF1010CD6F878E0F04508BF6146C8
:100AA000B7FBF5F7A74205D20A27BEFBF7F7A74227
:100AB00028BF63460CF101077836162FC8D31360A0
:100AC0000160BDE8F081032E3DD1B5F8CE80DFF89E
:100AD0005C6E01275FF00A05D6F828C0D6F800E062
:100AE000E04508BF3946BEFBF5FEA64505D2AE4639
:100AF000BCFBFEFEA64528BF3B4607F1010E376D45
:100B0000B84508BF7146BCFBF5FCA44505D2AC4610
:100B1000B7FBFCFCA44528BF73460EF1010CD6F8C8
:100B200078E0F04508BF6146B7FBF5F7A74205D26C
:100B30000A27BEFBF7F7A74228BF63460CF101075F
:100B40007836132FC8D313600160BDE8F081000030
:100B500038430020A00E0020AC0E0020B46300201B
:100B60000A65002044620020486200204C62002098
:100B70005062002054620020586200205C62002015
:100B80006062002064620020686200206C620020C5
:100B900070620020C40E0020980A00209A0A0020EB
:100BA0009C0A0020C80E0020CC0E0020980E0020C9
:100BB00080200020D49102087C9102080092020853
:100BC0002DE9F0430348DFF8CC44B0F8D010DFF84B
:100BD000606D01E038430020DFF8585D2160012995
:100BE000B0F8CE00306018BF022981B040F0E38039
:100BF000DD2840F2252840F2072740F215194BDA8C
:100C00003220A5F8860032217220FAF73BF8B5F8B9
:100C100086107320FAF736F8B5F886104846FAF7CA
:100C200031F8B5F886104FF48B70FAF72BF8B5F859
:100C300086107D20FAF726F8B5F886107E20FAF7A0
:100C400021F800BFB5F88610B8B2FAF71BF87F1C80
:100C50004745F7D35020A5F8860050217420FAF7B5
:100C600011F8B5F886107520FAF70CF8B5F886106B
:100C700040F21710FAF706F8B5F886104FF48C70AA
:100C8000FAF700F8206802280CBF05200720A5F815
:100C90008600B5F8861078E140F23B71884244DA6C
:100CA0004FF49670A5F8860001467220F9F7EAFF26
:100CB000B5F886107320F9F7E5FFB5F886104846B9
:100CC000F9F7E0FFB5F886104FF48B70F9F7DAFF0B
:100CD000B5F886107D20F9F7D5FFB5F886107E208F
:100CE000F9F7D0FFB5F88610B8B2F9F7CBFF7F1C43
:100CF0004745F7D34FF4FA70A5F8860001467420F3
:100D0000F9F7C0FFB5F886107520F9F7BBFFB5F805
:100D1000861040F21710F9F7B5FFB5F886104FF4BA
:100D20008C70F9F7AFFF04202CE14FF41670A5F892
:100D3000860001467220F9F7A5FFB5F886107320EA
:100D4000F9F7A0FFB5F886104846F9F79BFFB5F80C
:100D500086104FF48B70F9F795FFB5F886107D205B
:100D6000F9F790FFB5F886107E20F9F78BFF00BFEA
:100D7000B5F88610B8B2F9F785FF7F1C4745F7D361
:100D80004FF46170A5F8860001467420F9F77AFFE8
:100D9000B5F886107520F9F775FFB5F8861040F2A2
:100DA0001710F9F76FFFB5F886104FF48C70F9F74C
:100DB00069FF0320E6E0032940F09B80B0F5C87F7F
:100DC00048DC3220A5F8860032217220F9F75AFF5C
:100DD000B5F886107320F9F755FFB5F8861040F284
:100DE0001510F9F74FFFB5F886104FF48B70F9F72F
:100DF00049FFB5F886107D20F9F744FFB5F8861055
:100E00005FF07E00F9F73EFF40F2072740F2252809
:100E1000B5F88610B8B2F9F735FF7F1C4745F7D310
:100E20005020A5F8860050217420F9F72BFFB5F863
:100E300086107520F9F726FFB5F8861040F21710D6
:100E4000F9F720FFB5F886104FF48C70F9F71AFF08
:100E5000072097E040F6B93188424ADA4FF496709D
:100E6000A5F8860001467220F9F70CFFB5F8861048
:100E70007320F9F707FFB5F8861040F21510F9F75F
:100E800001FFB5F886104FF48B70F9F7FBFEB5F84B
:100E900086107D20F9F7F6FEB5F886105FF07E002B
:100EA000F9F7F0FE40F2072740F22528B5F8861042
:100EB000B8B2F9F7E7FE7F1C4745F7D34FF4FA7055
:100EC000A5F8860001467420F9F7DCFEB5F8861017
:100ED0007520F9F7D7FEB5F8861040F21710F9F72C
:100EE000D1FEB5F886104FF48C70F9F7CBFE0620D2
:100EF00048E04FF41670A5F8860001467220F9F715
:100F0000C1FEB5F886107320F9F7BCFEB5F886105F
:100F100040F21510F9F7B6FEB5F886104FF48B7055
:100F2000F9F7B0FEB5F886107D20F9F7ABFEB5F8FD
:100F300086107E20F9F7A6FE40F2072740F225280A
:100F4000B5F88610B8B2F9F79DFE7F1C4745F7D378
:100F50004FF46170A5F8860001467420F9F792FEFF
:100F6000B5F886107520F9F78DFEB5F8861040F2B9
:100F70001710F9F787FEB5F886104FF48C70F9F763
:100F800081FE0520A5F8860001468A20F9F77AFE41
:100F90002068012818BF022825D13068B0F5C87F25
:100FA0000ADD40F2EF218842B8BF40F6B83008DBD6
:100FB00040F69901884202DA4FF47A6001E04FF47A
:100FC000FA60A5F886009920B5F88610F9F75AFE60
:100FD0004FF49670A5F88600014640F22B30F9F7E1
:100FE00051FE32202EE003281BD1306840F2EF2161
:100FF00088420DDA4FF47A60A5F886000146992000
:10100000F9F740FE4FF47A70A5F88600014614E027
:1010100040F69901884204DA40F6B831A5F8861006
:1010200004E04FF47A60A5F8860001469920F9F7AC
:1010300029FE40F2DC51A5F8861040F22B30F9F77A
:1010400021FE4620A5F88600014640F24630F9F719
:1010500019FE5F20A5F886005F2140F24730F9F7BE
:1010600011FE2068032808BF8C2004D0012818BF77
:10107000022807D18220A5F88600014640F26120AF
:10108000F9F700FEFAF7C6FC01B0BDE8F043F9F746
:1010900072BE0000F8620020E40A0020140F002055
:1010A0009C0E002070B5944D2868012818BF0228B6
:1010B00073D1DFF8844ADFF8846A206800EB80018E
:1010C000C800315889B26620F9F7DCFD206800EBD2
:1010D0008001C800315889B24FF49B70F9F7D2FDF6
:1010E000206800EB8001480006EB80000A21406880
:1010F000B0FBF1F189B240F22130F9F7C3FDFFF7FF
:101100008DFC2868012807D1206800EB8001480089
:1011100006EB8000816806E0022809D1DFF8200A8A
:10112000216850F8211089B240F23A30F9F7AAFD4F
:10113000206800EB8001480006EB8000C16889B29E
:1011400040F22330F9F79EFD2068DFF8F82900EB24
:101150008001480006EB8000016A1160416A89B293
:101160004FF44E70F9F78EFDC8214FF43770F9F740
:1011700089FD4FF4D77140F2DD20F9F783FD4FF47C
:10118000BE7140F26320F9F77DFDDC2140F2223090
:10119000F9F778FD4FF4BE7174E00328DFF870565C
:1011A00040F08680DFF89049DFF89C69206800EB0A
:1011B0008001C800315889B26620F9F763FD2068C4
:1011C00000EB8001C800315889B24FF49B70F9F7E9
:1011D00059FD206800EB8001480006EB80000A21E1
:1011E0004068B0FBF1F189B240F22130F9F74AFDD5
:1011F000FFF714FC206800EB8001480006EB80003C
:10120000816889B240F23A30F9F73CFD206800EB82
:101210008001480006EB8000C16889B240F22330AB
:10122000F9F730FD2068DFF81C2900EB8001480049
:1012300006EB8000016A1160416A89B24FF44E707A
:10124000F9F720FD4FF4BE714FF43770F9F71AFD2E
:10125000B5F8CA01022818BF042835D04FF44871E8
:1012600040F2DD20F9F70EFD4FF42F7140F26320BC
:10127000F9F708FD4FF4BE7140F22230F9F702FD94
:101280004FF42F714FF41E70F9F7FCFC40F223303D
:10129000F3F77CFEDFF87855B5F8D00004281CDAA7
:1012A000B5F8CE0040F2EE21884210DA022115E0B6
:1012B0000428EBD14FF4C8714FF43770F9F7E2FC12
:1012C000B5F8CA010228C9D140F22A31C8E740F274
:1012D0003B718842B8BF0A2100DB142140F269202B
:1012E000F9F7D0FC00F0E8F9BDE87040F9F743BD2C
:1012F000642000200C150020E8610020D00E0020A2
:10130000C00E0020BC0E002050630020BC630020F3
:10131000880A0020100F00202DE9F041DFF82C088A
:10132000DFF8EC440068012818BF022840F08A80EA
:10133000DFF8D454DFF80468286800EB8001480027
:1013400006EB8000016989B240F22630F9F79AFC79
:10135000286800EB8001480006EB8000416989B2F3
:1013600040F22730F9F78EFC286800EB8001480036
:1013700006EB8000816989B24FF44A70F9F782FC6C
:101380002868DFF8B05500EB8001480006EB8000CC
:10139000C16989B240F22930F9F774FCB4F8D4007D
:1013A000062802D100F054F93BE0B4F842160529B2
:1013B00040F22E3640F2333740F22F3840F22D30D3
:1013C0000BDA1421A5F88610F9F75CFCB5F8861045
:1013D0004046F9F757FC14200AE06421A5F886106E
:1013E000F9F750FCB5F886104046F9F74BFC282079
:1013F000A5F8860001463846F9F744FC1420A5F804
:10140000860014213046F9F73DFCB5F886104FF4FC
:101410004C70F9F737FCB5F886104FF44D70F9F7BA
:1014200031FCB4F842160529B4BF3C212821A5F8A7
:10143000861040F24930F9F725FC6420A5F88600B3
:101440006421D8E0032840F0DA80DFF8BC53DFF8ED
:10145000F866286800EB8001480006EB800001690F
:1014600089B240F22630F9F70DFC286800EB8001C4
:10147000480006EB8000416989B240F22730F9F755
:1014800001FC286800EB8001480006EB80008169C0
:1014900089B24FF44A70F9F7F5FB286800EB800138
:1014A000480006EB8000C16989B240F22930F9F7A3
:1014B000E9FBB4F8D400062802D100F0C9F881E0B5
:1014C000B4F84216DFF86C54052940F22E3640F28B
:1014D000333740F22F3840F22D3012DA1421A5F8BC
:1014E0008610F9F7CFFBB5F886104046F9F7CAFB2E
:1014F0001420A5F8860014213846F9F7C3FB142000
:101500004CE0102914DA6421A5F88610F9F7BAFB2B
:10151000C820A5F88600C8214046F9F7B3FB28206B
:10152000A5F8860028213846F9F7ACFB502035E0B5
:1015300017290BDAC821A5F88610F9F7A3FBB5F82F
:1015400086104046F9F79EFB282020E01739352900
:101550000ED24FF4C871A5F88610F9F793FBC82096
:10156000A5F88600C8214046F9F78CFB32200EE032
:101570004FF44871A5F88610F9F784FB4FF4167004
:10158000A5F8860001464046F9F77CFBC820A5F87F
:10159000860001463846F9F775FB6420A5F88600F9
:1015A00001463046F9F76EFB1420A5F88600142199
:1015B0004FF44C70F9F766FBB5F886104FF44D7098
:1015C000F9F760FBB4F8420601461729B8BF3C2181
:1015D00007DB1738352838BF282102D34C2904DB14
:1015E0001C2140F24930F9F74DFBB4F8420625289A
:1015F000B4BF642150214FF44F70F9F743FBB4F8A6
:101600004206B0F5FA6F40F2433540F242360ADB4B
:101610000F214FF43870F9F735FBC8213046F9F740
:1016200031FBC82109E005214FF43870F9F72AFB96
:1016300032213046F9F726FB32212846F9F722FB02
:10164000F9F799FBDFF84C1B00200880BDE8F0811A
:1016500010B5B84CC820A4F88600C82140F22D303F
:10166000F9F710FBB4F8861040F22F30F9F70AFBB7
:10167000B4F8861040F23330F9F704FB1420A4F8D4
:101680008600142140F22E30F9F7FCFAB4F88610E7
:101690004FF44C70F9F7F6FAB4F88610BDE8104034
:1016A0004FF44D70F9F7EEBA0010014054200020BD
:1016B000040F0020000F0020554800B5B0F8D010EE
:1016C000032981B040F08D80B0F8CE004B28C0F2E5
:1016D00088804C280BDA3C2140F27730F9F7D2FAB7
:1016E00028214FF45E70F9F7CDFA962184E06F2837
:1016F0000BDA462140F27730F9F7C4FA46214FF46D
:101700005E70F9F7BFFA822176E097280BDA5A214A
:1017100040F27730F9F7B6FA32214FF45E70F9F7FC
:10172000B1FA962168E0DD280BDA6E2140F27730BD
:10173000F9F7A8FA5A214FF45E70F9F7A3FA5A2183
:101740005AE0B0F5C87F06DC962140F27730F9F711
:1017500099FA6E214BE040F2272188420BDAB4213E
:1017600040F27730F9F78EFA6E214FF45E70F9F798
:1017700089FA502140E040F2EF2188420BDA9621AD
:1017800040F27730F9F77EFA82214FF45E70F9F774
:1017900079FA782130E040F24D41884206DABE21E4
:1017A00040F27730F9F76EFA6E2120E040F2DD5119
:1017B00088420BDABE2140F27730F9F763FA322122
:1017C0004FF45E70F9F75EFA5A2115E040F23B7172
:1017D000884206DAD22140F27730F9F753FAD22163
:1017E00005E0962140F27730F9F74CFA64214FF486
:1017F0005E70F9F747FA642101B05DF804EB40F23E
:101800007930F9F73FBA0000E80A0020D4C702088F
:101810003843002010B50EF0F9F9DFF87C090068B4
:10182000C0F34001002901BFDFF870190988C1F336
:101830008001002978D1DFF868190988012973D15E
:10184000DFF86019B1F8D420042A18BF052A05D0A2
:10185000B1F84036062A08BF032B03D1BDE810407B
:10186000F2F76ABD73B1DFF840291268C2F30012C3
:1018700042B9DFF83819012008800020DFF8141978
:10188000088010BDDFF828291268C2F30022002A60
:101890004AD0DFF814291268C2F30012CAB9DFF87F
:1018A00014090068632809D12249DFF80C290020B7
:1018B000A1F88A00106840F4005034E0B1F8A001AB
:1018C000002802BFDFF8F008007810F0840F2BD159
:1018D0001AE0DFF8E4281368C3F3001424B3C0F35C
:1018E000C00000281CBFC3F38030002809D0114974
:1018F0000020A1F88A001946012060F34E311160E2
:1019000010BDB1F8A00178B9B1F8900101001CBF79
:101910000228042808D1DFF8A028DFF8A0181068F2
:10192000084040F00100106010BD0000C8CB020864
:10193000FC6200208020002030B5DFF88448B4F835
:10194000A4000F2881B018D1DFF84C180968C1F342
:10195000400129B1DFF86C180120088001B030BDCA
:10196000DFF86418098841B1DFF8601801200880A9
:1019700001B00020A4F8A40030BDDFF82C5829687D
:10198000C1F3001121B1DFF848281278012A5DD097
:10199000012815D1D4F8C400C0F34000B0B3D4F886
:1019A000C800DFF8301880F02000C4F8C8000978BB
:1019B00089074FD520F02000C4F8C80001B030BD21
:1019C000A9B9DFF8F4170978C90710D4DFF80818A7
:1019D0000A68143A0F2804D1042A02D20FF09CFCA2
:1019E00003E0042A3CBF002008600FF057FEB4F863
:1019F000A400002802BF2868C0F30010002802BF1E
:101A0000DFF8B407007810F0850F1FD1B4F8841008
:101A1000B4F87400A1F63402401C282AA4F874001B
:101A20000CD2DFF8802702EB410191F8501001F051
:101A30000F010F2902D080B2032801E080B20428F0
:101A400008D10020A4F8740001B030BD01B0BDE899
:101A5000304001E001B030BD70B4DFF84807B0F8A5
:101A600092110A001CBF0229042963D1DFF86C1708
:101A70000968C1F3001119B9B0F84618002959D105
:101A8000DFF82427DFF830171268C2F3001222B102
:101A90000B6843F002030B6009E0DFF8FC361C68BA
:101AA00024F0C0041C600323DFF8344723800B6854
:101AB0005C086400DFF82C370C601D68C5F3001665
:101AC00016B145F400751D60DFF8CC361D6825F0B1
:101AD00004051D6024F00403DFF80C570B6000249C
:101AE0002C60DFF808472468B4F5827F18BFB4F58E
:101AF000017F09D0DFF8F8462468032C02BFDFF825
:101B0000F4462468042C15D1B0F8E803022811D15A
:101B100012B143F020000860086820F4E07008600B
:101B20000020DFF8D4160880DFF8D0160880DFF830
:101B3000D016088070BC7047E40A0020D0C70208A5
:101B400068CB02089C0D0020C4CB0208E86100208D
:101B50002DE9F04FDFF86886DFF84866B8F8A40092
:101B60000025012881B006F1D00440F0A181D8F809
:101B7000C400C0F34001002900F0AD80D8F8C800CF
:101B8000C0F340110029B8F884103FD16422B1FBA2
:101B9000F2F2DFF87076DFF8700692B23A606423F2
:101BA00030F812005A43DFF864361A60491C41F2DB
:101BB0000813A8F88410F35C9B071CD540F6340387
:101BC00089B2994217DB40F65B0040F65C0107E002
:101BD0007F1CA8F88470BFB28F42A8BFA8F88420E9
:101BE000B8F8847006EB470EBEF850E0BEF1000F67
:101BF00001D19F42ECD1DFF818160860B8F88410C4
